:100000000C9446160C9477160C9477160C9477166D
:100010000C9477160C9477160C9477160C9477162C
:100020000C9477160C9477160C9477160C9477161C
:100030000C9477160C9455590C9477160C947716EB
:100040000C9477160C944DC40C9477160C94771678
:100050000C9477160C9477160C9480760C940B59AC
:100060000C9477160C94BE4B0C9477160C94771660
:100070000C9477160C9477160C9477160C947716CC
:100080000C9477160C9477160C9477160C947716BC
:100090000C9477160C9477160C9477160C947716AC
:1000A0000C9477160C9477160C9477160C9477169C
:1000B0000C9477160C9477160C9477160C9477168C
:1000C0000C9477160C9477160C9477160C9477167C
:1000D0000C9477160C9477160C9470580C94315835
:1000E0000C9477168731A431D531F2310732303292
:1000F0009D320333AC33F4370238FB3722382638CD
:1001000040389B3C5538A138C838EF3818396E391B
:100110007F399039A139B239C3399B3CA63B9B3C0E
:10012000B13B213C273C473C00B103B1F2B0F6B0F3
:10013000FCB03AB107B10BB111B115B119B11FB192
:1001400023B127B13AB12DB131B135B19AB69FB6CD
:10015000A4B6AEB6B8B631B7C2B6CAB6D2B6DCB679
:10016000E6B6F0B6FFB609B731B713B71DB727B774
:10017000084AD73B3BCE016E84BCBFFDC12F3D6C0E
:1001800074319ABD56833DDA3D00C77F11BED9E474
:10019000BB4C3E916BAAAABE000000803F05A84C54
:1001A000CDB2D44EB93836A9020C50B99186880820
:1001B0003CA6AAAA2ABE000000803F004E414E493C
:1001C0004E495459494E46CDCCCC3D0AD7233C1715
:1001D000B7D13877CC2B329595E6241FB14F0A0062
:1001E0000020410000C84200401C4620BCBE4CCA52
:1001F0001B0E5AAEC59D74434F4D4D554E4943415C
:1002000054494F4E0044525952554E004552524F98
:10021000525300494E464F004543484F0047322F46
:1002200047332062616420706172616D657465722C
:10023000730A00206F6620004D424C20473239205F
:10024000706F696E74200059206F7574206F66207E
:1002500072616E67652028312D35292E0A005820DD
:100260006F7574206F662072616E67652028312D6E
:1002700035292E0A004D6573682070726F62696EB1
:100280006720646F6E652E0A005374617274206D6E
:100290006573682070726F62696E67207769746831
:1002A0002022473239205331222066697273742E1E
:1002B0000A004732380A47323920533200537461FA
:1002C00074653A20004D65736820626564206C6532
:1002D00076656C696E6720686173206E6F2064615B
:1002E00074612E0A0053206F7574206F662072614E
:1002F0006E67652028302D35292E0A004D657368FC
:1003000020706F696E742063616E6E6F7420626519
:10031000207265736F6C7665640A00456E642066B2
:10032000696C65206C6973740A00426567696E20A8
:1003300066696C65206C6973740A00286E6F2066AC
:10034000696C6529005344207072696E74696E6728
:10035000206279746520004E6F74205344207072BF
:10036000696E74696E670A0043757272656E7420F7
:1003700066696C653A20002569730025696D202542
:100380006973002569682025696D2025697300253A
:100390006964202569682025696D20256973002519
:1003A000697920256964202569682025696D2025E3
:1003B0006973005072696E742074696D653A20002B
:1003C0006F6E2E0A006F66662E0A00473236204492
:1003D000656275672000180213020C020502F7011E
:1003E0006F66660044454255473A004B494C4C45C0
:1003F000442E20004D3131332053006F6B002C20F0
:10040000002C2000544845524D414C5F50524F54EF
:10041000454354494F4E004155544F5245504F5259
:10042000545F53445F53544154555300454D455216
:1004300047454E43595F5041525345520043415343
:10044000455F4C494748545F4252494748544E45DE
:10045000535300544F47474C455F4C49474854530A
:1004600000534F4654574152455F504F5745520035
:100470004255494C445F50455243454E54004C450B
:1004800056454C494E475F44415441005A5F5052D3
:100490004F4245004155544F4C4556454C00505233
:1004A000494E545F4A4F420050524F4752455353B2
:1004B000004155544F5245504F52545F54454D5092
:1004C00000564F4C554D45545249430045455052F6
:1004D0004F4D0053455249414C5F584F4E5F584F66
:1004E0004646004649524D574152455F4E414D45A3
:1004F0003A4D61726C696E20312E312E39202847B9
:1005000069746875622920534F555243455F434FC4
:1005100044455F55524C3A68747470733A2F2F6794
:1005200069746875622E636F6D2F4D61726C696EB0
:100530004669726D776172652F4D61726C696E20CC
:1005400050524F544F434F4C5F56455253494F4EB4
:100550003A312E30204D414348494E455F54595061
:10056000453A3344205072696E7465722045585480
:1005700052554445525F434F554E543A31205555DC
:1005800049443A63656465326132662D34316132C3
:100590002D343734382D396231322D633535633699
:1005A000326633363766660A002F2F20002054004B
:1005B000205200416363656C65726174696F6E3AC5
:1005C0002050005741524E494E4721204C6F772012
:1005D0005A204A65726B206D6179206C65616420D8
:1005E000746F20756E77616E7465642070617573C9
:1005F00065732E0A00546F6F206661722066726FF9
:100600006D207265666572656E636520706F696ED8
:10061000740A0020466C6F773A20000001363726B6
:10062000032BFFFFFF3C3D382AFFFFFFFF2E303E2C
:1006300012FFFFFFFFFFFFFF0809FF2C071A1C181E
:10064000FFFFFF08440A2C4324221E20643A0020A6
:10065000693A0020703A00496E76616C69642065E1
:10066000787472756465720A0043290A0061626CCD
:10067000656420286D696E2074656D702000436F7D
:100680006C6420657874727564657320617265208E
:100690000020643A0020693A0020703A004E6F2032
:1006A00063617365206C696768740A004545505240
:1006B0004F4D204F4B0A00205A004475616C204575
:1006C0006E6473746F702041646A7573746D656EC7
:1006D0007420286D6D293A20003F4B2076616C759F
:1006E00065206F7574206F662072616E67652028C3
:1006F000302D3130292E0A00416476616E63652009
:100700004B3D004163746976652045787472756469
:1007100065723A2000496E76616C69642065787470
:1007200072756465720A0043616E6E6F7420656E47
:10073000746572207375626469723A2000473931BA
:100740000A4731205A2D302E30320A4739300053B3
:1007500070656369616C204D656E753A205A20445E
:100760006F776E20302E310A004739310A47312029
:100770005A2D302E30320A47393000537065636984
:10078000616C204D656E753A205A20446F776E205B
:10079000302E30320A004739310A4731205A2B3087
:1007A0002E30320A473930005370656369616C201E
:1007B0004D656E753A205A20557020302E30320A21
:1007C000004739310A4731205A2B302E310A473938
:1007D00030005370656369616C204D656E753A2019
:1007E0005A20557020302E310A00473239205332BA
:1007F000005370656369616C204D656E753A204EDB
:10080000657874204D65736820506F696E740A00B6
:10081000473239205331005370656369616C204D54
:10082000656E753A205374617274204D657368204B
:100830004C6576656C696E670A004D313430205323
:100840003630005370656369616C204D656E753A92
:100850002050726568656174204265640A004D35F8
:100860003031005370656369616C204D656E753A77
:10087000205265616420454550524F4D0A004D3568
:100880003030005370656369616C204D656E753A58
:10089000205361766520454550524F4D0A004D3337
:1008A000303320452D312053363020433130205510
:1008B00031005370656369616C204D656E753A2037
:1008C0004175746F2054756E6520486F746265645D
:1008D000205069640A004D31303620533137380AD0
:1008E0004D333033204530205332313020433130C6
:1008F000205531005370656369616C204D656E75DC
:100900003A204175746F2054756E6520486F746588
:100910006E64205049440A003C5370656369616C01
:100920005F4D656E753E003C5370656369616C5F39
:100930004D656E753E002F002F002F002F2E2E0AC2
:10094000002F2E2E002F2E2E003C53706563696100
:100950006C5F4D656E753E0A003C5370656369615E
:100960006C204D656E753E003C5370656369616C2B
:10097000204D656E753E003C5265616420454550D2
:10098000524F4D3E003C5265616420454550524FE8
:100990004D3E003C4175746F2054756E6520486F64
:1009A00074626564205049443E003C4175746F2078
:1009B00054756E6520486F74626564205049443EEA
:1009C000003C4175746F2054756E6520486F7465E6
:1009D0006E64205049443E003C4175746F2054754C
:1009E0006E6520486F74656E64205049443E003C3B
:1009F000457869743E003C457869743E003C53611B
:100A0000766520454550524F4D3E003C536176651A
:100A100020454550524F4D3E003C4E657874204D68
:100A200065736820506F696E743E003C4E65787443
:100A3000204D65736820506F696E743E003C53749E
:100A4000617274204D657368204C6576656C696EC3
:100A5000673E003C5374617274204D657368204C8E
:100A60006576656C696E673E003C507265686561CD
:100A700074206265643E003C507265686561742054
:100A80006265643E003C5A20446F776E20302E3100
:100A90003E003C5A20446F776E20302E313E003CA1
:100AA0005A20446F776E20302E30323E003C5A2060
:100AB000446F776E20302E30323E003C5A20557005
:100AC00020302E30323E003C5A20557020302E30DF
:100AD000323E003C5A20557020302E313E003C5AA8
:100AE00020557020302E313E0056313136004A33C9
:100AF0003320004D3530300A4D3432302053310A26
:100B00004731205A313020463234300A473120589C
:100B100030205930204636303030004A3232004AD8
:100B20003232004731205A3520463234300A4731BC
:100B30002058313930205932302046363030300A92
:100B40004731205A302046323430004731205A3560
:100B500020463234300A473120583139302059315B
:100B600039302046363030300A4731205A3020465E
:100B7000323430004731205A3520463234300A476B
:100B8000312058313930205932302046363030301B
:100B90000A4731205A302046323430004739310A72
:100BA0004731205A313020463234300A4739300A32
:100BB0004732380A4732390A4731205832302059F3
:100BC00032302046363030300A4731205A30204605
:100BD000323430004A3032004A3132004731205A34
:100BE0003130004F4B004731205A31300047393007
:100BF00000473120452569463530300047312045D2
:100C00002D302E314625690047312045302E3146A2
:100C10002569004731205A2569462569004731205A
:100C20005A2D302E31462569004731205A302E3159
:100C30004625690047312059256946256900473115
:100C400020592D302E314625690047312059302E4C
:100C500031462569004731205825694625690047F6
:100C60003120582D302E314625690047312058302B
:100C70002E31462569004739310047323800473266
:100C800038205A004732382059004732382058005F
:100C90004132305620004731205A3130004A30343A
:100CA000004A3231004A3230004B494C4C45442E08
:100CB00020004A303400454E4400464E20004A3061
:100CC00032003939393A393939004D004800413755
:100CD000562000413656202D2D2D004A303200413D
:100CE000365620005A3A2000593A2000583A20003F
:100CF00041355600413456200041335620004132E0
:100D0000562000413156200041305620004D3834E5
:100D1000004A3136004A3138004739310A4731201C
:100D20005A313020463234300A473930004A3134A3
:100D3000004A3030004A3031004A31300024F4D4C7
:100D40003050C38E20C2A24017828B7011127A914C
:100D50000D816CD90AA861E108C758660761514343
:100D6000061E4B5D05C145A7041A411104093D98B3
:100D700003713931034036DB0265339102D43054BC
:100D800002802E1D02632CEE01752AC501B028A039
:100D900001102781018F2564012B244B01E02234AF
:100DA00001AC211F018D200D01801FFC00841EED70
:100DB00000971DDF00B81CD200E61BC600201BBC3C
:100DC00000641AB200B219A8000A19A0006A1899A2
:100DD00000D117910040178B00B516840031167EA4
:100DE00000B31579003A157300C7146F0058146AE0
:100DF00000EE1366008813630025135E00C7125BC4
:100E0000006C12570015125400C111510070114F9F
:100E10000021114B00D61049008D104700461044A8
:100E20000002104200C00F4000800F3E00420F3C05
:100E300000060F3B00CB0E3800930E37005C0E35DA
:100E400000270E3400F30D3200C10D3100900D303B
:100E500000600D2E00320D2D00050D2C00D90C2B3D
:100E600000AE0C2900850C29005C0C2700350C27EE
:100E7000000E0C2600E80B2400C40B2400A00B235A
:100E8000007D0B23005A0B2100390B2100180B2089
:100E900000F80A1F00D90A1E00BB0A1E009D0A1D89
:100EA00000800A1D00630A1C00470A1B002C0A1B55
:100EB00000110A1A00F7091A00DD091900C40919FE
:100EC00000AB091900920917007B09180063091784
:100ED000004C09160036091600200916000A0915EB
:100EE00000F5081500E0081400CC081400B8081438
:100EF00000A4081400900813007D0812006B08136A
:100F00000058081200460812003408110023081186
:100F1000001208110001081100F0071000E007108E
:100F200000D0071000C0071000B0070F00A1071085
:100F30000091070E0083070F0074070F0065070E6E
:100F40000057070E0049070E003B070D002E070E45
:100F50000020070D0013070D0006070D00F9060C11
:100F600000ED060D00E0060C00D4060C00C8060CCF
:100F700000BC060C00B0060C00A4060B0099060C81
:100F8000008D060B0082060B0077060B006C060B2B
:100F90000061060A0057060B004C060A0042060ACA
:100FA0000038060A002E060A0024060A001A060A5D
:100FB000001006090007060A00FD050900F40509EE
:100FC00000EB050900E2050900D9050900D0050973
:100FD00000C7050900BE050900B5050800AD0508F4
:100FE00000A50509009C050800940508008C05086B
:100FF00000840508007C050800740508006C0507DE
:1010000000650508005D050700560508004E050748
:1010100000470507004005080038050700310507AF
:10102000002A050700230507001C05060016050712
:10103000000F0507000805060002050700FB04066F
:1010400000F5040700EE040600E8040600E20407C9
:1010500000DB040600D5040600CF040600C9040620
:1010600000C3040600BD040600B7040600B1040571
:1010700000AC040600A6040600A00405009B0406BC
:101080000095040500900406008A04050085040507
:1010900000800406007A040500750405007004054C
:1010A000006B04050066040500610405005C04058E
:1010B0000057040500520405004D040500480405CE
:1010C00000430405003E0404003A0405003504050D
:1010D00000300404002C0405002704040023040548
:1010E000001E0404001A0404001604050011040480
:1010F000000D0404000904050004040400000404B5
:1011000000FC030400F8030400F4030400F00304EB
:1011100000EC030400E8030400E4030400E003041B
:1011200000DC030400D8030400D4030400D003044B
:1011300000CC030400C8030300C503030024F40427
:10114000D9201BC40C5C0E9804C4095F02650771AA
:1011500001F405F900FB04B30048048700C10369EA
:10116000005803550003034500BE023A00840231D3
:101170000053022A002902250004022000E4011C79
:1011800000C8011900AF0117009801140084011371
:1011900000710110006101100051010E0043010DAA
:1011A0000036010B002B010B0020010B001501097B
:1011B000000C01090003010800FB000800F300080F
:1011C00000EB000700E4000600DE000600D8000681
:1011D00000D2000600CC000500C7000500C20005D3
:1011E00000BD000400B9000400B5000400B1000413
:1011F00000AD000400A9000400A5000300A2000344
:10120000009F0004009B000300980003009500026B
:101210000093000300900003008D0002008B000388
:1012200000880002008600020084000300810002A2
:10123000007F0002007D0002007B000200790002B6
:1012400000770001007600020074000200720001C5
:1012500000710002006F0002006D0001006C0002CE
:10126000006A0001006900020067000100660001D9
:1012700000650001006400020062000100610001DD
:1012800000600001005F0002005D0001005C0001E1
:10129000005B0001005A00010059000100580001E4
:1012A00000570001005600010055000100540001E4
:1012B00000530000005300010052000100510001E2
:1012C00000500001004F0001004E0000004E0001E0
:1012D000004D0001004C0001004B0000004B0001DC
:1012E000004A0001004900010048000000480001D8
:1012F00000470001004600000046000100450000D4
:1013000000450001004400010043000000430001CB
:1013100000420000004200010041000000410001C5
:1013200000400001003F0000003F0001003E0000BF
:10133000003E0001003D0000003D0001003C0000B7
:10134000003C0000003C0001003B0000003B0001AD
:10135000003A0000003A00010039000000390001A5
:10136000003800000038000000380001003700009D
:101370000037000100360000003600000036000192
:101380000035000000350000003500010034000089
:10139000003400000034000100330000003300007E
:1013A0000033000100320000003200000032000172
:1013B0000031000000310000003100010030000069
:1013C0000030000000300001002F0000002F00005E
:1013D000002F0000002F0001002E0000002E000052
:1013E000002E0001002D0000002D0000002D000047
:1013F000002D0001002C0000002C0000002C00003B
:10140000002C0001002B0000002B0000002B00002E
:10141000002B0001002A0000002A0000002A000022
:10142000002A000100290000002900000029000016
:101430000029000000290001002800000028000009
:1014400000280000002800000028000100270000FC
:1014500000270000002700000027000000270001EF
:1014600000260000002600000026000000260000E4
:1014700000260001002500000025000000250000D6
:1014800000250000002500000025000100240000C8
:1014900000240000002400000024000000240001BB
:1014A00000230000002300000023000000230000B0
:1014B00000230000002300000023000100220000A0
:1014C0000022000000220000002200000022000094
:1014D0000022000100210000002100000021000086
:1014E0000021000000210000002100000021000177
:1014F000002000000020000000200000002000006C
:10150000002000000020000000200000002000015A
:10151000001F0000001F0000001F0000001F00004F
:10152000001F0000001F0000001F0001001E00003F
:10153000001E0000001E0000001E000000232C0002
:1015400000B8220000561800003A0F0000B808004A
:1015500000B1040000710200003E010000696E202D
:101560006D6F76655F746F282920666565645F76A8
:10157000616C756520666F722058593A002C2065A1
:10158000793D0029202D3E202865783D002C2073D0
:10159000793D0020436F6E6E656374696E672077D6
:1015A00069746820766572746963616C206C696E19
:1015B00065202873783D002C2065793D0029202D79
:1015C0003E202865783D002C2073793D0020436F34
:1015D0006E6E656374696E67207769746820686FE2
:1015E00072697A6F6E74616C206C696E6520287305
:1015F000783D003F53706563696669656420582CC7
:101600005920636F6F7264696E617465206F7574C1
:10161000206F6620626F756E64732E0A003F285239
:101620002965706561742076616C7565206E6F74D4
:1016300020706C61757369626C653B206D757374A5
:10164000206265206174206C6561737420312E0AFC
:10165000003F2852296570656174206D7573742090
:101660006265207370656369666965642077686583
:101670006E206E6F74207573696E6720616E204CEA
:1016800043442E0A003F53706563696669656420B0
:101690006E6F7A7A6C652074656D706572617475B1
:1016A0007265206E6F7420706C61757369626C6511
:1016B0002E0A003F53706563696669656420666938
:1016C0006C616D656E742073697A65206E6F74202D
:1016D000706C61757369626C652E0A003F537065AA
:1016E000636966696564207072696D65206C656EFA
:1016F000677468206E6F7420706C61757369626CBA
:10170000652E0A003F5072696D65206C656E6774C6
:1017100068206D75737420626520737065636966F7
:10172000696564207768656E206E6F7420757369D3
:101730006E6720616E204C43442E0A003F53706553
:10174000636966696564206E6F7A7A6C6520736977
:101750007A65206E6F7420706C61757369626C6558
:101760002E0A003F5370656369666965642052659F
:101770007472616374696F6E204D756C7469706CFE
:10178000696572206E6F7420706C61757369626C2C
:10179000652E0A003F52657472616374696F6E2032
:1017A0004D756C7469706C696572206D7573742009
:1017B0006265207370656369666965642E0A003F1F
:1017C000537065636966696564206C617965722030
:1017D000686569676874206E6F7420706C617573DA
:1017E00069626C652E0A003F5370656369666965BE
:1017F00064206265642074656D70657261747572D1
:1018000065206E6F7420706C61757369626C652001
:101810002834302D31343043292E0A004732362007
:10182000636F6D6D616E6420737461727465642E94
:101830002057616974696E6720666F722068656100
:101840007465722873292E0A00024A3135004A3124
:1018500032004A3137002020506C616E6E65724252
:10186000756666657242797465733A200020467227
:101870006565204D656D6F72793A2000436F6D701C
:10188000696C65643A204465632031372032303119
:10189000380A00207C20417574686F723A202864F1
:1018A0006176696472616D69726F2C20666F722057
:1018B000416E796375626963206933204D656761A4
:1018C000290A00323031382D31322D313300204C8D
:1018D00061737420557064617465643A2000312E20
:1018E000312E390A004D61726C696E0020536F66AB
:1018F00074776172652052657365740A00205761C0
:10190000746368646F672052657365740A002042CF
:10191000726F776E206F75742052657365740A005C
:101920002045787465726E616C2052657365740A27
:1019300000506F77657255700A0073746172740A93
:10194000004D3234004D3233202573006175746FC1
:1019500025692E67006572726F72207772697469EB
:101960006E6720746F2066696C650A00205A3A0021
:1019700020593A0020583A00656E6473746F707392
:10198000206869743A2000446F6E6520736176693F
:101990006E672066696C652E0A004D32390020742E
:1019A0006F6F206C6F6E6720657874727573696FE6
:1019B0006E2070726576656E7465640A0020636FD0
:1019C0006C6420657874727573696F6E20707265CF
:1019D00076656E7465640A00454550524F4D20642B
:1019E00061746173697A65206572726F722E0A0084
:1019F000290A002062797465733B206372632000BA
:101A000053657474696E67732053746F72656420D4
:101A10002800290A002062797465733B2063726391
:101A200020002073746F7265642073657474696E2E
:101A3000677320726574726965766564202800207A
:101A40002863616C63756C6174656429210A0020E8
:101A5000213D2000454550524F4D20435243206DBB
:101A600069736D61746368202D202873746F7265CB
:101A7000642920002053697A653A2000496E646524
:101A8000783A2000204D61726C696E3D56353529DB
:101A90000A0028454550524F4D3D00454550524F94
:101AA0004D2076657273696F6E206D69736D617418
:101AB000636820001000C90210012C0140012201BE
:101AC00070011801B0010E01F00104015002FA008A
:101AD000B002F0003003E600D003DC009004D20036
:101AE0007005C800A006BE000008B400B009AA0036
:101AF000D00BA000600E960060118C0000158200D3
:101B000020197800C01D6E00A0226400B0275A0082
:101B1000902C500000314600E0343C001038320078
:101B2000903A2800603C1E00A03D1400803E0A0050
:101B3000203F00002CFFFFFFFFFF0001010101011A
:101B40006265640A002C2073797374656D20737468
:101B50006F7070656421204865617465725F4944E7
:101B60003A20004265642068656174696E6720668A
:101B700061696C65640048656174696E67206661BF
:101B8000696C65640045312048656174696E672041
:101B90006661696C65640048656174696E6720669A
:101BA00061696C65640070012C0190012701B0012E
:101BB0002201C0011D01F0011801100213013002C1
:101BC0000E016002090190020401C002FF0000033F
:101BD000FA004003F5008003F000D003EB0020047E
:101BE000E6007004E100E004DC004005D700C00519
:101BF000D2004006CD00D006C8008007C3003008E0
:101C0000BE00F008B900C009B400B00AAF00B00BC4
:101C1000AA00D00CA500000EA000500F9B00C01021
:101C200096005012910000148C00C0158700B01768
:101C30008200B0197D00D01B7800001E7300402088
:101C40006E0090226900F024640040275F00902914
:101C50005A00E02B5500102E500020304B0010325F
:101C60004600E033410090353C00103737007038B3
:101C70003200A0392D00B03A2800A03B2300603C80
:101C80001E00103D1900903D1400103E0F00703EE4
:101C90000A00C03E0500003F0000403FFBFF803FC0
:101CA000F6FFC03FF1FF453120544845524D414CAD
:101CB0002052554E41574159004245442054484511
:101CC000524D414C2052554E415741590054686580
:101CD000726D616C2052756E6177617900453120BB
:101CE0004572723A204D415854454D50004572722C
:101CF0003A204D415854454D5020424544004D41F5
:101D00005854454D50207472696767657265640068
:101D10004531204572723A204D494E54454D500090
:101D20004572723A204D494E54454D50204245442B
:101D3000004D494E54454D50207472696767657275
:101D40006564004D383420582059205A2045002021
:101D50002F002042403A0020403A006F70656E200C
:101D60006661696C65642C2046696C653A200043A5
:101D7000616E6E6F74206F70656E2073756264693A
:101D80007220004A3035004A3233004739310A4761
:101D900031205A2D313020463234300A4739300054
:101DA00053442063617264206F6B0A006F70656E2C
:101DB000526F6F74206661696C65640A00766F6C9F
:101DC000756D652E696E6974206661696C65640A5B
:101DD000004572726F723A00534420696E69742034
:101DE0006661696C0A006563686F3A00205A3A00C0
:101DF00020593A0020436F756E7420583A002045F0
:101E00003A00205A3A0020593A00583A003A004322
:101E100061703A00205A00205900580020204D617E
:101E2000783A2000205A00205900580020204D699F
:101E30006E3A20004F6E20004F666600536F667446
:101E400020656E6473746F70733A20004B642000D9
:101E500023646566696E652044454641554C545F70
:101E6000004B69200023646566696E652044454621
:101E700041554C545F004B70200023646566696EC9
:101E8000652044454641554C545F0050494420412B
:101E900075746F74756E652066696E6973686564C4
:101EA000212050757420746865206C617374204B18
:101EB000702C204B6920616E64204B6420636F6E30
:101EC0007374616E74732066726F6D2062656C6FDF
:101ED0007720696E746F20436F6E666967757261F3
:101EE00074696F6E2E680A00504944204175746F02
:101EF00074756E65206661696C6564212074696D16
:101F0000656F75740A00453120544845524D414C67
:101F10002052554E415741590042454420544845AE
:101F2000524D414C2052554E41574159005468651D
:101F3000726D616C2052756E617761790045312058
:101F400048656174696E67206661696C656400420A
:101F500065642068656174696E67206661696C6597
:101F6000640048656174696E67206661696C6564C8
:101F700000504944204175746F74756E6520666128
:101F8000696C6564212054656D7065726174757249
:101F90006520746F6F20686967680A00204B643A97
:101FA0002000204B693A2000204B703A20000A2084
:101FB000436C617373696320504944200A002054C4
:101FC000753A2000204B753A2000206D61783A2048
:101FD00000206D696E3A200020643A20002062697A
:101FE00061733A2000504944204175746F74756ED6
:101FF00065206661696C65642120426164206578B2
:10200000747275646572206E756D6265720A005037
:102010004944204175746F74756E652073746172E4
:10202000740A004F66660A00466164652048656967
:102030006768742000426564204C6576656C696E43
:102040006720004661696C656420746F20656E616D
:10205000626C6520426564204C6576656C696E67CC
:102060000A004D65736820426564204C6576656C96
:1020700020646174613A0A004D65736820706F696D
:102080006E742063616E6E6F74206265207265737A
:102090006F6C7665640A004D34323120696E636F6F
:1020A000727265637420706172616D65746572200F
:1020B00075736167650A00656E7175657565696E32
:1020C000672022004B494C4C45442E200050726939
:1020D0006E7465722073746F7070656420647565CA
:1020E00020746F206572726F72732E20466978209B
:1020F000746865206572726F7220616E64207573FA
:1021000065204D39393920746F207265737461729E
:10211000742E202854656D70657261747572652027
:1021200069732072657365742E2053657420697419
:102130002061667465722072657374617274696E71
:1021400067290A004E6F20436865636B73756D20C5
:1021500077697468206C696E65206E756D62657252
:102160002C204C617374204C696E653A20004E6FD0
:1021700020436865636B73756D2077697468206CA4
:10218000696E65206E756D6265722C204C6173748A
:10219000204C696E653A2000636865636B73756DEA
:1021A000206D69736D617463682C204C61737420B9
:1021B0004C696E653A20004C696E65204E756D6203
:1021C0006572206973206E6F74204C617374204CAB
:1021D000696E65204E756D6265722B312C204C61E5
:1021E0007374204C696E653A20004D313130004DDA
:1021F00033310053442072656164206572726F72DE
:102200000A00446F6E65207072696E74696E672093
:1022100066696C650A007C3C3E5E2B3D3F2F5B5D32
:102220003B2C2A225C00627573793A2070617573C9
:10223000656420666F7220696E7075740A0062753D
:1022400073793A2070617573656420666F722075CA
:102250007365720A00627573793A2070726F6365F4
:102260007373696E670A004A3135004B494C4C451F
:10227000442E20004B494C4C2063617573656420EB
:102280006279204B494C4C20627574746F6E2F70CC
:10229000696E0A004B494C4C45442E20004B494C7A
:1022A0004C2063617573656420627920746F6F20C0
:1022B0006D75636820696E61637469766520746901
:1022C0006D65202D2063757272656E7420636F6D6D
:1022D0006D616E643A20004A3131005072696E744B
:1022E00065722068616C7465642E206B696C6C2863
:1022F000292063616C6C6564210A000000A0C000A5
:10230000000000000000005761726E696E673A209D
:10231000486F6D696E672042756D702044697669FB
:10232000736F72203C20310A000202040000A040BA
:102330000000A040000000400000614300005C433A
:1023400000004D43FFFFFF20496E76616C696420F9
:10235000657874727564657220000000A0C000008A
:1023600000000000000000005C4300005C4300002F
:102370004D43486F6D696E67206661696C656400E6
:10238000206E6F7420656E74657265642E0A004657
:10239000696C652064656C657465643A0044656CBD
:1023A0006574696F6E206661696C65642C2046698E
:1023B0006C653A200050726F7465637465642050D8
:1023C000696E0A004A3036004A3034004A3037001D
:1023D00020573A004A3038004A30390020573A0036
:1023E00000002100240027002A002D0030003300C7
:1023F00001010000040107010A010000220025007C
:1024000028002B002E0031003400020100000501DD
:1024100008010B01000020002300260029002C00E9
:102420002F0032000001000003010601090105052B
:102430000505070508080808020202020A0A08083A
:102440000404040401010101010101010303030368
:1024500003030303040707070C0C0C0C0C0C0C0CF7
:102460000202020206060606060606060B0B0B0B08
:102470000B0B0B0B0102102020080810204010202D
:102480004080020102010804020101020408102038
:102490004080804020100804020180040201804036
:1024A000201008040201080402010102040810209F
:1024B0004080010204081020408000000A0B02093D
:1024C0000C0D0E08070304010000000000000000CE
:1024D00000000000000000000000000000000000FC
:1024E00000000000000012111000000000000000B9
:1024F00000000000000000000000000000000000DC
:10250000556E6B6E6F776E20636F6D6D616E643AA2
:102510002022002066697273740A005A005900581C
:1025200000486F6D652000000048420000484200EE
:10253000008040000000005452494747455245443E
:10254000006F70656E003A20007A325F6D696E0030
:102550007A5F6D696E00795F6D696E00785F6D6995
:102560006E005265706F7274696E6720656E647379
:10257000746F70207374617475730A000A4D65611D
:10258000737572656420706F696E74733A0A005ACD
:10259000206F66667365743A20004E756D20582C66
:1025A000593A20352C350A000000000100000001D6
:1025B00000008000555555000000400033333300C3
:1025C000AAAA2A004992240000002000C7711C001A
:1025D00099991900D1451700555515003BB11300C5
:1025E0002449120011111100000010000F0F0F00FC
:1025F000E3380E0043790D00CCCC0C00C3300C0046
:10260000E8A20B0064210B00AAAA0A00703D0A0090
:102610009DD80900427B090092240900DCD3080000
:10262000888808001042080000000800F0C1070078
:102630008787070075500700711C07003EEB0600F6
:10264000A1BC06006990060066660600703E0600A2
:102650006118060017F4050074D105005BB0050091
:10266000B2900500627205005555050078390500E5
:10267000B81E0500050505004EEC040087D40400D3
:10268000A1BD040090A7040049920400C17D04008C
:10269000EE690400C7560400444404005C320400A0
:1026A0000821040041100400000004003FF0030072
:1026B000F8E0030026D20300C3C30300CCB5030037
:1026C0003AA803000A9B0300388E0300C081030070
:1026D0009F750300D0690300505E03001D53030083
:1026E00034480300913D03003333030016290300EF
:1026F000381F030097150300300C03000303030089
:102700000BFA020049F10200BAE802005CE00200A4
:102710002DD802002DD0020059C80200B0C002001E
:1027200031B90200DAB10200AAAA0200A0A3020095
:10273000BC9C0200FA9502005C8F0200DF88020058
:1027400082820200457C0200277602002770020088
:10275000436A02007C640200D05E02003F5902001E
:10276000C853020048617264636F64656420446505
:102770006661756C742053657474696E6773204C60
:102780006F616465640A00B80B0000B80B00003C80
:10279000000000102700000000FA430000FA430088
:1027A00000C040000070420000A0420000A04200B3
:1027B00000C8433333B94220286D6D290020204DD5
:1027C000393030204B004C696E656172204164766F
:1027D000616E63653A0A0020440020490020204DC4
:1027E00033303420500020440020490020204D3355
:1027F00030312050005049442073657474696E670D
:10280000733A0A00205A0020204D36363600456EB5
:102810006473746F702061646A7573746D656E742F
:102820003A0A00205A00205900202047323920530C
:1028300033205800205A0020204D343230205300DD
:102840004D65736820426564204C6576656C696EE1
:10285000673A0A00205A0020590020204D323036B5
:10286000205800486F6D65206F66667365743A0A7C
:1028700000204500205A0020590020580020540014
:1028800020530020204D32303520510020453C6D32
:1028900061785F655F6A65726B3E0020583C6D61D0
:1028A000785F785F6A65726B3E20593C6D61785F36
:1028B000795F6A65726B3E205A3C6D61785F7A5F22
:1028C0006A65726B3E00416476616E6365643A20AE
:1028D000513C6D696E5F7365676D656E745F746999
:1028E0006D655F75733E20533C6D696E5F6665650F
:1028F00064726174653E20543C6D696E5F747261F0
:1029000076656C5F66656564726174653E0020542F
:102910000020520020204D323034205000416363AB
:10292000656C65726174696F6E2028756E69747369
:102930002F7332293A20503C7072696E745F616364
:1029400063656C3E20523C726574726163745F61B2
:102950006363656C3E20543C74726176656C5F61A4
:102960006363656C3E0A00204500205A0020590030
:1029700020204D3230312058004D6178696D756DE1
:1029800020416363656C65726174696F6E202875A0
:102990006E6974732F7332293A0A00204500205A59
:1029A0000020590020204D3230332058004D6178EE
:1029B000696D756D20666565647261746573202844
:1029C000756E6974732F73293A0A00204500205AE6
:1029D0000020590020204D39322058005374657072
:1029E000732070657220756E69743A0A0020204D5C
:1029F0003230302044300A0020204D323030204424
:102A0000002044697361626C65640A0046696C6108
:102A10006D656E742073657474696E67733A002017
:102A200020473231202020203B00FFFDFCFAF8F641
:102A3000F4F2F0EEECEAE9E7E5E3E1E0DEDCDAD936
:102A4000D7D5D4D2D0CFCDCBCAC8C7C5C3C2C0BFDB
:102A5000BDBCBAB9B7B6B4B3B2B0AFADACAAA9A851
:102A6000A6A5A4A2A1A09E9D9C9A9998979594939F
:102A700092908F8E8D8B8A898887868483828180CD
:102A80007F7E7D7B7A797877767574737271706FDB
:102A90006E6D6C6B6A696867666564636261605FCE
:102AA0005E5D5C5B5A5958585756555453525150B5
:102AB000504F4E4D4C4B4A4A494847464645444381
:102AC000424241403F3E3E3D3C3B3B3A393838373D
:102AD000363535343332323130302F2E2E2D2C2BEB
:102AE0002B2A29292827272625252423232221218B
:102AF00020201F1E1E1D1C1C1B1B1A19191818171D
:102B00001616151514131312121111100F0F0E0EA5
:102B10000D0D0C0C0B0A0A09090808070706060523
:102B200005040403030202010000526573656E642C
:102B30003A20006F6B0020746F6F206C6F6E6720FF
:102B4000657874727573696F6E2070726576656EE4
:102B50007465640A0020636F6C6420657874727514
:102B600073696F6E2070726576656E7465640A00B5
:102B70004572726F722077726974696E6720746F24
:102B800020454550524F4D210A0057726974696EB5
:102B90006720746F2066696C653A20006F70656EFF
:102BA000206661696C65642C2046696C653A20007A
:102BB0006F70656E206661696C65642C2046696C77
:102BC000653A200046696C652073656C65637465C1
:102BD000640A002053697A653A200046696C6520D2
:102BE0006F70656E65643A20002066696C653A20F6
:102BF00000646F696E67006672657368004E6F7778
:102C00002000454E4420535542524F5554494E459D
:102C10000A002220706F73002220706172656E744A
:102C20003A2200535542524F5554494E4520434194
:102C30004C4C207461726765743A22004B494C4CCD
:102C400045442E2000747279696E6720746F20638A
:102C5000616C6C207375622D67636F6465206669B3
:102C60006C6573207769746820746F6F206D616E76
:102C700079206C6576656C732E204D4158206C650B
:102C800076656C2069733A00C4DF7AE111241FBEB7
:102C9000CFEFD1E2DEBFCDBF00E00CBF14E0A0E07B
:102CA000B2E0EEEAFCED01E00BBF02C007900D922E
:102CB000A431B107D9F728E1A4E1B4E001C01D9225
:102CC000A83CB207E1F716E1C5E4D6E100E006C092
:102CD00021970109802FFE010E94AFEDC434D10776
:102CE00080E00807A9F70E9424DA0C9446EE0C94C1
:102CF00000002F923F924F925F926F927F928F923D
:102D00009F92AF92BF92CF92DF92EF92FF920F937A
:102D10001F93CF93DF93CDB7DEB7CA58D1090FB653
:102D2000F894DEBF0FBECDBF21E020933F1080910D
:102D300015188D3411F40C947721843511F40C940A
:102D40009F2E873411F00C94EB2E809113189091E4
:102D500014188A31910509F4BEC79CF4843091059A
:102D60003CF482309105B4F597FF2DC00C9473218B
:102D70008430910509F4D2C1059709F40EC20C9470
:102D800073218A32910511F40C946A204CF48C3131
:102D9000910509F4A4C74D9709F4A6C70C947321B3
:102DA0008B35910511F40C94F5208C35910511F4B7
:102DB0000C94F9208A35910511F00C94732110922E
:102DC00027040C94ED2E8091270281110C94F22E91
:102DD0000C94ED2E20912702222311F40C94ED2E59
:102DE00011E0029709F010E00E94D6AA19821A8217
:102DF0001B821C821D821E821F82188682E50E9411
:102E0000984C882309F43AC10E94184C4B015C018C
:102E100020E030E0A9010E9467E6882309F444C15C
:102E2000C0903204D0903304E0903404F090350424
:102E3000CCAADDAAEEAAFFAAC0903604D09037042F
:102E4000E0903804F0903904C8AED9AEEAAEFBAEDB
:102E5000C090AE10D090AF10E090B010F090B110D4
:102E6000CCAEDDAEEEAEFFAEC090B210D090B310DF
:102E7000E090B410F090B5102496CCAEDDAEEEAE7E
:102E8000FFAE24972CAD3DAD4EAD5FAD6CA97DA9D5
:102E90008EA99FA90E9467E681110BC0A701960128
:102EA00068AD79AD8AAD9BAD0E9467E6882309F4D1
:102EB000FBC020E030E0A901C501B4010E9467E633
:102EC000881F8827881F181739F0C12CD12C80E85B
:102ED000E82E8FEBF82E06C0C12CD12C00E8E02E96
:102EE0000FE3F02E2C96CCAEDDAEEEAEFFAE2C97FF
:102EF0002CA93DA94EA95FA96CAD7DAD8EAD9FAD4E
:102F00000E94B2EA28966CAF7DAF8EAF9FAF289734
:102F100028AD39AD4AAD5BAD24966CAD7DAD8EADBF
:102F20009FAD24970E94B2EA6B017C0128962CADDC
:102F30003DAD4EAD5FAD2897CA01B9010E94CCE608
:102F40002B013C01A7019601C701B6010E94CCE606
:102F50009B01AC01C301B2010E94B3EA0E941EEDC5
:102F60002B013C0120E030E040E05FE30E94CCE632
:102F700060966CAF7DAF8EAF9FAF6097A501940157
:102F8000C501B4010E94CCE64B015C0160962CADFA
:102F90003DAD4EAD5FAD6097CA01B9010E94CCE670
:102FA0009B01AC01C501B4010E94B2EA0E941EED72
:102FB0002C962CAD3DAD4EAD5FAD2C970E94CCE66E
:102FC0004B015C01C701B6019058A30192010E9418
:102FD0008FEBA50194010E94CCE66B017C012CAD26
:102FE0003DAD4EAD5FAD6CA97DA98EA99FA90E9494
:102FF000B3EA20E030E040E05FE30E94CCE69B01D2
:10300000AC01C701B6010E94B3EA2CA93DA94EA9A3
:103010005FA90E94B2EA69837A838B839C8324969A
:103020002CAD3DAD4EAD5FAD249768AD79AD8AADA9
:103030009BAD0E94B3EA20E030E040E05FE30E94F5
:10304000CCE66B017C01A301920128966CAD7DADAD
:103050008EAD9FAD28970E948FEBA50194010E9431
:10306000CCE69B01AC01C701B6010E94B3EA28ADD2
:1030700039AD4AAD5BAD0E94B2EA12C089E40E944C
:10308000984C882331F00E94184C69837A838B8393
:103090009C838AE40E94984C882331F00E94184C4B
:1030A0006D837E838F83988720E030E0A90169815A
:1030B0007A818B819C810E9467E681110EC020E09D
:1030C00030E0A9016D817E818F8198850E9467E63D
:1030D000811103C0E1EDFDE10DC0412FBE016F5F25
:1030E0007F4F8EEA90E10E94F8A40C94ED2E0E948E
:1030F000EE93F80184918F010F5F1F4F8111F7CF7D
:10310000EDE1F2E084918F010F5F1F4F882311F4EE
:103110000C94ED2E0E94EE93F801F4CF80E50E940E
:10312000984C882379F08091210490912204009793
:1031300049F04AE050E060E070E00E94E6E46B0194
:103140007C0103C0C12CD12C760183E50E94984CF0
:10315000882361F00E94184C20E030E04AE754E4F4
:103160000E94CCE60E94FCEB6B017C010E941F6A6E
:103170000E94FF58C60ED71EE81EF91E0E94FF5877
:10318000DC01CB018C199D09AE09BF09B7FD02C056
:103190000C94ED2E0E942CA1F1CF80912702882360
:1031A00011F40C94ED2E0E94D6AA89E40E94984C4A
:1031B000882329F00E94184C2B013C0103C0412CAC
:1031C000512C32018AE40E94984C882329F00E94F5
:1031D000184C4B015C0103C0812C912C540180E5FB
:1031E0000E94984C882329F00E94184C6B017C01A6
:1031F00003C0C12CD12C760181E50E94984C882314
:1032000039F00E94184C6CAB7DAB8EAB9FAB04C009
:103210001CAA1DAA1EAA1FAA20913E10C657DF4F46
:103220002883CA58D0406091020270910302072E91
:10323000000C880B990B0E946DE6209130023091B2
:10324000310240913202509133020E94CCE62AE0D2
:1032500037ED43E25CE30E94CCE668AB79AB8AAB26
:103260009BAB4091320450913304609134047091CF
:10327000350448AF59AF6AAF7BAF9A01AB01C301C8
:10328000B2010E94B3EAA1966CAF7DAF8EAF9FAF43
:10329000A1974090360450903704609038047090A5
:1032A0003904A3019201C501B4010E94B3EAA596B5
:1032B0006CAF7DAF8EAF9FAFA5972091AE103091D0
:1032C000AF104091B0105091B110C701B6010E94EB
:1032D000B3EAA9966CAF7DAF8EAF9FAFA99720914F
:1032E000B2103091B3104091B4105091B5106CA948
:1032F0007DA98EA99FA90E94B3EAAD966CAF7DAF60
:103300008EAF9FAFAD97C8ACD9ACEAACFBACC9826D
:10331000DA82EB82FC824D825E826F8278860E9426
:10332000FF589B01AC0128533F4F4F4F5F4FCB5786
:10333000DF4F288339834A835B83C558D040BDEC77
:103340008B2EBCEC9B2EA92CBDE3BB2E25961FAE6D
:10335000259729961FAE29972D961FAE2D9761961A
:103360001FAE61970E94D07B0E94FF588B019C0189
:10337000CB57DF4FC880D980EA80FB80C558D0404A
:103380000C191D092E093F0937FD10C09B01AC0126
:1033900028533F4F4F4F5F4FCB57DF4F2883398321
:1033A0004A835B83C558D0400E942CA125967FADEF
:1033B000259729966FAD29972D969FAD2D976196EC
:1033C0008FAD6197272F362F492F582FC501B40194
:1033D0000E94B3EA6CAB78AF8CAF21969FAF219778
:1033E00020E030E040E85FE30E94D9EC181644F496
:1033F0001CAA18AE30E83CAF4FE321964FAF21979F
:103400006091AE107091AF108091B0109091B1109A
:10341000E1966CAF7DAF8EAF9FAFE19780913204A4
:1034200090913304A0913404B0913504E5968CAFAB
:103430009DAFAEAFBFAFE59721969FAD21979F930C
:10344000ACADAF93B8ADBF93ECA9EF93E196ACAC44
:10345000BDACCEACDFACE197A996ECACFDAC0EAD4B
:103460001FADA997A1962CAD3DAD4EAD5FADA19717
:10347000E5966CAD7DAD8EAD9FADE5970E94B2C572
:103480000F900F900F900F9062966FAF62976396B8
:103490007FAF639764968FAF649765969FAF65978C
:1034A000C090B210D090B310E090B410F090B5106E
:1034B000E996CCAEDDAEEEAEFFAEE99720913604D4
:1034C000309137044091380450913904ED962CAF77
:1034D0003DAF4EAF5FAFED9721963FAD21973F9344
:1034E0004CAD4F9358AD5F936CA96F93E996ACAC1C
:1034F000BDACCEACDFACE997AD96ECACFDAC0EAD9F
:103500001FADAD97A5962CAD3DAD4EAD5FADA5976A
:10351000ED966CAD7DAD8EAD9FADED970E94B2C5C1
:103520000F900F900F900F9066966FAF669767960B
:103530007FAF679768968FAF689769969FAF6997D7
:1035400089819A81AB81BC81C358DF4F888399837D
:10355000AA83BB83CD57D040CD80DE80EF80F88436
:10356000CF57DF4FC882D982EA82FB82C158D04050
:103570006A961FAE6A9725967FAD259729966FADFF
:1035800029972D969FAD2D9761968FAD6197272F27
:10359000362F492F582FBCA9A8ADFCAD2196EFAD11
:1035A00021976B2F7A2F8F2F9E2F0E94B2EA2FE642
:1035B00032E143E05BE30E9467E687FD29C125967F
:1035C0007FAD259729966FAD29972D969FAD2D97A5
:1035D00061968FAD6197272F362F492F582FBCA9A1
:1035E000A8ADFCAD2196EFAD21976B2F7A2F8F2FD1
:1035F0009E2F0E94B3EA20E030E040E05FE30E94AB
:10360000CCE6662E972E882E792E9F938F937F93EC
:103610006F93E196ACACBDACCEACDFACE197A996B4
:10362000ECACFDAC0EAD1FADA997A1962CAD3DAD98
:103630004EAD5FADA197E5966CAD7DAD8EAD9FAD06
:10364000E5970E94B2C50F900F900F900F906B9668
:103650006FAF6B976C967FAF6C976D968FAF6D97D2
:10366000C757DF4F9883C958D0407F928F929F925F
:103670006F92E996ACACBDACCEACDFACE997AD9641
:10368000ECACFDAC0EAD1FADAD97A5962CAD3DAD30
:103690004EAD5FADA597ED966CAD7DAD8EAD9FAD9A
:1036A000ED970E94B2C50F900F900F900F90162FBC
:1036B000072FB82EA92E66962FAD669767963FAD59
:1036C000679768964FAD689769965FAD6997CF57D2
:1036D000DF4F688179818A819B81C158D0400E94E7
:1036E000B3EA20E030E040E05FE30E94CCE61B015B
:1036F0002C0162962FAD629763963FAD63976496F7
:103700004FAD649765965FAD6597C358DF4F68818D
:1037100079818A819B81CD57D0400E94B3EA20E015
:1037200030E040E05FE30E94CCE69B01AC016B9689
:103730006FAD6B976C967FAD6C976D968FAD6D97F7
:10374000C757DF4F9881C958D0400E94B2EA6B0139
:103750007C0120E030E0A9010E94D9EC87FF04C081
:10376000F7FAF094F7F8F094A2019101612F702F0D
:103770008B2D9A2D0E94B2EA1B012C0120E030E033
:10378000A9010E94D9EC87FF04C057FA509457F85A
:103790005094A2019101C701B6010E94B3EA2DEC39
:1037A0003CEC4CEC5DE30E9467E618168CF56696DF
:1037B0001FAF669767960FAF67976896BFAE68971B
:1037C0006996AFAE69976B96DFAC6B976296DFAE8A
:1037D00062976C96EFAC6C976396EFAE63976D96BD
:1037E000FFAC6D976496FFAE6497C757DF4F288193
:1037F000C958D04065962FAF65976CAA98AE8CAE2D
:1038000021967FAE219731E06A963FAF6A97B3CE9B
:103810006A964FAD6A97411144C125967FAD2597B1
:1038200029966FAD29972D969FAD2D9761968FADF7
:103830006197272F362F492F582FBCA9A8ADFCAD73
:103840002196EFAD21976B2F7A2F8F2F9E2F0E94FD
:10385000B2EA6B017C012DEC3CEC4CEC5DE30E9488
:10386000D9EC18160CF41DC1A7019601C701B601C9
:103870000E94B3EA2596EFAD25972996BFAD29970B
:103880002D96AFAD2D976196FFAD61972E2F3B2FF3
:103890004A2F5F2F0E94B3EA662E972E882E792E2C
:1038A00020E030E040E85FE30E94D9EC87FFF9C0F8
:1038B0007F928F929F926F92E196ACACBDACCEACF2
:1038C000DFACE197A996ECACFDAC0EAD1FADA997AE
:1038D000A1962CAD3DAD4EAD5FADA197E5966CAD1B
:1038E0007DAD8EAD9FADE5970E94B2C50F900F9054
:1038F0000F900F906A966FAF6A976B967FAF6B973A
:103900006C968FAF6C976D969FAF6D977F928F92ED
:103910009F926F92E996ACACBDACCEACDFACE997B0
:10392000AD96ECACFDAC0EAD1FADAD97A5962CAD34
:103930003DAD4EAD5FADA597ED966CAD7DAD8EAD59
:103940009FADED970E94B2C50F900F900F900F9012
:10395000162F072FB82EA92E262F372F482F592F75
:10396000CF57DF4F688179818A819B81C158D040D0
:103970000E94B3EA20E030E040E05FE30E94CCE642
:103980006B017C016A962FAD6A976B963FAD6B9782
:103990006C964FAD6C976D965FAD6D97C358DF4FCA
:1039A000688179818A819B81CD57D0400E94B3EA9A
:1039B00020E030E040E05FE30E94CCE69B01AC01F8
:1039C00062966FAD629763967FAD639764968FAD95
:1039D000649765969FAD65970E94B2EA1B012C0122
:1039E00020E030E0A9010E94D9EC87FF04C057FA1B
:1039F000509457F85094A701960166966FAD66975C
:103A000067967FAD679768968FAD689769969FAD0B
:103A100069970E94B2EA6B017C0120E030E0A901C5
:103A20000E94D9EC87FF04C0F7FAF094F7F8F094FD
:103A3000A2019101C701B6010E94B3EA2DEC3CEC52
:103A40004CEC5DE30E94D9EC18165CF166961FAF52
:103A5000669767960FAF67976896BFAE6897699647
:103A6000AFAE69976A965FAD6A9762965FAF6297ED
:103A70006B966FAD6B9763966FAF63976C967FADE8
:103A80006C9764967FAF64976D968FAD6D976596D2
:103A90008FAF65976CAA98AE8CAE21967FAE2197BA
:103AA000BCCE25967FAD259729966FAD29972D968B
:103AB0009FAD2D9761968FAD6197272F362F492F98
:103AC000582FBCA9A8ADFCAD2196EFAD21976B2F67
:103AD0007A2F8F2F9E2F0E94B2EA4B015C016296D3
:103AE0008FAD629763969FAD63976496AFAD649711
:103AF0006596BFAD659789839A83AB83BC836696D1
:103B00008FAD669767969FAD67976896AFAD6897DC
:103B10006996BFAD69978D839E83AF83B8877CA973
:103B200068AD9CAD21968FAD2197272F362F492F59
:103B3000582F60E070E080E89FE30E94B2EA6B01DA
:103B40007C0120913A0430913B0440913C04509117
:103B50003D040E94CCE62B013C012091B61030912F
:103B6000B7104091B8105091B910BCA9A8ADFCADE8
:103B70002196EFAD21976B2F7A2F8F2F9E2F0E94CA
:103B8000CCE69B01AC01C301B2010E94B3EA698794
:103B90007A878B879C8720913E0430913F04409127
:103BA000400450914104C701B6010E94CCE66B016C
:103BB0007C012091BA103091BB104091BC10509103
:103BC000BD10BCA9A8ADFCAD2196EFAD21976B2F20
:103BD0007A2F8F2F9E2F0E94CCE69B01AC01C7014C
:103BE000B6010E94B3EA6D877E878F87988BCE01DE
:103BF00001960E94EFC91CA61DA61EA61FA68981BC
:103C00009A81AB81BC8188A399A3AAA3BBA38D8110
:103C10009E81AF81B8858CA39DA3AEA3BFA38985E8
:103C20009A85AB85BC8588A799A7AAA7BBA7AE0133
:103C3000485D5F4FBE016C5D7F4FCE0180960E9454
:103C4000F2BCDE019C966D01C657DF4FE880CA5872
:103C5000D0408E01005D1F4F9E01235F3F4FAE019C
:103C6000485D5F4FBE016C5D7F4FCE0180960E9424
:103C7000FB59882329F120E030E040E85FE3BCA94C
:103C8000A8ADFCAD2196EFAD21976B2F7A2F8F2F2A
:103C90009E2F0E9467E687FF13C03CA925963FAF81
:103CA000259748AD29964FAF29975CAD2D965FAF0C
:103CB0002D9721966FAD219761966FAF619752CB8B
:103CC00080E1EEEAF0E1A2E3B4E001900D928A9582
:103CD000E1F70C94ED2E0E94354E0C94ED2E80E011
:103CE0000E9476AC0C94ED2E83E50E94984C8823BC
:103CF00021F10E94F84B182F863070F0E5EEF2E0CB
:103D000084918F010F5F1F4F882311F40C94ED2EC7
:103D10000E94EE93F801F4CF833009F44AC130F4E5
:103D2000813091F1823009F43FC008C0843009F439
:103D30009FC1853009F4ACC101C010E00E9429ACDC
:103D4000811103C0E5ECF2E013C080917C10882360
:103D500019F063E173E002C067E173E08DEB92E07C
:103D60000E9497C58AE00E94EE930E942CBD96C1E6
:103D700084917F01BFEFEB1AFB0A882309F48EC1FF
:103D80000E94EE93F701F4CF0E94DFBD1092010272
:103D90001092000282EB92E09093A4078093A30715
:103DA0000E941A940C94ED2E8091000290910102D1
:103DB00097FF0EC0E9E8F2E084918F010F5F1F4F7B
:103DC000882311F40C94ED2E0E94EE93F801F4CFA9
:103DD0000097A1F4809152028093280419821A82DC
:103DE0001B821C8218A219A21AA21BA2BE016F5F1D
:103DF0007F4FCE0180960E9475B427C0815065E048
:103E00000E947BED80FF03C024E0291B922F25E058
:103E10009202F0011124E80FF11D87FDFA95EE0FD3
:103E2000FF1FEE0FFF1FEA53FF4E80913A0490915F
:103E30003B04A0913C04B0913D0480839183A28314
:103E4000B383809128048093520280910002909164
:103E50000102893191050CF067C0109252029C0159
:103E60002F5F3F4F309301022093000265E00E94D4
:103E70007BED80FF03C024E0291B922F40913A0480
:103E800050913B0460913C0470913D0448A359A3B8
:103E90006AA37BA319821A821B821C8244E08402DB
:103EA00090011124B9016751764F4B01DB012D912F
:103EB0003D914D915C91B4E09B02C0011124FC0145
:103EC000E350F64F5F016081718182819381DE0151
:103ED00011966D01E12CF12C00EA10E40E94A8B3C8
:103EE00019821A821B821C82B601CE0180960E9422
:103EF00075B4F50180819181A281B38180933204F0
:103F000090933304A0933404B0933504F40180817A
:103F10009181A281B3818093360490933704A0935A
:103F20003804B0933904BCC080E090E0A0EAB0E46B
:103F300080933A0490933B04A0933C04B0933D04D7
:103F40000E9469AD0E941F6A8FEF9FEF909301025C
:103F500080930002E5E7F2E084918F010F5F1F4F2D
:103F6000882321F00E94EE93F801F6CF83E992E0D6
:103F70009A83898304E610E019A308A3BE016F5F4A
:103F80007F4FCE0180960E9490B58AEB92E09A8393
:103F9000898319A308A3BE016F5F7F4FCE0180966E
:103FA0000E9490B581E00E9476AC81E00E9456AC00
:103FB00077C088E50E94984C8823A1F00E94E84BC6
:103FC0001FEF160F1530A8F0EEE5F2E084918F0197
:103FD0000F5F1F4F882311F40C94ED2E0E94EE9377
:103FE000F801F4CF88E50E94EE930E94B6E10C94AC
:103FF000ED2E89E50E94984C8823A1F00E94E84BA1
:104000000FEF060F0530A8F0E7E4F2E084918F018E
:104010000F5F1F4F882311F40C94ED2E0E94EE9336
:10402000F801F4CF89E50E94EE930E94B6E10C946A
:10403000ED2E8AE50E94984C882399F00E94184C36
:1040400025E0129FF0011124E00FF11DEE0FFF1F7C
:10405000EE0FFF1FEA53FF4E6083718382839383C9
:1040600035C08AE50E94EE930E94B6E10C94ED2ED5
:104070008AE50E94984C8823A1F30E94184C609313
:10408000C2107093C3108093C4109093C5101EC0CB
:1040900080E00E9456AC0E94DFBD18C01230B1F41F
:1040A00060910002709101026931710514F069E1BB
:1040B00070E088E392E00E947EC569E170E083E3EE
:1040C00092E00E947EC58AE00E94EE930E94428D9B
:1040D0000C94ED2E80912702882311F40C94ED2E80
:1040E00089E40E94984CE82E882321F00E94E84B36
:1040F000062F01C000E08AE40E94984CF82E882325
:1041000021F00E94E84B162F01C010E0EE2011F0C4
:10411000053020F4FF2081F0153070F0ECEFF2E074
:1041200084918F010F5F1F4F882311F40C94ED2EA3
:104130000E94EE93F801F4CF0E94A44CEE2091F07F
:1041400034E00302F0011124E350F64F80819181A5
:10415000A281B3818093AE109093AF10A093B01062
:10416000B093B110FF2091F044E01402F00111244B
:10417000E751F64F80819181A281B3818093B21083
:104180009093B310A093B410B093B51080E50E9443
:10419000984C882319F00E94094C03C080E50E94C6
:1041A0004F4C86E40E94984C8823D9F00E94184C0A
:1041B0006B017C0120E030E0A9010E94D9EC1816C7
:1041C00084F420E030E040E752E4C701B6010E94E9
:1041D0008FEB6093300270933102809332029093A0
:1041E00033020E9486CA0C94ED2E209327040C946F
:1041F000ED2E97E5292E92E0392E2DE4E22E20E1D6
:10420000F22E62E374E07DAB6CAB34E1C32E34E09C
:10421000D32E00E010E0D1018D911D010E94984C39
:10422000882309F44BC00E94184C2B013C01133029
:1042300049F0F60120813181428153810E94B2EA26
:104240002B013C01ACA9BDA92D913D914D915C91F3
:10425000C301B2010E94B2EA4B015C012DEB37E3CE
:1042600046E855EB0E94D9EC87FD0AC02DEB37E3F9
:1042700046E855E3C501B4010E9467E61816F4F458
:10428000133051F440923E0450923F046092400437
:104290007092410401E012C0A5019401F701608110
:1042A0007181828193810E94B3EAD7016D937D93DE
:1042B0008D939C931397812F0E94C0AD1F5FB4E034
:1042C000EB0EF11CECA9FDA93496FDABECABF4E0D0
:1042D000CF0ED11C143009F09ECF002309F4F6CE86
:1042E0000E9444B3F3CE0E94C4B50C94ED2E80918D
:1042F0001318909114188537910511F40C94ED2E34
:104300000CF0C0C08C34910509F43CC40CF058C0CA
:104310008A31910509F42EC224F58531910509F4FD
:10432000E7C184F48231910509F4A9C5843191056E
:1043300009F49EC1419711F00C949C2E0E94EDA4AB
:104340000C94ED2E8731910509F4DCC10CF4D4C135
:104350008831910509F4ECC1499709F4F4C10C9432
:104360009C2E8F31910509F401C39CF48C31910589
:1043700009F4A6C20CF40CC28D31910511F40C9411
:10438000ED2E4E9711F00C949C2E0E943FB00C9491
:10439000ED2E8A32910509F49CC32CF4809709F420
:1043A00099C20C949C2E8133910509F4C6C38B34B9
:1043B000910511F00C949C2E0E94C4780C94ED2E63
:1043C0008A36910509F40AC5B4F58435910509F4D6
:1043D00056C5E4F48135910509F42CC54CF48D34AF
:1043E000910511F00C949C2E0E94FB780C94ED2EFC
:1043F0008235910509F440C58335910511F00C947F
:104400009C2E81E0809326040C94ED2E8C35910532
:1044100009F47BC534F48535910509F45DC50C9428
:104420009C2E8836910509F4B1C38936910509F4AB
:1044300075C40C949C2E8F36910509F4E3C384F463
:104440008C36910509F431C40CF4E4C48D36910521
:1044500009F4A6C48E36910509F4C1C30C949C2EB0
:104460008137910509F42DC40CF423C482379105DA
:1044700009F4D3C58337910511F00C949C2EE3EE1B
:10448000F4E008C68E3221E0920711F40C94D82C87
:104490000CF071C08B3C910509F416C7CCF58C3833
:1044A000910509F481C4ACF48737910509F49AC6E3
:1044B0000CF44BC68837910509F497C689379105E6
:1044C00011F00C949C2E10923705109236050C9426
:1044D000ED2E8E3B910509F47DC434F48B399105A2
:1044E00009F437C40C949C2E883C910509F483C6CA
:1044F000893C910511F00C949C2EF7E5EF2EF2E02B
:10450000FF2E0FE411E1AFE5CA2EA1E1DA2EC3C6FA
:104510008C3D910511F40C946B2B9CF48D3C910512
:1045200009F463C70CF4ECC68E3C910509F4EAC7A4
:10453000833D910511F00C949C2E0E94378C0C94B5
:10454000ED2E823E910511F40C94E62B3CF48D3D4A
:10455000910511F40C94782B0C949C2E8C3241E034
:10456000940711F40C940F2C8D32914011F40C949B
:10457000382C0C949C2E853F61E0960711F40C9426
:10458000C52DDCF58A39A1E09A0709F496C3BCF47D
:104590008033E1E09E0711F40C942F2D14F40C9459
:1045A0002C2D833621E0920709F45EC080399140BA
:1045B00011F00C949C2E0E941F6A0C94ED2E853AEB
:1045C00041E0940711F40C94C22D4CF4843A9140CC
:1045D00011F00C949C2E0E94088E0C94ED2E8C3AB7
:1045E00071E0970709F4B1C7843F914011F00C9432
:1045F0009C2E0E9466700C94ED2E8A39B2E09B07C7
:1046000011F40C94042EB4F4873FF1E09F0711F4E9
:104610000C94CB2D14F40C94C82D883F31E09307F3
:1046200011F40C94D72D8C30924011F40C94FB2D86
:104630000C949C2E8B3853E0950711F40C94ED2EBE
:104640003CF48438934011F40C94312E0C949C2E3D
:10465000803AA3E09A0709F47CC1873E934011F4A5
:104660000C94892E0C949C2EE1EDFDE10C94AF2D61
:10467000EAE2F3E084918F010F5F1F4F882321F05E
:104680000E94EE93F801F6CF1092AF0C82E69AE00A
:104690000E94669A8BE1E2E6FAE0DE01159601904F
:1046A0000D928A95E1F78091600A9091610A9C834E
:1046B0008B838DEE92E09A83898340E050E0BE01C7
:1046C0006F5F7F4F80E090E00E94ED82CE01019607
:1046D0000E94C2A0EBE1F3E084918F010F5F1F4FB6
:1046E000882311F40C94ED2E0E94EE93F801F4CF80
:1046F0000E94BC800C94ED2E1092310A1092320A66
:104700000C94ED2EE0911118F091121880818823FD
:1047100029F0803209F410823196F8CF40E061E050
:1047200080911118909112180E94B5D50C94ED2E1D
:104730008091320A882319F081E08093310A0E9427
:10474000C4780C94ED2E1092310A80912B078130A1
:1047500011F00C94ED2E82E080932B070E94FF58FD
:1047600060932707709328078093290790932A075F
:104770000C94ED2E8091320A882311F40C94ED2EC6
:1047800083E50E94984C81110C94F72E0C94ED2E29
:1047900083E40E944F4C882309F450C0E8E6F3E01C
:1047A00084918F010F5F1F4F882321F00E94EE93A9
:1047B000F801F6CF8091FD0B811103C0EBE3F3E02C
:1047C00012C0BE016F5F7F4F8AEF9BE00E942E995F
:1047D0008E010F5F1F4FF80181918F01882349F1EE
:1047E0000E94EE93F8CF84918F010F5F1F4F8823B3
:1047F00001F10E94EE93F801F6CF06EDC02E03E022
:10480000D02EE12CF12C20E08091100790E00E2CAE
:1048100002C0959587950A94E2F780FD23C2BFEF09
:10482000EB1AFB0AE2E0CE0ED11CF5E0EF16F10424
:1048300059F78AE00E94EE930C94ED2E8091320A93
:10484000882339F08091310A882319F0E5E4F3E0F8
:1048500003C0E7E5F3E028C084918F010F5F1F4F8D
:10486000882321F00E94EE93F801F6CF6091AB0C03
:104870007091AC0C8091AD0C9091AE0C4AE00E940E
:104880000F978FE20E94EE936091A70C7091A80C95
:104890008091A90C9091AA0C4AE00E940F978AE09F
:1048A0000E94EE930C94ED2E84918F010F5F1F4FA9
:1048B000882311F40C94ED2E0E94EE93F801F4CFAE
:1048C00040E060E080911118909112180E94B5D5D7
:1048D0000C94ED2E8091310A81110E941F6A809103
:1048E000320A882311F40C94ED2E80E50E94984C36
:1048F000882319F00E94094C03C080E50E944F4CA8
:10490000182F482F61E080911118909112180E9481
:10491000B5D583E50E94984C882381F00E94E84B2E
:10492000AB01BC014093AB0C5093AC0C6093AD0C4D
:104930007093AE0C8AEF9BE00E941F988091320A20
:10494000882319F081E08093310A11110C94ED2E27
:10495000F6CE809111189091121821E02093300A20
:1049600040E060E00E94B5D50C94ED2E0E94757871
:104970007B018C0120E831E541E050E00E9455EADE
:10498000C9016DE671E00E9488ED4B015C01C80130
:10499000B70120E13EE040E050E00E9455EACA0144
:1049A000B90128E130E040E050E00E9455EA762E5F
:1049B000672EC62ED72E8CE3282E312C412C512C5D
:1049C000C801B701A20191010E9455EAF62EE72E17
:1049D000CA01B901A20191010E9455EACB018E01E1
:1049E0000F5F1F4F81149104D1F0EF92FF927F93DC
:1049F0006F936F927F92BF92AF929F928F928FE947
:104A000093E09F938F931F930F930E9439E60FB605
:104A1000F894DEBF0FBECDBFE6EEFDE145C0A114A8
:104A2000B10489F0EF92FF927F936F936F927F9220
:104A3000BF92AF928FE893E09F938F931F930F9352
:104A40000E9439E6E4CFCD2879F0EF92FF927F9370
:104A50006F936F927F9283E893E09F938F931F935E
:104A60000F930E9439E6D3CF892B69F0EF92FF9222
:104A70007F936F938BE793E09F938F931F930F9395
:104A80000E9439E6C4CFEF92FF9287E793E09F93AD
:104A90008F931F930F930E9439E60F900F900F9002
:104AA0000F900F900F90B8CF84917F019FEFE91A7C
:104AB000F90A882321F00E94EE93F701F5CFB8019F
:104AC00083EB93E00E9497C58AE00E94EE930C94DA
:104AD000ED2E83E50E94984C882311F40C94ED2E62
:104AE0000E94F84BE82E80E50E94984C882339F00C
:104AF0000E94F84B182F87FF03C00C94ED2E1DE089
:104B000089E40E94984C882341F00E94094C81114D
:104B10000C94732FEBE1F6E00BC089E40E944F4C3C
:104B2000F6CF3196A6E0EB34FA0711F40C94732F0C
:104B300084911813F6CF0C94482FF090200481E054
:104B4000F826F0922004EBECF3E084918F010F5FE4
:104B50001F4F882321F00E94EE93F801F6CFFF202B
:104B600019F0E0ECF3E002C0E5ECF3E084918F0192
:104B70000F5F1F4F882311F40C94ED2E0E94EE93CB
:104B8000F801F4CF0E94E6780C94ED2E88E690E0D0
:104B90000E9400AE81110C94ED2E8091100783FFCE
:104BA00002C00C94ED2E83E50E94984C882399F066
:104BB0000E94184C0E94F7EBCB010E94F4590E940E
:104BC000184C20E030E044EB52E40E9467E61816EF
:104BD00014F00E94FB780E94C1C70C94ED2E8EE465
:104BE0000E94984C882311F40C94ED2E0E94E84BFF
:104BF0006093BE187093BF188093C0189093C1182B
:104C00000C94ED2E83E50E944F4C882359F083E5E8
:104C10000E94984C882319F00E94F84B01C080E054
:104C200080931007E6EEFDE184918F010F5F1F4F27
:104C3000811103C0E4EEF3E004C00E94EE93F8019A
:104C4000F3CF84918F010F5F1F4F882321F00E94C3
:104C5000EE93F801F6CF809110078111CECDE0EEF2
:104C6000F3E018C0BB24B394B20E222319F08CE2F7
:104C70000E94EE93F60185919491FC0184918F013D
:104C80000F5F1F4F882321F00E94EE93F801F6CFAB
:104C90002B2DC5CD84918F010F5F1F4F882309F401
:104CA000C8CD0E94EE93F801F5CF109220020C942B
:104CB000ED2E8BEE93E00E94E5A00E949B860C9463
:104CC000ED2E83E50E94984C811103C0E6EEFDE1D4
:104CD0000DC00E94F84B8D3320F480932B020C946E
:104CE000ED2E8CE380932B020C94ED2E84918F019A
:104CF0000F5F1F4F882321F00E94EE93F801F6CF3B
:104D000040912B0250E060E070E084EF93E00E945D
:104D100044C58AE00E94EE930C94ED2E89E690E063
:104D20000E9400AE811111C0EBEFF3E084918F017E
:104D30000F5F1F4F882321F00E94EE93F801F6CFFA
:104D40000E94FD758AE00E94EE9310923F100C9431
:104D5000882F83E50E94984C882311F40C94ED2E43
:104D60000E94F84B182F8D3308F01CE310934C1061
:104D70000E94FF586B017C01212F30E0A8EEB3E0C8
:104D80000E94A3EAC60ED71EE81EF91EC092481064
:104D9000D0924910E0924A10F0924B100C94ED2EF4
:104DA0000E9442AE0C94ED2E8091100783FF02C04A
:104DB0000C94ED2E83E50E94984C882311F40C94FA
:104DC000ED2E0E94184C0E94F7EBCB010E94274E5B
:104DD0000C94ED2E0E9406A90C94ED2E80E50E9405
:104DE000984C811106C083E50E94984C882359F0A5
:104DF00005C00E94F84B8111F0C7F5CF0E94E84B27
:104E00006F3F710510F06FEF70E070934304609393
:104E10004204E3C780E50E94984C811105C01092BE
:104E2000430410924204D9C70E94E84B672B09F053
:104E3000D4C7F5CF0E9410790E94D4B710924304D2
:104E40001092420400E010E062E370E080E090E045
:104E50000E943AB70E94D07B0F5F1F4F03311105AC
:104E600099F762E370E080E090E00E943AB70E9418
:104E7000D07B0E94A22FB1C710922604AEC783E553
:104E80000E94984C882399F00E94184C20E030E052
:104E90004AE754E40E94CCE60E94FCEB60932C02AB
:104EA00070932D0280932E0290932F0296C788E56F
:104EB0000E944F4C8111ACC789E50E944F4C811173
:104EC000A7C78AE50E944F4C8111A2C785E40E94C2
:104ED0004F4C81119DC7CEC783E50E944F4C88235C
:104EE00009F47BC70E94184C20E030E04AE754E404
:104EF0000E94CCE60E94FCEB609344107093451036
:104F0000809346109093471068C7B7E5CB2EB2E068
:104F1000DB2E12E9E12E10E1F12E10E0D6018D9189
:104F20006D010E944F4C882309F46DC0133009F0C5
:104F300063C00E94184C4B015C0120E030E040EA65
:104F400051E40E9467E687FF4EC0A501940160917D
:104F50009E1070919F108091A0109091A1100E94BE
:104F60008FEB2B013C019B01AC016091DF0670913E
:104F7000E0068091E1069091E2060E94CCE6609303
:104F8000DF067093E0068093E1069093E206A301AA
:104F900092016091FF067091000780910107909146
:104FA00002070E94CCE66093FF067093000780938F
:104FB00001079093020760914B1170914C11809101
:104FC0004D1190914E110E946BE6A30192010E9437
:104FD000CCE60E94FCEB60934B1170934C118093D4
:104FE0004D1190934E1180929E1090929F10A0921E
:104FF000A010B092A11007C00E94184CF701608366
:105000007183828393831F5FF4E0EF0EF11C1430F1
:1050100009F084CF0E9462C9E0C60E941F6A83E53E
:105020000E94984C882309F451C80E94E84B6230D2
:10503000710509F04BC80E94D3C98BE50E94EE931D
:105040006091A4187091A5188091A6189091A71846
:1050500042E00E9494974091A8185091A91860913D
:10506000AA187091AB1881E094E00E9461C540914C
:10507000AC185091AD186091AE187091AF188EEFCA
:1050800093E00E9461C58DE50E94EE938AE00E9444
:10509000EE93A3C684918F010F5F1F4F882321F0E9
:1050A0000E94EE93F801F6CF60E083ED94E00E9459
:1050B0000F8D61E08CEC94E00E940F8D61E081EC3B
:1050C00094E00E940F8D61E081EB94E00E940F8DCF
:1050D00060E088EA94E00E940F8D61E08EE994E040
:1050E0000E940F8D60E084E994E00E940F8D60E0E3
:1050F0008CE894E00E940F8D61E08EE794E00E94BE
:105100000F8D60E080E794E00E940F8D60E081E603
:1051100094E00E940F8D60E083E594E00E940F8D83
:1051200060E08DE394E00E940F8D60E08CE294E0FB
:105130000E940F8D60E087E194E00E940F8D61E096
:1051400084E094E00E940F8D48C6009111181091E0
:10515000121883E0D12C40E08150E9F0D8019C91F5
:10516000292F2B7F2134C1F711962C912133A1F7E0
:10517000913421F0953421F441E002C0DD24D39430
:1051800098012E5F3F4F89012F5F3F4FF8019081BB
:105190009032C9F3E1CF442369F0E6EEFDE184915A
:1051A0007F012FEFE21AF20A882321F00E94EE938A
:1051B000F701F5CFDD2069F0E9EAF5E084917F01A0
:1051C0003FEFE31AF30A882321F00E94EE93F701E0
:1051D000F5CFD8018D918D01882309F42ACB0E9447
:1051E000EE93F7CF0E9477BEF8C581E08093370534
:1051F00080933605F2C588EC90E00E9400AE8111E4
:10520000ECC584E40E944F4C882309F441C00E94FD
:10521000184C6B017C0111E020E030E0A9010E94F4
:1052200067E6811101C010E010932A1120E030E000
:10523000A901C701B6010E9467E6882349F10E94CF
:10524000184CE0914E07B4E0EB9FF0011124E15DB2
:10525000FE4E608371838283938320E030E0A90156
:1052600060912F1170913011809131119091321114
:105270000E9467E681110CC080E090E0A0EEBFE3E1
:1052800080932F1190933011A0933111B09332116C
:105290000E9412B8A2C5F70181917F010E944F4C74
:1052A000882351F00E94184C0E94FCEBD8016D93AA
:1052B0007D938D939C9313970C5F1F4FC016D1065F
:1052C00051F70E94F1C789C5E7E5EE2EE2E0FE2E18
:1052D00003EF16E0F70181917F010E944F4C882374
:1052E00041F00E94184CD8016D937D938D939C934F
:1052F00013970C5F1F4FB7E003301B0759F76DC5BD
:1053000083E50E94984C8823A1F00E94184C60937A
:10531000EB067093EC068093ED069093EE06609397
:10532000E7067093E8068093E9069093EA0610E09A
:1053300001C011E080E50E94984C882359F00E943A
:10534000184C6093EB067093EC068093ED069093F7
:10535000EE0610E082E50E94984C882359F00E94E6
:10536000184C6093EF067093F0068093F1069093CB
:10537000F20610E084E50E94984C882359F00E94C0
:10538000184C6093E7067093E8068093E9069093C3
:10539000EA0623C5112309F420C54091EB0650917C
:1053A000EC066091ED067091EE0683EB95E00E94AD
:1053B00061C54091EF065091F0066091F106709141
:1053C000F20680EB95E00E9461C54091E70650919E
:1053D000E8066091E9067091EA068DEA95E00E9480
:1053E00061C58AE00E94EE93F8C481E50E944F4CAB
:1053F0008823C1F08091210490912204009739F014
:105400004AE050E060E070E00E94E6E403C060E043
:1054100070E0CB0160930307709304078093050746
:105420009093060783E50E944F4C882351F00E9419
:10543000184C60930B0770930C0780930D079093A3
:105440000E0784E50E944F4C882351F00E94184CAF
:1054500060930707709308078093090790930A07E2
:1054600088E50E944F4C882351F00E94184C6093AD
:10547000D3067093D4068093D5069093D60689E51B
:105480000E944F4C882351F00E94184C6093D7061D
:105490007093D8068093D9069093DA068AE50E9425
:1054A0004F4C8823F1F00E94184C6093DB067093F8
:1054B000DC068093DD069093DE062DEC3CEC4CEC94
:1054C0005DE30E9467E6181664F0E3ECF5E0849172
:1054D0008F010F5F1F4F882321F00E94EE93F80188
:1054E000F6CF85E40E944F4C882309F476C40E94CD
:1054F000184C6093DF067093E0068093E10690936A
:10550000E2066BC467E5C62E62E0D62E78E3E72E8E
:1055100075E0F72E10E0F60181916F010E944F4C6B
:10552000882359F00E94184CD7016D937D938D9379
:105530009C931397812F0E94C0AD1F5FB4E0EB0EC8
:10554000F11C133041F70C9466200E9493B4811132
:1055500044C40BEF12E2E2E3F4E0FDABECAB9E01DE
:105560002F5F3F4F590154E4852E53E2952E1901C8
:10557000F8016591759185919491ACA9BDA9CD90E3
:10558000DD90ED90FD90BDABACABA70196010E9404
:10559000B2EA2B013C01F101608371838283938322
:1055A00020E030E040EA51EC0E94D9EC87FD0AC0CF
:1055B00020E030E040EA51E4C301B2010E9467E616
:1055C00018162CF4F401849118160CF456C4D10169
:1055D000CD90DD90ED90FD901D0120E030E040EA9F
:1055E00051ECC701B6010E94D9EC87FD0AC020E04A
:1055F00030E040EA51E4C701B6010E9467E61816A0
:105600004CF5E1EDFDE184918F010F5F1F4F81119A
:1056100003C0E5EFF5E004C00E94EE93F801F3CF7C
:1056200084918F010F5F1F4F882321F00E94EE931A
:10563000F801F6CF88E290E099A388A388EC90E087
:105640009DA78CA7BE01605E7F4FCE018C960E9405
:1056500090B5C3C30C5F1F4FBFEF8B1A9B0AE7E0E7
:10566000F3E2E017F10709F083CF48E3E42E45E0C9
:10567000F42E10E0F50181919191A191B1915F011A
:10568000F70181939193A193B1937F01812F0E94A0
:10569000C0AD1F5F133071F70E94428D83E992E025
:1056A0009DA78CA704E610E019A308A3BE01645DC2
:1056B0007F4FCE0180960E9490B58AEB92E09DA725
:1056C0008CA719A308A3BE01645D7F4FCE0180960D
:1056D0000E9490B582C383E50E94984C882309F408
:1056E0007CC30E94E84B709303026093020275C36F
:1056F0008DED90E00E9400AE81116FC383E50E94A2
:10570000984C811103C0E6EEFDE13AC000914E07CE
:1057100010E00E94E84B000F111FF801E85CFD4FFC
:105720007183608380914E0790E07C01EE0CFF1C3A
:10573000EE0CFF1C87010F5D1D4F880F991FFC01A8
:10574000E85CFD4F60817181072E000C880B990B7E
:105750000E946DE62AE037ED43E25CE30E94CCE66E
:10576000F701E55DFE4E20813181428153810E9427
:10577000CCE6D8016D937D938D939C9313972DC3A5
:1057800084918F010F5F1F4F882321F00E94EE93B9
:10579000F801F6CF85E40E94EE9380914E07805D7C
:1057A0000E94EE93E0914E07F0E0EE0FFF1FE85CE1
:1057B000FD4F6081718183E196E00E947EC585E2A4
:1057C0000E94EE938AE00E94EE9307C380E50E9458
:1057D0004F4C882309F401C30E94E84B6B017C0104
:1057E00083E50E94984C882321F00E94E84B8B01AE
:1057F00002C00FEF1FEFC8010196039708F0EDC23A
:10580000D7FCEBC28C2DEBE1F6E09491891709F4FB
:105810003FC33196B6E0EB34FB07B9F73CC383E5F1
:105820000E94984C882319F00E94E84B02C064E063
:1058300071E079A368A380E50E94984C882339F031
:105840000E94E84B6938E3E17E0730F402C068EE5D
:1058500073E07A83698304C088E893E19A8389833B
:10586000BE01605E7F4FCE0101960E9490B5B5C229
:1058700085E40E94984C811110C080E50E944F4C35
:10588000882391F00E94184C60933C0770933D0769
:1058900080933E0790933F0707C00E94F84B8823F0
:1058A00061F3E1EDFDE171C089E40E944F4C882372
:1058B00081F00E94184C2CEA35EC47E25EE30E942E
:1058C000CCE6609338077093390780933A0790933A
:1058D0003B0784E40E944F4C882381F00E94184CBF
:1058E0002CEA35EC47E25EE30E948FEB60934007C1
:1058F000709341078093420790934307E6EEFDE1E2
:1059000084918F010F5F1F4F882321F00E94EE9337
:10591000F801F6CF40913C0750913D0760913E075A
:1059200070913F0783E596E00E9461C52CEA35EC53
:1059300047E25EE3609138077091390780913A073A
:1059400090913B070E948FEBAB01BC018FE496E086
:105950000E9461C52CEA35EC47E25EE360914007A6
:105960007091410780914207909143070E94CCE6D5
:10597000AB01BC018BE496E00E9461C58AE00E9405
:10598000EE932BC20E94EE93F80184918F010F5F7A
:105990001F4F8111F7CFE7E5F6E084918F010F5F8C
:1059A0001F4F882309F419C20E94EE93F801F5CF26
:1059B00083E50E944F4C182F882371F00E94184CE9
:1059C0000E94F7EB709326026093250221E0672B7B
:1059D00009F020E020930F0780E50E944F4C8823B8
:1059E00059F02091250230912602232B11F00E94BC
:1059F000094C80930F07F1C11111EFC1E6EEFDE1F3
:105A000084918F010F5F1F4F882321F00E94EE9336
:105A1000F801F6CF80910F07882319F06BE173E04E
:105A200002C06EE173E08EE796E00E9497C5609138
:105A30002502709126028DE696E00E947EC5E9E679
:105A4000F6E084918F010F5F1F4F882309F4C5C1D1
:105A50000E94EE93F801F5CF0E94D886BEC180E582
:105A60000E944F4C882351F00E94184C60933407D9
:105A700070933507809336079093370789E40E9427
:105A80004F4C882381F00E94184C2CEA35EC47E2F9
:105A90005EE30E94CCE660933007709331078093F9
:105AA00032079093330784E40E944F4C882381F09F
:105AB0000E94184C2CEA35EC47E25EE30E948FEB23
:105AC00060932C0770932D0780932E0790932F07D8
:105AD000E6EEFDE184918F010F5F1F4F882321F0D7
:105AE0000E94EE93F801F6CF4091340750913507AC
:105AF000609136077091370789E996E00E9461C589
:105B00002CEA35EC47E25EE3609130077091310793
:105B100080913207909133070E948FEBAB01BC015B
:105B200085E996E00E9461C52CEA35EC47E25EE328
:105B300060912C0770912D0780912E0790912F076F
:105B40000E94CCE6AB01BC0181E996E00E9461C5F0
:105B50008AE00E94EE9341C10E94EE93F801849185
:105B60008F010F5F1F4F8111F7CFEDE9F6E08491B0
:105B70008F010F5F1F4F882309F42FC10E94EE93FE
:105B8000F801F5CF0E94B08528C10E945A7025C146
:105B90000E941BC322C183E50E944F4C882321F041
:105BA0000E94094C91E089270E94ACBE16C181E099
:105BB000809317070E94506A10921707882309F4F0
:105BC0000CC1E6EEFDE184918F010F5F1F4F811143
:105BD00003C0ECEAF6E004C00E94EE93F801F3CFB4
:105BE00084918F010F5F1F4F882309F4F6C00E9434
:105BF000EE93F801F5CF8091310A882309F4EDC0C6
:105C000081E08093340AE9C08AE50E94984C8111B2
:105C100003C0EAEBF6E00BC00E94184C609337110A
:105C2000709338118093391190933A11D6C08491B2
:105C30008F010F5F1F4F882321F00E94EE93F80120
:105C4000F6CF409137115091381160913911709110
:105C50003A1187EB96E00E9461C58AE00E94EE93BC
:105C6000BCC08BE40E94984C811103C0E6EEFDE1BC
:105C700036C08BE40E94984C8823C1F00E94184CD7
:105C80006B017C0120E030E0A9010E94D9EC87FD86
:105C90000AC020E030E040E251E4C701B6010E94B2
:105CA00067E6181634F4E9EDF6E00EC0C12CD12CED
:105CB00076010E941F6AC092E306D092E406E09249
:105CC000E506F092E60689C084918F010F5F1F4FB1
:105CD000882309F482C00E94EE93F801F5CF8491E5
:105CE0008F010F5F1F4F882321F00E94EE93F80170
:105CF000F6CF4091E3065091E4066091E50670917D
:105D0000E60688EF96E00E9461C58AE00E94EE9365
:105D100064C081E08093270283E50E94984C882329
:105D200039F00E94094C811158C00E9477CE55C0AD
:105D300083E50E944F4CF7CF0E94C4B54EC0F0904F
:105D400013180E941F6A10917C1080E00E9456ACCC
:105D5000FF2029F1E6EEFDE184918F010F5F1F4FD7
:105D6000882321F00E94EE93F801F6CF84E50E948B
:105D7000EE936F2D70E080E090E04AE00E940F9774
:105D800080E20E94EE93E5E1F7E084918F010F5FDE
:105D90001F4F882311F10E94EE93F801F6CF109265
:105DA0003E10812F0E9456ACE6EEFDE184918F01FA
:105DB0000F5F1F4F882321F00E94EE93F801F6CF6A
:105DC00060913E1070E083E097E00E947EC58AE01B
:105DD0000E94EE9302C00E94C4B510923F100E9430
:105DE0005ACE96C00E94D6AA0E9486CAF6CF0E94BA
:105DF000E84BAB01BC014093AB0C5093AC0C6093EF
:105E0000AD0C7093AE0C8AEF9BE00E941F98E5CF1B
:105E10000E941F6A88E50E944F4C882331F05F9AE8
:105E2000809131048E7F8093310489E50E944F4C2C
:105E3000882339F08A9A479A809131048D7F809324
:105E400031048AE50E944F4C882361F0809108015B
:105E50008095817080930601479A809131048B7FF1
:105E60008093310485E40E944F4C882309F4B5CF18
:105E7000129AB3CF0E94D4B7B0CFF7FAF094F7F8E4
:105E8000F094D101CD92DD92ED92FC9213979FCBCD
:105E90000E949BE1A2CF0E941F6ABC2C60E08C2D67
:105EA0000E9437B60F3FBFEF1B0759F48C2D0E949D
:105EB000E1B531E020E0892B09F030E0032F122F0B
:105EC00005C00130110561F401E010E08B2D0E9446
:105ED000E1B58017910709F480CF0E942CA1F6CF7D
:105EE00000E010E0F3CF61E0812F0E9437B66E2D05
:105EF000812F0E9409B6F12CB701812F0E9473B641
:105F0000193009F06ACFF0924304E092420465CF61
:105F1000C657DF4F0FB6F894DEBF0FBECDBFDF917F
:105F2000CF911F910F91FF90EF90DF90CF90BF9096
:105F3000AF909F908F907F906F905F904F903F9029
:105F40002F9008952F923F924F925F926F927F927F
:105F50008F929F92AF92BF92CF92DF92EF92FF9279
:105F60000F931F93CF93DF93CDB7DEB76F970FB625
:105F7000F894DEBF0FBECDBFC0904C04D0904D044E
:105F8000E0904E04F0904F0420E030E040EA50E40E
:105F9000C701B6010E9467E687FD19C120E030E025
:105FA00041E953E4C701B6010E94D9EC18160CF47C
:105FB0000EC110924E0E10924D0E8091090140912B
:105FC0004C0E042E000C550B817021E0822790E0CE
:105FD0004817590709F433C08091090181702827B7
:105FE00020934C0E81111BC00E94BC80E1E3FDE0B8
:105FF00084918F01882351F0082E000C990B0E9488
:10600000B7800F5F1F4FF8018491F4CF8DE090E0CF
:106010000E94B7808AE090E00E94B78010C0E5E35C
:10602000FDE084918F01882389F3082E000C990BE1
:106030000E94B7800F5F1F4FF8018491F4CF8091C9
:106040003F0E833009F44CC02CF4882351F081308A
:10605000D9F072C0843009F43EC0853009F44DC0D7
:106060006BC08091310A882309F466C081E0809377
:106070003F0E0E94FF586093430E7093440E80932E
:10608000450E9093460E58C08091310A811154C03C
:106090008091FD0B882321F082E080933F0E4CC05D
:1060A00010923F0EEDE2FDE084918F01882351F0C4
:1060B000082E000C990B0E94B7800F5F1F4FF8014C
:1060C0008491F4CF8DE090E00E94B7808AE090E068
:1060D0000E94B78031C080918C0E8823E9F22CC0D9
:1060E0008091310A811128C08091B3099091B4093F
:1060F000891B8F7009F496C01FC08091310A8111ED
:106100001BC08091B3099091B409891B8F7009F469
:10611000ABC012C08DE090E00E94B7808AE090E0B2
:106120000E94B78010923F0E8DE09DE09093A407EF
:106130008093A3070E941A948091340E9091350E9B
:1061400003974CF571E4272E79E0372EE0E68E2E8A
:10615000EAEE9E2EA12CB12C8AE99FE00E946A4BA8
:1061600018161906C4F48091340E9091350E0497D8
:1061700094F48AE99FE00E942E4B80933A0EE091BE
:106180003B0EF0913C0E8A3019F08D3009F07DC045
:10619000309709F083C08091340E9091350E0097AE
:1061A00011F40C94233F01979093350E8093340E95
:1061B0008091360E9091370E019664E070E00E9457
:1061C0009CED9093370E8093360E0C94233F809174
:1061D0004D0E90914E0E8136FAEE9F07E8F0109228
:1061E0004E0E10924D0EE9E3FDE084918F0188235D
:1061F00051F0082E000C990B0E94B7800F5F1F4FC3
:10620000F8018491F4CF8DE090E00E94B7808AE09D
:1062100090E00E94B780D1CE019690934E0E80936D
:106220004D0ECBCE89E19DE09093A4078093A30708
:106230000E941A9480918C0E882311F082E001C094
:1062400084E080933F0EE5E1FDE084918F01882397
:1062500009F438CF082E000C990B0E94B7800F5F0D
:106260001F4FF8018491F3CFE1E1FDE084918F01AC
:10627000882309F44FCF082E000C990B0E94B78099
:106280000F5F1F4FF8018491F3CF8A3309F480CF59
:10629000EF35F10514F40C94B73C7ACF8091380EA9
:1062A0009091390E20E6289F7001299FF00C11244F
:1062B00087010C54134FE00FF11F108261E470E06E
:1062C000C8010E9403EE009711F40C949B3C90933C
:1062D0003E0E80933D0E801B910B8E0D9F1D60E046
:1062E00070E08B54934F0E9468E20E94F7EBCB0161
:1062F000770FAA0BBB0B8232910510F00C949B3CDC
:10630000FC018827EE58FF4F8F4F0C94AFEDE8E06B
:10631000FDE084918F01882351F0082E000C990B29
:106320000E94B7800F5F1F4FF8018491F4CF20E0E7
:1063300030E040E05FE360914C0470914D04809147
:106340004E0490914F041EC0E3E0FDE084918F0164
:10635000882351F0082E000C990B0E94B7800F5F24
:106360001F4FF8018491F4CF60914A0470914B045F
:10637000072E000C880B990B0E946DE620E030E0A0
:1063800040E05FE30E94B3EA0E94F7EBCB010E947A
:10639000F14D0E94EBD78DE090E00E94B7808AE03B
:1063A00090E00E94B7800C949B3CEEEFFCE084915F
:1063B0008F01882351F0082E000C990B0E94B780A2
:1063C0000F5F1F4FF8018491F4CF20E030E040E0F0
:1063D0005FE3609146047091470480914804909176
:1063E0004904D0CFE9EFFCE084918F01882351F07C
:1063F000082E000C990B0E94B7800F5F1F4FF80109
:106400008491F4CF6091440470914504B1CF209100
:1064100042043091430444E6429FC001439F900DE3
:1064200011246FEF70E00E949CED8B0165367105C1
:1064300010F004E610E0E4EFFCE084917F01882393
:1064400059F0082E000C990B0E94B780FFEFEF1A4D
:10645000FF0AF7018491F3CFB80180E090E036C7DE
:10646000E0EFFCE084918F01882351F0082E000CAE
:10647000990B0E94B7800F5F1F4FF8018491F4CFF2
:1064800080E290E00E94B780ECEEFCE084918F0106
:10649000882351F0082E000C990B0E94B7800F5FE3
:1064A0001F4FF8018491F4CF60913204709133044E
:1064B00080913404909135040E94ECD780E290E002
:1064C0000E94B780E8EEFCE084918F01882351F0B0
:1064D000082E000C990B0E94B7800F5F1F4FF80128
:1064E0008491F4CF60913604709137048091380420
:1064F000909139040E94ECD780E290E00E94B7802E
:10650000E4EEFCE084918F01882351F0082E000C0A
:10651000990B0E94B7800F5F1F4FF8018491F4CF51
:1065200060913A0470913B0480913C0490913D0449
:106530000E94ECD780E290E0A0C58091310A8823C8
:1065400009F450C0EFEDFCE084918F01882351F0F5
:10655000082E000C990B0E94B7800F5F1F4FF801A7
:106560008491F4CF8091320A882359F18091FD0BF8
:10657000882329F18091A70C9091A80CA091A90CD7
:10658000B091AA0C0097A105B105C1F0BC01CD01E5
:106590006D597F4F8F4F9F4F24E630E040E050E031
:1065A0000E9455EA6091AB0C7091AC0C8091AD0CDF
:1065B0009091AE0C0E9455EA822F01C080E090E0DD
:1065C000E6CEEBEDFCE084918F01882309F4E3CE65
:1065D000082E000C990B0E94B7800F5F1F4FF80127
:1065E0008491F3CFE3EDFCE084918F01882309F4DB
:1065F000D2CE082E000C990B0E94B7800F5F1F4F60
:10660000F8018491F3CFEEECFCE084918F018823B4
:1066100051F0082E000C990B0E94B7800F5F1F4F9E
:10662000F8018491F4CF8091430E9091440EA09193
:10663000450EB091460E892B8A2B8B2B09F477C01F
:106640000E94FF58A50194010E9455EA69017A0150
:106650006091430E7091440E8091450E9091460ECC
:10666000A50194010E9455EA8601021B130BC80183
:106670006CE370E00E9488EDCB019927EAE0F0E03E
:10668000BF010E949CED282FCB01BF010E949CED11
:10669000805D80932904205D20932A0410922B04AE
:1066A00089E294E00E94EBD780E290E00E94B780FC
:1066B000ECECFCE084917F01882359F0082E000C5B
:1066C000990B0E94B780FFEFEF1AFF0AF701849140
:1066D000F3CF80E290E00E94B780C8016CE370E0E5
:1066E0000E9488ED6AE070E00E949CED605D60931E
:1066F0002904805D80932A0410922B0489E294E09F
:106700000E94EBD780E290E00E94B780EAECFCE0C8
:1067100084918F01882309F43ECE082E000C990B3A
:106720000E94B7800F5F1F4FF8018491F3CF80E282
:1067300090E00E94B780E2ECFCE084918F01882316
:1067400009F429CE082E000C990B0E94B7800F5F28
:106750001F4FF8018491F3CF10926D0E80910901C3
:1067600080FF11C0EEEBFCE084918F01882309F4D7
:1067700012CE082E000C990B0E94B7800F5F1F4F9E
:10678000F8018491F3CF83E50E9487D7882341F0F5
:106790000E94A2D70E94FCEB7093420E6093410EC0
:1067A000EAEBFCE084918F01882351F0082E000C65
:1067B000990B0E94B7800F5F1F4FF8018491F4CFAF
:1067C0008DE090E00E94B7808AE090E00E94B78060
:1067D00080918B0E882309F442C28091410E9091E2
:1067E000420E8430910509F4C8C08830910509F43F
:1067F0007DC1892B09F0E7C3EEEDFAE084918F01AA
:10680000882351F0082E000C990B0E94B7800F5F6F
:106810001F4FF8018491F4CF8DE090E00E94B78083
:106820008AE090E00E94B780E3EDFAE084918F0166
:10683000882351F0082E000C990B0E94B7800F5F3F
:106840001F4FF8018491F4CF8DE090E00E94B78053
:106850008AE090E00E94B780E7ECFAE084918F0133
:10686000882351F0082E000C990B0E94B7800F5F0F
:106870001F4FF8018491F4CF8DE090E00E94B78023
:106880008AE090E00E94B780EBEBFAE084918F0100
:10689000882351F0082E000C990B0E94B7800F5FDF
:1068A0001F4FF8018491F4CF8DE090E00E94B780F3
:1068B0008AE090E00E94B780EDEAFAE084918F01CF
:1068C000882351F0082E000C990B0E94B7800F5FAF
:1068D0001F4FF8018491F4CF8DE090E00E94B780C3
:1068E0008AE090E00E94B780EFE9FAE084918F019E
:1068F000882351F0082E000C990B0E94B7800F5F7F
:106900001F4FF8018491F4CF8DE090E00E94B78092
:106910008AE090E00E94B780E2E9FAE084918F017A
:10692000882351F0082E000C990B0E94B7800F5F4E
:106930001F4FF8018491F4CF8DE090E00E94B78062
:106940008AE090E00E94B780E5E8FAE084918F0148
:10695000882351F0082E000C990B0E94B7800F5F1E
:106960001F4FF8018491F4CF8DE090E00E94B78032
:106970008AE090E00E94B78026C3E7E7FAE08491BE
:106980008F01882351F0082E000C990B0E94B780CC
:106990000F5F1F4FF8018491F4CF8DE090E00E94CB
:1069A000B7808AE090E00E94B780E9E6FAE084913F
:1069B0008F01882351F0082E000C990B0E94B7809C
:1069C0000F5F1F4FF8018491F4CF8DE090E00E949B
:1069D000B7808AE090E00E94B780E3E5FAE0849116
:1069E0008F01882351F0082E000C990B0E94B7806C
:1069F0000F5F1F4FF8018491F4CF8DE090E00E946B
:106A0000B7808AE090E00E94B780EDE3FAE08491DD
:106A10008F01882351F0082E000C990B0E94B7803B
:106A20000F5F1F4FF8018491F4CF8DE090E00E943A
:106A3000B7808AE090E00E94B780EBE2FAE08491B0
:106A40008F01882351F0082E000C990B0E94B7800B
:106A50000F5F1F4FF8018491F4CF8DE090E00E940A
:106A6000B7808AE090E00E94B780E9E1FAE0849183
:106A70008F01882351F0082E000C990B0E94B780DB
:106A80000F5F1F4FF8018491F4CF8DE090E00E94DA
:106A9000B7808AE090E00E94B780EBE0FAE0849152
:106AA0008F01882351F0082E000C990B0E94B780AB
:106AB0000F5F1F4FF8018491F4CF8DE090E00E94AA
:106AC000B7808AE090E00E94B780EDEFF9E0849112
:106AD0008F01882309F448CF082E000C990B0E94DF
:106AE000B7800F5F1F4FF8018491F3CFE6EFF9E015
:106AF00084918F01882351F0082E000C990B0E947D
:106B0000B7800F5F1F4FF8018491F4CF8DE090E0C4
:106B10000E94B7808AE090E00E94B780EFEEF9E033
:106B200084918F01882351F0082E000C990B0E944C
:106B3000B7800F5F1F4FF8018491F4CF8DE090E094
:106B40000E94B7808AE090E00E94B780E8EDF9E00B
:106B500084918F01882351F0082E000C990B0E941C
:106B6000B7800F5F1F4FF8018491F4CF8DE090E064
:106B70000E94B7808AE090E00E94B780E1ECF9E0E3
:106B800084918F01882351F0082E000C990B0E94EC
:106B9000B7800F5F1F4FF8018491F4CF8DE090E034
:106BA0000E94B7808AE090E00E94B780EAEAF9E0AC
:106BB00084918F01882351F0082E000C990B0E94BC
:106BC000B7800F5F1F4FF8018491F4CF8DE090E004
:106BD0000E94B7808AE090E00E94B780E3E9F9E084
:106BE00084918F01882351F0082E000C990B0E948C
:106BF000B7800F5F1F4FF8018491F4CF8DE090E0D4
:106C00000E94B7808AE090E00E94B780E5E8F9E052
:106C100084918F01882351F0082E000C990B0E945B
:106C2000B7800F5F1F4FF8018491F4CF8DE090E0A3
:106C30000E94B7808AE090E00E94B780E7E7F9E021
:106C400084918F01882309F48FCE082E000C990BB4
:106C50000E94B7800F5F1F4FF8018491F3CF80919E
:106C6000320A882309F486C181E08093AF0C109228
:106C7000B10C1092B00C81E89AE00E94669A8BE108
:106C8000E1E8FAE0DE01159601900D928A95E1F7B0
:106C900080917F0A9091800A9C838B838DEE92E095
:106CA0009A83898340E050E0BE016F5F7F4F80E0B0
:106CB00090E00E94ED82CE0101960E94C2A0C09099
:106CC000B00CD090B10C0091410E1091420EC60153
:106CD000801B910B049720F06801F3E0CF0ED11CCC
:106CE00058E6452E59E0552E69E5662E69E0762E68
:106CF000C016D10608F467C10115110509F0A1C03D
:106D000065E37AE081E89AE00E942E9962E273E0FE
:106D100085E39AE00E940EEE892B09F04AC0F20149
:106D2000849148E6E42E49E0F42E882359F0082E99
:106D3000000C990B0E94B780FFEFEF1AFF0AF701D2
:106D40008491F3CF8DE090E00E94B7808AE090E0DC
:106D50000E94B780F301849139E5E32E39E0F32EE8
:106D6000882359F0082E000C990B0E94B780FFEF82
:106D7000EF1AFF0AF7018491F3CF8DE090E00E94B3
:106D8000B7808AE090E00E94B7804AE060E070E05F
:106D9000CB010E940F97E9E4F9E084917F012FEF86
:106DA000E21AF20A882309F4E2C00E94EE93F70186
:106DB000F4CFE5E4F9E084917F01882359F0082EAF
:106DC000000C990B0E94B780FFEFEF1AFF0AF70142
:106DD0008491F3CF8DE090E00E94B7808AE090E04C
:106DE0000E94B780F101849121E4E22E29E0F22E85
:106DF000882359F0082E000C990B0E94B780FFEFF2
:106E0000EF1AFF0AF7018491F3CF8DE090E00E9422
:106E1000B7808AE090E00E94B7804AE060E070E0CE
:106E2000CB010E940F97ECE3F9E084917F012FEFF3
:106E3000E21AF20A882309F49AC00E94EE93F7013D
:106E4000F4CF60E070E0C80101970E94B3848091A4
:106E5000330A882309F45FC0EAE3F9E084917F01F3
:106E6000882359F0082E000C990B0E94B780FFEF81
:106E7000EF1AFF0AF7018491F3CF85E39AE00E94AD
:106E8000EBD78DE090E00E94B7808AE090E00E940E
:106E9000B780E8E3F9E084917F01882359F0082E58
:106EA000000C990B0E94B780FFEFEF1AFF0AF70161
:106EB0008491F3CF82E49AE00E94EBD78DE090E0DA
:106EC0000E94B7808AE090E00E94B780C801A0E0ED
:106ED000B0E04AE0BC01CD010E940F97E6E3F9E083
:106EE00084917F012FEFE21AF20A882321F00E9499
:106EF000EE93F701F5CF92E4E92E9AE0F92EF7012F
:106F000081917F01882319F00E94EE93F8CF8AE0E7
:106F10000E94EE932CC085E39AE00E94EBD78DE0AF
:106F200090E00E94B7808AE090E00E94B78082E4FF
:106F30009AE00E94EBD78DE090E00E94B7808AE053
:106F400090E00E94B780C801A0E0B0E04AE0BC0138
:106F5000CD010E940F9782E4E82E8AE0F82EF70117
:106F600081917F01882399F20E94EE93F8CF0F5F01
:106F70001F4FBECEE7E2F9E084918F01882351F0E4
:106F8000082E000C990B0E94B7800F5F1F4FF8016D
:106F90008491F4CF8DE090E00E94B7808AE090E089
:106FA0000E94B780E8E1F9E084918F01882309F419
:106FB000DBCC082E000C990B0E94B7800F5F1F4F8F
:106FC000F8018491F3CFE6EBFCE084918F018823F4
:106FD00009F4E1C9082E000C990B0E94B7800F5FDD
:106FE0001F4FF8018491F3CF8091310A882339F043
:106FF0000E941F82A0C48091310A8823E9F00E9478
:107000003BB199C480913F0E823019F0833609F06C
:1070100092C40E94FE81E2EBFCE084918F01882300
:1070200009F4B9C9082E000C990B0E94B7800F5FB4
:107030001F4FF8018491F3CF80913F0E833609F002
:107040007AC4DDCF89EA9CE00E94E5A08091B30973
:107050009091B409891B8F7009F06DC480913F0E27
:10706000823009F468C4833609F099C464C48DE0A1
:1070700090E00E94B7808AE090E00E94B7808BC9C0
:107080008091B3099091B409891B8F7009F053C4A2
:1070900080913F0E823009F44EC4833609F44BC40C
:1070A0008091FD0B8111CFC446C483E50E9487D730
:1070B000811126C083E40E9487D7882309F43BC44A
:1070C0008091B3099091B409891B8F7009F033C482
:1070D00020E030E040E251E460913A0470913B04DA
:1070E00080913C0490913D040E9467E687FF08C0B0
:1070F00086E99CE09093A4078093A3070E941A94CA
:107100000E94A2D720E030E0A9010E9467E687FD37
:1071100010C00E94A2D720E030E849E853E40E9462
:10712000D9EC18164CF00E94A2D70E94FCEBCB01C0
:1071300005C080E090E002C083E191E00E94F45934
:10714000FAC383E50E9487D7882309F4F4C30E9419
:10715000A2D720E030E0A9010E9467E687FD10C0B9
:107160000E94A2D720E030E046E153E40E94D9EC2F
:1071700018164CF00E94A2D70E94FCEBCB0105C070
:1071800080E090E002C086E990E00E94274ED3C3E1
:1071900083E50E9487D78823D9F00E94A2D720E0F8
:1071A00030E04FE753E40E94CCE620E030E048ECCA
:1071B00052E40E948FEB0E94FCEB6F3F710519F0C7
:1071C00010F06FEF70E07093430460934204E3C8E3
:1071D0008FEF90E09093430480934204DCC8809149
:1071E000B3099091B409891B8F7009F0D4C88091BC
:1071F000310A8111D0C80E949B865F9A8091310428
:107200008E7F809331048A9A479A809131048D7FD2
:1072100080933104809108018095817080930601EC
:10722000479A809131048B7F80933104129AB3C8BE
:1072300083E50E9487D7882319F10E94A2D720E016
:1072400030E040E252E40E9467E687FD0FC00E94F2
:10725000A2D720E030EC49E754E40E94D9EC18169C
:1072600044F00E94A2D70E94F7EB05C068E270E0EC
:1072700002C067EE73E070930302609302025BC387
:10728000E0E9FCE084918F01882351F0082E000C86
:10729000990B0E94B7800F5F1F4FF8018491F4CFC4
:1072A000C0900202D09003020D2C000CEE08FF08E3
:1072B000F7FE0EC06DE28AE99FE00E94E14A662770
:1072C0007727CB016C197D098E099F094AE003C01D
:1072D0004AE0C701B6010E94ABD75DC88091B309EF
:1072E0009091B409891B8F7009F025C380913F0EDE
:1072F000823009F420C3833609F0EBC21CC38091AD
:10730000B3099091B409891B8F7009F044C880912A
:107310003F0E823009F43FC8833609F0B6C33BC83C
:107320008091B3099091B409891B8F7009F003C350
:1073300080913F0E823009F4FEC2833609F0FBC40F
:10734000FAC28091B3099091B409891B8F7009F03A
:10735000F2C280913F0E823009F4EDC2833609F00B
:1073600020C5E9C28091B3099091B409891B8F703F
:1073700009F0E1C280913F0E823009F4DCC283360D
:1073800009F045C5D8C280916D0E811103C00E94DD
:10739000BC80C4C18E3271F580916E0E8E3209F0C0
:1073A00046C18091D20B882309F4B8C181508093E3
:1073B000D20B882361F090E001974FE1489F900144
:1073C000499F300D1124C9018456954F02C08EE5A6
:1073D0009AE02BE1FC013496A1E8BAE001900D920D
:1073E0002A95E1F7FC01828193819093800A809332
:1073F0007F0A94C18C3309F01AC164E273E08DE610
:107400009EE00E940EEE892B21F481E080938B0E8A
:1074100085C163E373E08DE69EE00E940EEE892B4A
:1074200079F4E4EFF8E084918F010F5F1F4F882318
:1074300021F00E94EE93F801F6CF86ED98E0E4C0CB
:107440006AE473E08DE69EE00E940EEE892B79F4EB
:10745000E2EBF8E084918F010F5F1F4F882321F04A
:107460000E94EE93F801F6CF8EE998E0CDC061E678
:1074700073E08DE69EE00E940EEE892B79F4E3E83E
:10748000F8E084918F010F5F1F4F882321F00E9445
:10749000EE93F801F6CF8EE798E0B6C06FE673E0A2
:1074A0008DE69EE00E940EEE892B79F4E3E6F8E08B
:1074B00084918F010F5F1F4F882321F00E94EE936C
:1074C000F801F6CF8EE598E09FC06DE773E08DE69A
:1074D0009EE00E940EEE892B79F4E3E4F8E08491BB
:1074E0008F010F5F1F4F882321F00E94EE93F80158
:1074F000F6CF8AE398E088C06BE873E08DE69EE003
:107500000E940EEE892B71F407E118E0F8018491D6
:10751000882329F00F5F1F4F0E94EE93F7CF80E181
:1075200098E072C061EA73E08DE69EE00E940EEE84
:10753000892B79F4E1EFF7E084918F010F5F1F4F02
:10754000882321F00E94EE93F801F6CF8AEE97E0AF
:107550005BC063EB73E08DE69EE00E940EEE892B2C
:1075600079F4E2EDF7E084918F010F5F1F4F8823DC
:1075700021F00E94EE93F801F6CF81EC97E044C031
:107580006EEB73E08DE69EE00E940EEE892B79F49F
:10759000E8EAF7E084918F010F5F1F4F882321F005
:1075A0000E94EE93F801F6CF86E997E02DC06AECD1
:1075B00073E08DE69EE00E940EEE892B79F4EBE7F6
:1075C000F7E084918F010F5F1F4F882321F00E9405
:1075D000EE93F801F6CF89E697E016C068ED73E008
:1075E0008DE69EE00E940EEE892BA9F4EFE4F7E011
:1075F00084918F010F5F1F4F882321F00E94EE932B
:10760000F801F6CF8DE397E09093A4078093A3074A
:107610000E941A9483C065EE73E08DE69EE00E949E
:107620000EEE892B09F07AC010928B0E77C01D8266
:1076300018861C821B828DEE92E09A83898380914A
:10764000840A811103C06EE57AE002C06DE77AE03A
:107650006115710519F06C5F7F4F02C060E070E04A
:1076600021E04DE65EE0CE0105960E94959E8823BE
:1076700061F18BE1FE013596A1E8BAE001900D922F
:107680008A95E1F72B813C813093800A20937F0A11
:107690008091D20B8A3008F03DC091E0980F909312
:1076A000D20BFFE18F9FC0011124DC01A056B54F22
:1076B0004BE1E1E8FAE001900D924A95E1F7FC0117
:1076C000E456F54F3383228325C0E6EEFDE1849135
:1076D0008F010F5F1F4F882321F00E94EE93F80166
:1076E000F6CFE7E2F7E084918F010F5F1F4F882309
:1076F00021F00E94EE93F801F6CF0DE61EE0F801AE
:1077000081918F01882319F00E94EE93F8CF8AE0CF
:107710000E94EE93CE0101960E94C2A010926D0EBF
:107720008091090180FF07C1E4EDFBE084918F01A6
:10773000882311F40C94CB31082E000C990B0E9475
:10774000B7800F5F1F4FF8018491F2CF8FE40E9442
:1077500087D781110C94CB3183E40E9487D70C9496
:10776000CB3183E50E9487D7811159C08FE40E94F5
:1077700087D7882319F08CE99BE007C084E50E9435
:1077800087D7882349F084E79BE09093A4078093F0
:10779000A3070E941A9443C083E40E9487D78823DA
:1077A00019F08BE49BE0F1CF81E50E9487D7882315
:1077B00019F083E29BE0E9CF88E40E9487D7882311
:1077C000C9F0EFE1FBE084918F01882351F0082E8E
:1077D000000C990B0E94B7800F5F1F4FF801849136
:1077E000F4CF8DE090E00E94B7808AE090E00E94A4
:1077F000B78015C08CE40E9487D7882381F0EBE125
:10780000FBE084918F01882361F3082E000C990B13
:107810000E94B7800F5F1F4FF8018491F4CFE3EE11
:10782000FBE084918F01882311F40C94CB31082E56
:10783000000C990B0E94B7800F5F1F4FF8018491D5
:10784000F2CF8091B3098091B4090C94CB3183E5D8
:107850000E9487D7882309F46EC083EF9AE0909343
:10786000A4078093A3070E941A94E3EEFBE084919F
:107870008F01882311F40C94CB31082E000C990B46
:107880000E94B7800F5F1F4FF8018491F2CFEEEE98
:10789000FAE084918F01882351F0082E000C990B97
:1078A0000E94B7800F5F1F4FF8018491F4CFE9EE7B
:1078B000FAE084918F01882311F40C94CB31082EC7
:1078C000000C990B0E94B7800F5F1F4FF801849145
:1078D000F2CF88E50E9487D7811106C089E50E9412
:1078E00087D7882309F4C3C088E50E9487D78823F7
:1078F00041F08AE89CE09093A4078093A3070E943C
:107900001A9489E50E9487D7882341F084E89CE097
:107910009093A4078093A3070E941A948AE50E947B
:1079200087D7882341F08EE79CE09093A40780934B
:10793000A3070E941A948091380E9091390E0196F7
:1079400064E070E00E949CED9093390E8093380EB5
:107950008091340E9091350E01969093350E809360
:10796000340E10923C0E10923B0E0C94AC304091B1
:10797000380E5091390E9F012F5F3F4F30933C0ED0
:1079800020933B0E90E6949F9001959F300D11241B
:107990002C54334FE20FF31F80830C94AC300091D2
:1079A0003D0E10913E0E780124E0E20EF11C6AE2D9
:1079B00070E0C7010E9403EEF80124812F3221F408
:1079C000B8016B5F7F4F03C02C3339F4B7018DE6EC
:1079D0009EE00E9417EE0C94CB3110926D0E009732
:1079E00019F0FC013197108280913D0E90913E0E6E
:1079F00040E061E004960E94B5D58091FD0B88239C
:107A000089F0E5EAFCE084918F01882309F42FCB0B
:107A1000082E000C990B0E94B7800F5F1F4FF801D2
:107A20008491F3CFE1EAFCE084918F01882309F48B
:107A30001ECB082E000C990B0E94B7800F5F1F4FC2
:107A4000F8018491F3CF0E94FE81EDE9FCE084917E
:107A50008F01882311F40C94CB31082E000C990B64
:107A60000E94B7800F5F1F4FF8018491F2CF8AE523
:107A70000E9487D7811138CF83E40E9487D788235B
:107A800009F459CF8AE79CE050CF86E40E9487D75B
:107A9000882309F44DC10E94A2D70E94FCEB8B0100
:107AA00086E79CE09093A4078093A3070E941A9412
:107AB00088E50E9487D7882309F451C00E94A2D785
:107AC0002B013C012DEC3CEC4CE45EE30E9467E6AC
:107AD0009E012F5F3F4F7901181674F020E030E0CF
:107AE000A901C301B2010E94D9EC18162CF41F930E
:107AF0000F938BE69CE005C12DEC3CEC4CEC5DEB70
:107B0000C301B2010E9467E618167CF020E030E065
:107B100040E85FEBC301B2010E94D9EC18162CF4C7
:107B20001F930F938FE59CE0ECC01F930F93C3014D
:107B3000B2010E94F7EB7F936F9385E59CE09F93E2
:107B40008F93FF92EF920E9439E60FB6F894DEBF52
:107B50000FBECDBFCE0101960E94F593DFC089E52F
:107B60000E9487D7882309F441C00E94A2D72B0125
:107B70003C012DEC3CEC4CE45EE30E9467E6FE0128
:107B800031967F01181674F020E030E0A901C3019E
:107B9000B2010E94D9EC18162CF41F930F938AE4BB
:107BA0009CE0AFC02DEC3CEC4CEC5DEBC301B201B2
:107BB0000E9467E618167CF020E030E040E85FEBBA
:107BC000C301B2010E94D9EC18162CF41F930F9335
:107BD0008EE39CE096C01F930F93C301B2010E94F5
:107BE000F7EB7F936F9384E39CE0A9CF8AE50E9433
:107BF00087D7882309F441C00E94A2D72B013C01FA
:107C00002DEC3CEC4CE45EE30E9467E6FE0131960D
:107C10007F01181674F020E030E0A901C301B20121
:107C20000E94D9EC18162CF41F930F9389E29CE064
:107C300068C02DEC3CEC4CEC5DEBC301B2010E9442
:107C400067E618167CF020E030E040E85FEBC30107
:107C5000B2010E94D9EC18162CF41F930F938DE1FA
:107C60009CE04FC01F930F93C301B2010E94F7EB3A
:107C70007F936F9383E19CE062CF85E40E9487D776
:107C8000882309F44BC00E94A2D72B013C012DECA4
:107C90003CEC4CE45EE30E9467E6FE0131967F0116
:107CA000181674F020E030E0A901C301B2010E946F
:107CB000D9EC18162CF41F930F9388E09CE021C098
:107CC0002DEC3CEC4CEC5DEBC301B2010E9467E68D
:107CD00018167CF020E030E040E85FEBC301B20111
:107CE0000E94D9EC18162CF41F930F938CEF9BE095
:107CF00008C0C301B2010E94F7EB7F936F9381EF3D
:107D00009BE09F938F93FF92EF920E9439E60F9032
:107D10000F900F900F900F900F901CCF8DEE9BE067
:107D20009093A4078093A3070E941A940C94CB31DC
:107D300000E010E0B5CE20E030E040E251E4609198
:107D40003A0470913B0480913C0490913D040E9460
:107D500067E687FF08C086EE9BE09093A4078093B8
:107D6000A3070E941A9482E390E0909345048093C5
:107D700044040E94B77688EC90E00E94F459E3EE48
:107D8000FBE084918F01882311F40C94CB31082EF1
:107D9000000C990B0E94B7800F5F1F4FF801849170
:107DA000F2CF20E030E040E251E460913A0470917B
:107DB0003B0480913C0490913D040E9467E687FF5C
:107DC00008C08CED9BE09093A4078093A3070E94CA
:107DD0001A9480E590E090934504809344040E94B7
:107DE000B77680EF90E00E94F459E3EEFBE08491D7
:107DF0008F01882311F40C94CB31082E000C990BC1
:107E00000E94B7800F5F1F4FF8018491F2CF80E08E
:107E100090E00E94F45910924504109244040E948C
:107E2000B776E8EDFBE084918F01882311F40C9480
:107E3000CB31082E000C990B0E94B7800F5F1F4FAB
:107E4000F8018491F2CF6F960FB6F894DEBF0FBEA3
:107E5000CDBFDF91CF911F910F91FF90EF90DF90F9
:107E6000CF90BF90AF909F908F907F906F905F90DA
:107E70004F903F902F9008952F923F924F925F9294
:107E80006F927F928F929F92AF92BF92CF92DF922A
:107E9000EF92FF920F931F93CF93DF93CDB7DEB78F
:107EA00062970FB6F894DEBF0FBECDBFF8948FEF88
:107EB0009FEF90938900809388002AE02A8B212CE1
:107EC000312C78948091A2049091A304A091A404F1
:107ED000B091A504892B8A2B8B2B09F016C28091B7
:107EE0001A078823E1F010921A07809118079091E1
:107EF0001907892B09F409C210925A041092190724
:107F0000109218079091B3098091B409981709F459
:107F1000FCC18091B4098F5F8F708093B409809108
:107F2000180790911907892B09F4EFC140919E041D
:107F300050919F046091A0047091A10480919A04D3
:107F400090919B04A0919C04B0919D040091910498
:107F500010E020E030E0841B950BA60BB70B081750
:107F600019072A073B0710F4D901C801E82F840F2D
:107F7000951FA61FB71F80939E0490939F04A09304
:107F8000A004B093A1042091840030918500225E6A
:107F90003F4F40917604509177046091780470913E
:107FA00079048091660490916704A0916804B0916F
:107FB0006904840F951FA61FB71F809376049093C2
:107FC0007704A0937804B0937904B7FD1CC0889A15
:107FD0008091821090918310A0918410B0918510AF
:107FE00040910402042E000C550B660B770B840F96
:107FF000951FA61FB71F8093821090938310A093A4
:108000008410B093851040917A0450917B04609164
:108010007C0470917D0480916A0490916B04A0911E
:108020006C04B0916D04840F951FA61FB71F809339
:108030007A0490937B04A0937C04B0937D04B7FDF5
:108040001CC08E9A8091861090918710A091881004
:10805000B091891040910502042E000C550B660B5F
:10806000770B840F951FA61FB71F809386109093E0
:108070008710A0938810B093891040917E0450918E
:108080007F04609180047091810480916E049091CE
:108090006F04A0917004B0917104840F951FA61F06
:1080A000B71F80937E0490937F04A0938004B093C5
:1080B0008104B7FD3FC080915404F09106028823EB
:1080C000C9F08091520482FF02C0F7FD06C0809182
:1080D0005104882311F40C94F44880915204909137
:1080E000530493FF02C0F7FD0CC08091500481112E
:1080F00008C006C080910B018095887080930901AB
:10810000419A40918A1050918B1060918C1070911F
:108110008D108F2FFF0F990BAA0BBB0B840F951F90
:10812000A61FB71F80938A1090938B10A0938C107A
:10813000B0938D1040918204509183046091840427
:10814000709185048091720490917304A0917404DD
:10815000B0917504840F951FA61FB71F80938204EA
:1081600090938304A0938404B0938504B7FD3AC030
:1081700040918E1050918F106091901070919110DD
:10818000C09007020C2C000CDD08EE08FF084C0D17
:108190005D1D6E1D7F1D40938E1050938F10609358
:1081A000901070939110409162045091630460911B
:1081B000640470916504841B950BA60BB70B809328
:1081C000820490938304A0938404B09385049091D7
:1081D000550480918F0493FF02C0815001C08F5FCE
:1081E00080938F048091840090918500821793077B
:1081F000C8F38091760490917704A0917804B091AF
:108200007904B7FD15C040916204509163046091F8
:10821000640470916504841B950BA60BB70B8093C7
:10822000760490937704A0937804B09379048898A7
:1082300080917A0490917B04A0917C04B0917D049C
:10824000B7FD15C0409162045091630460916404CD
:1082500070916504841B950BA60BB70B80937A0471
:1082600090937B04A0937C04B0937D048E988091BE
:108270007E0490917F04A0918004B0918104B7FDA9
:108280003AC040916204509163046091640470911B
:108290006504841B950BA60BB70B80937E0490930B
:1082A0007F04A0938004B0938104809154048823B8
:1082B000E1F08091520482FF04C08091060287FDA4
:1082C00005C080915104882309F496C78091520417
:1082D0009091530493FF04C08091060287FD0BC068
:1082E00080915004811107C005C080910B018870F6
:1082F000809309014198E15041F080918400909170
:10830000850082179307C8F342CE809111029091A5
:108310001202A0911302B0911402892B8A2B8B2B8D
:1083200009F091C080919004882309F453C0809093
:108330009E0490909F04A090A004B090A104C090CF
:108340008B04D0908C04E0908D04F0908E044091CA
:108350008F04C814D904EA04FB0480F480915B0400
:1083600090915C0420915F043091600428173907D4
:1083700028F4415040938F04019714C08C149D043D
:10838000AE04BF04E0F480915B0490915C04209102
:108390005D0430915E048217930788F44F5F409329
:1083A0008F04019690935C0480935B0440910D02CE
:1083B00050910E0260910F02709110020EC08FEF6B
:1083C0009FEFDC0180930D0290930E02A0930F02A9
:1083D000B09310024FEF5FEFBA0180918F0487FDD9
:1083E00002C0169A01C01698809184009091850071
:1083F0004E9620918F042223F1F0149A209184004C
:108400003091850028173907C8F320918F0427FF82
:1084100002C02F5F01C0215020938F041498209137
:108420008F04222331F32091840030918500281796
:108430003907C8F3DDCF40931102509312026093C5
:108440001302709314028091A2049091A304A0914E
:10845000A404B091A504892B8A2B8B2B09F049C663
:10846000A0911807B0911907109711F40C949D4A28
:1084700080909E0490909F04A090A004B090A104CE
:1084800040919A0450919B0460919C0470919D04CA
:1084900084169506A606B706D8F010925A041092D4
:1084A0001907109218079091B3098091B409981791
:1084B00011F40C949D4A8091B4098F5F8F70809362
:1084C000B40940EDC42E47E0D42EE12CF12C1AC49F
:1084D000409196045091970460919804709199048A
:1084E000481559056A057B0508F4AAC14091920414
:1084F000509193046091940470919504D6960D91D7
:108500001D912D913C91D997401751076207730730
:1085100008F077C1411551056105710549F4809056
:10852000560490905704A0905804B090590464C128
:10853000E12CF980842E952F862F0A811B81FD81E5
:10854000EE813F8128859C80E091EF17E89D912C7A
:10855000FF273091F017389D900CF11D1090F11706
:10856000189CF00DE99F900CF11D399FF00DE89FCC
:10857000F00D092D1F2F099DE12D332722270F9F75
:10858000E00D311D2E1D199DE00D311D2E1D1F9F6B
:10859000300D211D032F122F099DF12C3327222787
:1085A0000F9FF00C311D2E1D199DF00C311D2E1D3D
:1085B0001F9F300D211D032F122FEE278090560490
:1085C00090915704809158040090B2040E2809F449
:1085D00083C03091AE04309FE1198E089E098E0948
:1085E0002091AF04209FE01981089E098E09F09028
:1085F000B004F09E801891098E09319FE01981081E
:108600009E098E09219F801891098E09F19E90196B
:108610008109099DF12C332722270F9FF00C311D72
:108620002E1D199DF00C311D2E1D1F9F300D211D7B
:10863000032F122F3091AA04309FE10D8E1C9E1D36
:108640008E1D2091AB04209FE00D811C9E1D8E1D70
:10865000F090AC04F09E800C911D8E1D319FE00DBA
:10866000811C9E1D8E1D219F800C911D8E1DF19ED3
:10867000900D811D099DF12C332722270F9FF00CAF
:10868000311D2E1D199DF00C311D2E1D1F9F300D0B
:10869000211D032F122F3091A604309FE1198E085F
:1086A0009E098E092091A704209FE01981089E0948
:1086B0008E09F090A804F09E801891098E09319FD0
:1086C000E01981089E098E09219F801891098E0961
:1086D000F19E9019810982C03091AE04309FE10D66
:1086E0008E1C9E1D8E1D2091AF04209FE00D811CCD
:1086F0009E1D8E1DF090B004F09E800C911D8E1D6D
:10870000319FE00D811C9E1D8E1D219F800C911DAF
:108710008E1DF19E900D811D099DF12C332722277E
:108720000F9FF00C311D2E1D199DF00C311D2E1DBB
:108730001F9F300D211D032F122F3091AA04309F4F
:10874000E1198E089E098E092091AB04209FE01943
:1087500081089E098E09F090AC04F09E8018910962
:108760008E09319FE01981089E098E09219F80188A
:1087700091098E09F19E90198109099DF12C3327E9
:1087800022270F9FF00C311D2E1D199DF00C311D5D
:108790002E1D1F9F300D211D032F122F3091A60477
:1087A000309FE10D8E1C9E1D8E1D2091A704209FE1
:1087B000E00D811C9E1D8E1DF090A804F09E800C83
:1087C000911D8E1D319FE00D811C9E1D8E1D219FD0
:1087D000800C911D8E1DF19E900D811D11249C8297
:1087E000F9820A831B83FD83EE833F832887912CC4
:1087F000992AA12CB12CA82A8DE395E121E0298B9F
:1088000014C0D2968D909D90AD90BC90D597F4CF2A
:10881000B694A79497948794D988DD0CD98A049646
:1088200025E18935920709F4EDC4FC010591159104
:1088300025913491081519052A053B0548F3E2C432
:1088400040908B0450908C0460908D0470908E0446
:10885000481459046A047B0408F0C3C180918A0457
:10886000811121C0FD01EE5BFF4FE080F1800281AC
:10887000138178962081318142815381D2966D9106
:108880007D918D919C91D5970E948DC4DD24D394C8
:10889000D0928A04E0911807F091190782A993A950
:1088A000A4A9B5A98EC14091860450918704609116
:1088B000880470918904DA960D911D912D913C9157
:1088C000DD97401751076207730708F073C1411520
:1088D00051056105710549F4809156049091570442
:1088E000A0915804B09159046CC1F0E0E985842F3F
:1088F000352F262FAA857B856C855D85BE854F85A6
:108900009889B091EF17B89F612D55274091F017C6
:10891000489F600D511D1090F117189E500DB39F88
:10892000600D511D439F500DB29F500DA62F752F06
:10893000A69FB12D44279927A59FB00D411D9F1FCC
:10894000769FB00D411D9F1F759F400D911DA42F57
:10895000792FA69FE12D44279927A59FE00D411D62
:108960009F1F769FE00D411D9F1F759F400D911D1C
:10897000A42F792FBB278091560430915704209162
:1089800058040090B2040F2A09F483C04091AE0449
:108990004A9FB1198F0B3F0B2F0B9091AF049A9FF9
:1089A000B01981093F0B2F0BE091B004EA9F8019A9
:1089B00031092F0B479FB01981093F0B2F0B979F50
:1089C000801931092F0BE79F30192109A69FE12D4E
:1089D00044279927A59FE00D411D9F1F769FE00D1D
:1089E000411D9F1F759F400D911DA42F792F409110
:1089F000AA044A9FB10D8F1F3F1F2F1F9091AB04F8
:108A00009A9FB00D811D3F1F2F1FE091AC04EA9F7C
:108A1000800D311D2F1F479FB00D811D3F1F2F1F40
:108A2000979F800D311D2F1FE79F300D211DA69FA1
:108A3000E12D44279927A59FE00D411D9F1F769F9B
:108A4000E00D411D9F1F759F400D911DA42F792F93
:108A50004091A6044A9FB1198F0B3F0B2F0B9091A9
:108A6000A7049A9FB01981093F0B2F0BE091A8042E
:108A7000EA9F801931092F0B479FB01981093F0BDD
:108A80002F0B979F801931092F0BE79F3019210970
:108A900082C04091AE044A9FB10D8F1F3F1F2F1F10
:108AA0009091AF049A9FB00D811D3F1F2F1FE09141
:108AB000B004EA9F800D311D2F1F479FB00D811D0F
:108AC0003F1F2F1F979F800D311D2F1FE79F300DD8
:108AD000211DA69FE12D44279927A59FE00D411D4B
:108AE0009F1F769FE00D411D9F1F759F400D911D9B
:108AF000A42F792F4091AA044A9FB1198F0B3F0BE5
:108B00002F0B9091AB049A9FB01981093F0B2F0B4B
:108B1000E091AC04EA9F801931092F0B479FB019EF
:108B200081093F0B2F0B979F801931092F0BE79F6E
:108B300030192109A69FE12D44279927A59FE00D13
:108B4000411D9F1F769FE00D411D9F1F759F400D8A
:108B5000911DA42F792F4091A6044A9FB10D8F1F1C
:108B60003F1F2F1F9091A7049A9FB00D811D3F1F9B
:108B70002F1FE091A804EA9F800D311D2F1F479FF2
:108B8000B00D811D3F1F2F1F979F800D311D2F1F7F
:108B9000E79F300D211D1124E987AA877B876C8709
:108BA0005D87BE874F87988B90E0932BA0E0B0E065
:108BB000A22B07C0A65ABF4F8D919D910D90BC91DD
:108BC000A02D2DE335E141E0498BF9014591559107
:108BD00065917491481759076A077B0708F49CC38D
:108BE000A9C380918F048823E1F0FD01E85BFF4F6A
:108BF0004081518160E070E000910D0210910E0201
:108C000020910F023091100240175107620773073D
:108C100041F010921102109212021092130210925F
:108C200014024091090250910A0260910B02709166
:108C30000C0277FF5FC0AE5ABF4FCD90DD90ED9034
:108C4000FC908DE395E121E0FC0145915591659102
:108C500074914C155D056E057F0550F4F694E7940C
:108C6000D794C794220F049675E18935970761F769
:108C70002093910480E2C816D104E104F10428F4A1
:108C800070E2C72ED12CE12CF12C90E2C91AD10848
:108C9000E108F108C114A8E0DA06E104F10408F4DF
:108CA00005C4B4E0DB9EC0011124835C9E4EFC0130
:108CB000329625913491EC2D6627E39FA001E29F27
:108CC000410D561F0694461F561F112460E070E0A8
:108CD000FC0125913491C901A0E0B0E0841B950B03
:108CE000A60BB70B8093090290930A02A0930B0284
:108CF000B0930C02C0900902D0900A02E0900B02DF
:108D0000F0900C028091180790911907892B09F0B7
:108D1000E8C10E940FC59093190780931807892B0B
:108D200009F4DFC1E0911807F0911907808183FFF2
:108D30003EC085899689A789B08D809382109093D3
:108D40008310A0938410B0938510818D928DA38D94
:108D5000B48D8093861090938710A0938810B09361
:108D60008910858D968DA78DB0A180938A109093E0
:108D70008B10A0938C10B0938D1081A192A1A3A110
:108D8000B4A180938E1090938F10A0939010B09305
:108D900091109091B3098091B409981709F4B9CF53
:108DA0008091B4098F5F8F708093B409B2CFC5886A
:108DB000D688E788F08C81E0C114D104E104F10485
:108DC00009F480E0018D128D238D348D011511057C
:108DD0002105310509F08260458D568D678D70A1A2
:108DE000411551056105710509F0846080935A04AD
:108DF00010928604109287041092880410928904BD
:108E0000109292041092930410929404109295047C
:108E100085A196A1A7A1B0A580939A0490939B04E5
:108E2000A0939C04B0939D04882499245401881A2B
:108E3000990AAA0ABB0A8092820490928304A092A3
:108E40008404B092850480927E0490927F04A09264
:108E50008004B092810480927A0490927B04A09264
:108E60007C04B0927D048092760490927704A09264
:108E70007804B0927904CC0CDD1CEE1CFF1CC0926F
:108E80006604D0926704E0926804F0926904000FCF
:108E9000111F221F331F00936A0410936B04209349
:108EA0006C0430936D04440F551F661F771F409369
:108EB0006E0450936F04609370047093710441A129
:108EC00052A163A174A1440F551F661F771F4093E1
:108ED0007204509373046093740470937504880F44
:108EE000991FAA1FBB1F8093620490936304A093F1
:108EF0006404B093650410929E0410929F04109233
:108F0000A0041092A10482A593A5A4A5B5A5809361
:108F1000960490939704A0939804B093990486A51F
:108F200097A5A0A9B1A980938B0490938C04A093DA
:108F30008D04B0938E0481A580936104DF01A95B49
:108F4000BF4F9C9190939004992339F115962D91E0
:108F50003C9111973093600420935F0412972D91F8
:108F60003C91119730935E0420935D04109211029E
:108F700010921202109213021092140212972D9165
:108F80003C91A90160E070E040930D0250930E0205
:108F900060930F02709310020CC088248A94982C5E
:108FA000540180920D0290920E02A0920F02B09294
:108FB0001002EA5BFF4F90812091550492130AC082
:108FC0002091080230E0482F082E000C550B421764
:108FD000530731F090935504809308020E94DFC438
:108FE0008091370581110E94EFBD2FEF3FEFA9015E
:108FF0002093090230930A0240930B0250930C0213
:10900000E0911807F0911907DF01DE96ED90FD90D1
:109010000D911C9122A933A944A955A9EA5AFF4FE1
:1090200060817181828193810E948DC410928A0433
:10903000E0911807F0911907EA5AFF4F808091805C
:10904000A280B3808DE395E121E0FC01459155912B
:1090500065917491481559056A057B0558F4B694D5
:10906000A79497948794220F0496A9E5B5E1A817D1
:10907000B90759F720939104B0E28B169104A1042B
:10908000B10428F4B0E28B2E912CA12CB12C30E24B
:10909000831A9108A108B108811448E09406A1043C
:1090A000B10408F427C254E0959EC0011124835CEA
:1090B0009E4EFC01329625913491782D6627739F40
:1090C000A001729F410D561F0694461F561F112482
:1090D000FC01C590D490E12CF12CC41AD50AE1080A
:1090E000F108C092A204D092A304E092A404F092EA
:1090F000A5040091A2041091A3042091A40430912E
:10910000A5044091110250911202609113027091D6
:109110001402F02E198BF22FE32F4017510762072C
:10912000730720F4F42E598BF62FE72F8F2D998992
:10913000AF2FBE2F0097E1E0AE07B10520F08FEF13
:109140009FEFA0E0B0E0081B190B2A0B3B0B00932C
:10915000A2041093A3042093A4043093A5044F3FCA
:10916000FFEF5F076F077F0761F0481B590B6A0B22
:109170007B0B409311025093120260931302709381
:109180001402F8942091840030918500205F3F4FB5
:109190004A8941504A8B442341F0280E391E221639
:1091A000330610F40C94613F01C01901309289001C
:1091B00020928800789462960FB6F894DEBF0FBEB6
:1091C000CDBFDF91CF911F910F91FF90EF90DF9076
:1091D000CF90BF90AF909F908F907F906F905F9057
:1091E0004F903F902F90089580910B01809588704B
:1091F000809309010C946D4080910B0188708093DD
:10920000090164C839893093910480E28816910479
:10921000A104B10428F430E2832E912CA12CB12CAE
:1092200030E2831A9108A108B108811488E09806F9
:10923000A104B10420F1E4E09E9EC0011124835CEE
:109240009E4EFC01329625913491F82DEE27F39F26
:109250007001F29FE10CFE1E0694EE1EFE1E11240C
:10926000FC01C590D490860120E030E0480159010E
:109270008E189F08A108B1087501640122C09501EC
:1092800084013695279517950795F801EC7FCF0156
:10929000835C924FFC01C590D490FC0132962591DD
:1092A0003491E82DE770E29FC001E39F900D1124F7
:1092B00023E0969587952A95E1F7C81AD90AE12CFB
:1092C000F12C4C0D5D1D6E1D7F1D4093920450933B
:1092D000930460939404709395049091900480910A
:1092E0008F04992309F473C0882309F40BCDA85B7C
:1092F000BF4F8D919C91A0E0B0E040910D02509144
:109300000E0260910F027091100284179507A60754
:10931000B70709F05FC0F6CCB695A79597958795E6
:10932000D988DD0CD98A2C5F3F4F45E129353407B8
:1093300009F04BCC59895093910480329105A105D5
:10934000B10520F480E290E0A0E0B0E08097A109B0
:10935000B109811558E09507A105B10508F443C08E
:1093600074E0979F90011124235C3E4EF9013296E0
:1093700045915491EE27859FB001849F610D7E1F1A
:1093800006946E1F7E1F1124F901C590D490E12C24
:10939000F12CC61AD70AE108F10880918604909151
:1093A0008704A0918804B09189048C0D9D1DAE1D89
:1093B000BF1D8093860490938704A0938804B09384
:1093C000890480919004811130C080918F0488239A
:1093D00009F498CC1092110210921202109213020A
:1093E000109214028FCCAC01BD017695679557950C
:1093F0004795FA01EC7F9F01235C324FF901C5903C
:10940000D490F9013296459154918770849F9001D0
:10941000859F300D1124F3E036952795FA95E1F7F5
:10942000C21AD30AE12CF12CB8CF8989480E511CFD
:10943000611C711C809118079091190748145904F8
:109440006A047B04D8F420918F04222309F45ACCB7
:10945000FC01E85BFF4F20813181A90160E070E0F1
:1094600000910D0210910E0220910F023091100216
:10947000401751076207730709F444CC1092110298
:10948000109212021092130210921402FC01E85B77
:10949000FF4F80819181A0E0B0E080930D02909316
:1094A0000E02A0930F02B09310022CCCD701C6017C
:1094B000B695A79597958795FC01EC7FCF01835CC6
:1094C000924FFC0125913491FC01329645915491C3
:1094D0006C2D6770649FC001659F900D112463E03F
:1094E000969587956A95E1F7281B390BC901A0E08D
:1094F000B0E0F8CBD501C401B695A79597958795AF
:10950000FC01EC7FCF01835C924FFC01C590D490AD
:10951000FC01329625913491482D4770429FC0013D
:10952000439F900D1124A3E096958795AA95E1F7A6
:10953000C81AD90AE12CF12CD4CD80EDC82E87E0D1
:10954000D82EE12CF12CE5CBCF92DF92EF92FF9257
:10955000CF93DF936B017C01EA0121E338E040EA1D
:1095600050EC0E94D9EC87FD23C022E430E04CE5AA
:1095700053E4C701B6010E9467E61816CCF0C88014
:10958000D980EA80FB802FE632E143E85AEBC7013D
:10959000B6010E94D9EC87FD0BC0C1E022E430E0A7
:1095A0004CE553E4C701B6010E9467E618160CF4B7
:1095B000C0E08C2FDF91CF91FF90EF90DF90CF90A4
:1095C00008950F931F93CF93DF93FC01A685B78572
:1095D0008D0100581F4FE8018881998101968F778E
:1095E0009927AD014E575F4FEA012881398128172D
:1095F0003907D1F3E80128813981A20FB31F6C9399
:10960000A685B785A058BF4F11969C938E93A689C7
:10961000B7892C9181E090E0078C02C0880F991FD8
:109620000A94E2F7822B8C9381E081A30488F58968
:10963000E02D80818064808381E090E0DF91CF9194
:109640001F910F910895FC0181A1882329F0A4891D
:10965000B5898C9186FFFBCF11A20895FC01A485EA
:10966000B585FD01E058FF4F208131813296808120
:1096700091812817390779F080819181A80FB91F4E
:109680008C91208131812F5F3F4F2F77332731839A
:10969000208390E008958FEF9FEF0895DC011C96E2
:1096A000ED91FC911D97DF01A058BF4F2D913C918A
:1096B000119712968D919C9111972817390739F0BF
:1096C0008D919C91E80FF91F808190E008958FEFB4
:1096D0009FEF0895FC0124853585F901E058FF4F7F
:1096E0008081918132962081318180589F4F821BE9
:1096F000930B60E870E00C949CED0895089580E071
:1097000090E00895CF92DF92EF92FF92C0903002E6
:10971000D0903102E0903202F0903302FC0180815F
:109720009181A281B3818093300290933102A09302
:109730003202B09333020E9486CAC0923002D092A5
:109740003102E0923202F0923302FF90EF90DF900C
:10975000CF9008958091961890919718981759F086
:10976000E92FF0E0EA5EF74E80819F5F9F7790934C
:10977000971890E008958FEF9FEF08951F920F9232
:109780000FB60F9211240BB60F922F938F939F93C6
:10979000EF93FF9320919718E091961881E08E0F38
:1097A0008F779091C600281729F0F0E0EA5EF74E17
:1097B0009083E82FE0939618FF91EF919F918F91FE
:1097C0002F910F900BBE0F900FBE0F901F9018950A
:1097D0008091210490912204009731F04AE050E0FA
:1097E00060E070E00C94BBE360E070E0CB010895B2
:1097F000EFDF97FD0AC0ECDF6F3F71058105910532
:1098000009F02CF4E5DF862F089580E008958FEFAE
:1098100008958091210490912204892B31F0E8DF92
:1098200091E0811103C090E001C091E0892F08957B
:109830000F931F93CF93809121049091220400975E
:1098400011F1FC018F01C1912C2F2F7DA9F0C5349E
:1098500011F0C536B9F7F801108260E070E0809130
:109860002104909122040E9468E2F801C083562FDF
:10987000472F382F292F0BC060E070E0CF911F9148
:109880000F910C9468E250E040E030E020E0652F5A
:10989000742F832F922FCF911F910F910895815490
:1098A0008A3108F042C0E82FF0E040910D18509145
:1098B0000E1860910F187091101804C07695679576
:1098C000579547958A95D2F7842F817040FF2FC016
:1098D000ED50F84E9081992309F1E0917210F091CA
:1098E0007310E90FF11D908120ED290F2A3098F0B7
:1098F0009E3211F491810CC09D3211F09B3271F4B3
:10990000918120ED290F2A3030F09E3239F4928176
:1099100090539A3018F42E2F9F2F02C020E090E031
:109920002093210490932204089580E008950895DF
:10993000B6DF882341F081E0209121043091220498
:10994000232B09F480E0089580E1E2E3F4E0AEEA3D
:10995000B0E101900D928A95E1F708952F923F9220
:109960004F925F926F927F928F929F92AF92BF922F
:10997000CF92DF92EF92FF920F931F93CF93DF93DB
:1099800000D01F921F92CDB7DEB77C018B016A0118
:1099900019018090320490903304A0903404B09068
:1099A0003504A5019401FC0160817181828193815C
:1099B0000E9467E6F1E0FD83811112C02091360418
:1099C000309137044091380450913904F801608196
:1099D0007181828193810E9467E6811101C01D829D
:1099E000F601408051806280738020911502309191
:1099F00016024091170250911802C301B2010E9451
:109A000067E6882309F453C040921502509216026B
:109A1000609217027092180220E030E040E450E4B7
:109A20006091FB067091FC068091FD069091FE0608
:109A30000E948FEB69837A838B839C838092AE1024
:109A40009092AF10A092B010B092B11080913604F5
:109A500090913704A0913804B09139048093B210EA
:109A60009093B310A093B410B093B510F601808119
:109A70009181A281B3818093B6109093B710A09387
:109A8000B810B093B91080913E0490913F04A0911A
:109A90004004B09141048093BA109093BB10A093FE
:109AA000BC10B093BD10CE0101962CDE4DDFFD81C0
:109AB000FF2309F16090F7067090F8068090F90690
:109AC0009090FA06A090F306B090F406C090F506C8
:109AD000D090F6069501A601B301C4010E94D9EC0D
:109AE000181614F05301640120E030E040E251E424
:109AF000B501C6010CC020E030E040EC5FE36091AE
:109B0000FF067091000780910107909102070E9463
:109B10008FEB69837A838B839C832091200422239B
:109B200049F0AB01BC018DE595E10E9461C58AE079
:109B30000E94EE93F70180819181A281B38180938D
:109B4000AE109093AF10A093B010B093B110F80185
:109B500080819181A281B3818093B2109093B310E0
:109B6000A093B410B093B510F101208131814281EE
:109B700053816091BA107091BB108091BC1090918C
:109B8000BD100E94B3EA6093BA107093BB1080932B
:109B9000BC109093BD10CE010196B4DDD5DE0F90C0
:109BA0000F900F900F900F90DF91CF911F910F9119
:109BB000FF90EF90DF90CF90BF90AF909F908F90ED
:109BC0007F906F905F904F903F902F90089580E12D
:109BD000EEEAF0E1A2E3B4E001900D928A95E1F79C
:109BE00008959C0197FD0EC08436910584F064E6CB
:109BF00070E00E949CEDCB016AE070E00E949CED59
:109C0000805D06C03195219531098DE201C080E269
:109C100080932D042A30310564F0EAE0F0E0C901B8
:109C2000BF010E949CEDCB01BF010E949CED805DB5
:109C300001C080E280932E04C9016AE070E00E94B6
:109C40009CED805D80932F048DE294E008958E3624
:109C500091051CF02EE680E002C0282F892F20936A
:109C60004404809345040C94B7762F923F924F9210
:109C70005F926F927F928F929F92AF92BF92CF929C
:109C8000DF92EF92FF920F931F93CF93DF93CDB7A5
:109C9000DEB7C455D1090FB6F894DEBF0FBECDBFF5
:109CA000ECE1F8E184918F010F5F1F4F882321F0D1
:109CB0000E94EE93F801F6CF0E9493B481110C94A8
:109CC000175880E090E0A0E8BFE38093A61090933F
:109CD000A710A093A810B093A91080E090E0A0EC8A
:109CE000B0E48093AA109093AB10A093AC10B09303
:109CF000AD108DEC9CECACE4BEE38093A21090938D
:109D0000A310A093A410B093A51080E090E0A8EC5D
:109D1000B1E48093240590932505A0932605B09384
:109D200027058CE390E0909323058093220588EC2F
:109D300090E0909321058093200510921F058FE4F9
:109D4000F7DD882311F074DD04C060E070E080E18D
:109D500090E46BAF7CAF8DAF9EAF83E4E9DD8823E9
:109D600011F057DD02C083E49ADD61968FAF6197F1
:109D70008BE4DEDD882311F04CDD02C08BE48FDD47
:109D800060968FAF609782E4D3DD8823E9F050DDE1
:109D90000E94F7EB7093230560932205611571050E
:109DA00099F0685271096536710570F0E7EEF7E1D8
:109DB00084918F010F5F1F4F882311F40C94175863
:109DC0000E94EE93F801F4CF8CE4B2DD882351F1C8
:109DD0002FDD6B017C016093A2107093A310809320
:109DE000A4109093A51020E030E0A9010E94D9ECC6
:109DF00087FD0AC020E030E040E050E4C701B60132
:109E00000E9467E6181674F4EFEBF7E184918F0176
:109E10000F5F1F4F882311F40C9417580E94EE9384
:109E2000F801F4CF81E53BDD882309F440C080913F
:109E3000210490912204892B19F4E4E9F7E12BC065
:109E4000F7DC6B017C016093AA107093AB108093D8
:109E5000AC109093AD102DEC3CEC4CE45DE30E9413
:109E6000D9EC87FD0AC020E030E040E751E4C701AB
:109E7000B6010E9467E61816D4F4E3E6F7E1849190
:109E80008F010F5F1F4F882311F40C9417580E9405
:109E9000EE93F801F4CF84918F010F5F1F4F882359
:109EA00011F40C9417580E94EE93F801F4CF83E557
:109EB0003FDD882319F1BCDC4B015C012DEC3CEC4F
:109EC0004CEC5DE30E94D9EC87FD0AC020E030E055
:109ED00040E85FE3C501B4010E9467E61816ACF4E0
:109EE000ECE3F7E184918F010F5F1F4F882311F49A
:109EF0000C9417580E94EE93F801F4CF5DEC852E78
:109F00005CEC952EA92C5EE3B52E80E5C8DC882399
:109F100009F443C08091210490912204892B71F4AB
:109F2000E4E0F7E184918F010F5F1F4F882311F464
:109F30000C9417580E94EE93F801F4CF80911F05FE
:109F40008F5F80931F0574DC6B017C016093240597
:109F500070932505809326059093270520E030E037
:109F6000A9010E94D9EC87FD0AC020E030E048EC4E
:109F700051E4C701B6010E9467E6181674F4ECEDCF
:109F8000F6E184918F010F5F1F4F882311F40C9429
:109F900017580E94EE93F801F4CF86E4C9DC8823B9
:109FA00019F146DC6B017C0120E030E040E85FE322
:109FB0000E94D9EC87FD0AC020E030E040E850E480
:109FC000C701B6010E9467E61816A4F4E3EBF6E1B8
:109FD00084918F010F5F1F4F882311F40C94175841
:109FE0000E94EE93F801F4CFC12CD12C40EEE42E68
:109FF0004FE3F42EA7019601C701B6010E94CCE6FB
:10A000009B01AC0160E070E084E490E40E948FEB7F
:10A010002091A6103091A7104091A8105091A9103E
:10A020000E94CCE62B013C01A5019401C501B401BD
:10A030000E94CCE6A70196010E94CCE62CEE31E509
:10A0400048EB5DE30E948FEB9B01AC01C301B201C1
:10A050000E94CCE66093A6107093A7108093A8107E
:10A060009093A91088E464DC8823C9F0E1DB0E94A6
:10A07000F7EB7093210560932005655A71096437E9
:10A08000710568F0E5E8F6E184918F010F5F1F4FDD
:10A09000882309F4CCC70E94EE93F801F5CF85E53B
:10A0A000FEDB8823E9F00E94FF58611571058105E8
:10A0B000910511F00E945FE28091210490912204A9
:10A0C000892B11F0B5DB04C060E070E088E492E415
:10A0D00060931B0570931C0580931D0590931E05CE
:10A0E00082E5DDDB81110DC0E1E5F6E184918F01B0
:10A0F0000F5F1F4F882309F49AC70E94EE93F8015F
:10A10000F5CF8091210490912204892BA9F060DB86
:10A110002F967FAF6EAF2F97161617069CF0EDE1C6
:10A12000F6E184918F010F5F1F4F882309F47FC7E9
:10A130000E94EE93F801F5CF8AE190E02F969FAF51
:10A140008EAF2F9788E5F4DB882361F071DB2091D7
:10A1500014043091150440911604509117040E9484
:10A16000B2EA08C0609132047091330480913404E3
:10A170009091350460931705709318058093190525
:10A1800090931A0589E5D4DB882361F051DB209197
:10A1900018043091190440911A0450911B040E9434
:10A1A000B2EA08C060913604709137048091380497
:10A1B00090913904609313057093140580931505ED
:10A1C00090931605609117057091180580911905F7
:10A1D00090911A0543E155E0B7D981110DC0E3EF25
:10A1E000F5E184918F010F5F1F4F882309F41FC78A
:10A1F0000E94EE93F801F5CF84E451DB91E08927CA
:10A200000E9456AC20E030E040EA50E460913A040D
:10A2100070913B0480913C0490913D040E9467E65C
:10A2200087FF14C0198A1A8A1B8A1C8A80E090E072
:10A23000A0EAB0E489839A83AB83BC83BE016F5EDE
:10A240007F4FCE0101960E9475B4C1DCD8D76B0157
:10A250007C01A8E8CA0EA3E1DA1EE11CF11C809182
:10A26000220590912305F3DC60912205709123056E
:10A27000072E000C880B990B0E946DE69B01AC0128
:10A28000609146047091470480914804909149047C
:10A290000E94B2EA4B015C0120E030E0A9010E947B
:10A2A000D9EC87FF04C0B7FAB094B7F8B09420E0B7
:10A2B00030E040E450E4C501B4010E94D9EC181626
:10A2C000F4F49DD7DC01CB018C199D09AE09BF09BF
:10A2D000B7FD0EC094D76B017C01B8E8CB0EB3E19B
:10A2E000DB1EE11CF11C0E94FD758AE00E94EE93CA
:10A2F0000E942CA18091961880939718B5CF8091D9
:10A300002005909121050E94F459609120057091DB
:10A310002105072E000C880B990B0E946DE69B010E
:10A32000AC0160914C0470914D0480914E04909169
:10A330004F040E94B2EA4B015C0120E030E0A90129
:10A340000E94D9EC87FF04C0B7FAB094B7F8B09474
:10A3500020E030E040E450E4C501B4010E94D9ECB3
:10A360001816F4F44CD7DC01CB018C199D09AE0909
:10A37000BF09B7FD0EC043D76B017C01E8E8CE0EE4
:10A38000E3E1DE1EE11CF11C0E94FD758AE00E94E3
:10A39000EE930E942CA18091961880939718B5CFC8
:10A3A00010923E0410923F04109240041092410417
:10A3B0000E9444B380911F05882399F1C5DA20914A
:10A3C000240530912505409126055091270560917F
:10A3D000BA107091BB108091BC109091BD100E947A
:10A3E000B3EA6093BA107093BB108093BC10909343
:10A3F000BD1020E030E040E751E46091FF0670912D
:10A40000000780910107909102070E948FEB6983FA
:10A410007A838B839C83CE01019674D995DA0E944E
:10A4200051B180E2E3EFF4E0DF01282F1D922A957D
:10A43000E9F7E3EDF4E0DF01282F1D922A95E9F713
:10A44000E3EBF4E0DF011D928A95E9F77DDA809174
:10A45000A2109091A310A091A410B091A510809388
:10A46000B6109093B710A093B810B093B91019829A
:10A470001A821B821C829E012F5F3F4F46EB50E1E8
:10A4800062EB70E18EEA90E169DA9E01255C3F4F54
:10A4900046EB50E162EB70E18EEA90E15FDA6196A3
:10A4A000BFAD6197BB2329F066E374E082E394E0DB
:10A4B00004C063E175E087E195E00E94B7D8298F79
:10A4C0003A8F4B8F5C8F6D8F7E8F3FAF2D962FAF66
:10A4D0002D972D96EFAD2D97E7FD81C4FFADF7FDCC
:10A4E0007EC424E0E202F0011124E350F64F4080E4
:10A4F0005180628073803FAD84E03802F001112406
:10A50000E751F64FD080C180328023808D2D9C2D65
:10A51000A32DB22D8FAB98AFA9AFBAAFAE01495CF6
:10A520005F4FB201C30110D8882309F45CC420E056
:10A5300030E040EA50E4B201C3010E94B3EAF62ED3
:10A54000072F182FE92E862F902FA12FBE2D8BAB12
:10A550009CABADABBEAB8D2D9C2DA32DB22D8FA78B
:10A5600098ABA9ABBAAB2D969FAD2D97911152C068
:10A57000AFADA11105C05F2D402F312F2E2D04C08E
:10A58000542D452D362D272D852F942FA32FB22FF7
:10A590008BAB9CABADABBEABBFADB43034F4F42CE5
:10A5A000052D162DE72CBB2369F020E030E040EAB2
:10A5B00050E46D2D7C2D832D922D0E94B2EA362F12
:10A5C000272F03C09601832D922D432F522FBC01BC
:10A5D0004FA758AB69AB7AABEFADE4300CF0A7C036
:10A5E00020E030E040EA50E46D2D7C2D832D922D4B
:10A5F0000E94B3EA21966FAF219723967FAF2397EE
:10A6000025968FAF259727969FAF2797FFADF1111E
:10A6100085C099C02D962FAD2D9724300CF453C0D2
:10A620003FAD34305CF020E030E040EA50E4B2016D
:10A63000C3010E94B2EA362F272F03C0342D252DE7
:10A64000C301432F522FBC014BAB5CAB6DAB7EAB58
:10A650008FAD8111E3C420E030E040EA50E4B20164
:10A66000C3010E94B2EAF62E072F182FE92E20E030
:10A6700030E040EA50E46D2D7C2D832D922D0E9418
:10A68000B3EA6FA778AB89AB9AAB9FAD992309F476
:10A690004EC020E030E040EA50E46D2D7C2D832D4B
:10A6A000922D0E94B2EA21966FAF219723967FAF39
:10A6B000239725968FAF259727969FAF2797AFAD06
:10A6C000A43064F140C0BFADB1110DC020E030E056
:10A6D00040EA50E4B201C3010E94B2EAF62E072F0D
:10A6E000182FE92E0FC0EFADE430B4F120E030E0D8
:10A6F00040EA50E4B201C3010E94B2EA6BAB7CAB0A
:10A700008DAB9EAB2196DFAE21972396CFAE2397DC
:10A7100025963FAE259727962FAE279732ED832EAD
:10A7200033E5932E3BE7A32E31E4B32E29C02196C7
:10A73000DFAE21972396CFAE239725963FAE259780
:10A7400027962FAE279722ED822E23E5922E2BEF10
:10A75000A22E20E4B22E14C02196DFAE21972396BC
:10A76000CFAE239725963FAE259727962FAE2797F6
:10A7700092ED892E93E5992E9BEFA92E91E4B92EA7
:10A780008BA99CA9ADA9BEA92C968CAF9DAFAEAFED
:10A79000BFAF2C979C01AD01B201C3010E94B2EA88
:10A7A000698B7A8B8B8B9C8B4FA458A869A87AA84D
:10A7B000A30192016D2D7C2D832D922D0E94B2EA72
:10A7C0006D8B7E8B8F8B988F2C962CAD3DAD4EADC7
:10A7D0005FAD2C9760913204709133048091340402
:10A7E000909135040E94B2EA2C966CAF7DAF8EAF8B
:10A7F0009FAF2C97A30192016091360470913704AA
:10A8000080913804909139040E94B2EA2B013C01F6
:10A810008F2D902FA12FBE2D89839A83AB83BC836C
:10A8200021968FAD219723969FAD23972596AFADA7
:10A8300025972796BFAD27978D839E83AF83B887D3
:10A840008091A2109091A310A091A410B091A51096
:10A8500089879A87AB87BC872DEC3CEC4CEC5CE39A
:10A86000C501B4010E94CCE62091A6103091A7103A
:10A870004091A8105091A9100E94CCE620913E046E
:10A8800030913F0440914004509141040E94B3EA4A
:10A890006D877E878F87988B2C962CAD3DAD4EAD06
:10A8A0005FAD2C97CA01B9010E94CCE66B017C0117
:10A8B000A3019201C301B2010E94CCE69B01AC014D
:10A8C000C701B6010E94B3EA20E030E040E050E466
:10A8D0000E94D9EC18160CF046C00E9451B11BA280
:10A8E0001CA21DA21EA220E030E040E05FE36091C8
:10A8F0003A0470913B0480913C0490913D040E9485
:10A90000B3EA6F8F78A389A39AA39E012D5D3F4F71
:10A91000AE01415E5F4F66E374E082E394E01ED8CF
:10A920001BA21CA21DA21EA220E030E040E05FE3BB
:10A930006091A2107091A3108091A4109091A51025
:10A940000E94B3EA6F8F78A389A39AA39E012D5D1D
:10A950003F4FAE01415E5F4FBE01615D7F4FCE0153
:10A96000C3960E94AE4C1F8E18A219A21AA29E0175
:10A97000215E3F4F42EA50E1BE01615D7F4FCE0153
:10A98000C3960E94AE4C0E947DB140903002509020
:10A9900031026090320270903302E090F706F0903E
:10A9A000F8060091F9061091FA06A090F306B0900F
:10A9B000F406C090F506D090F6069501A601B70101
:10A9C000C8010E94D9EC181614F47501860120E024
:10A9D00030E040E251E4B701C8010E948FEB609380
:10A9E000300270933102809332029093330240E040
:10A9F000BE016F5E7F4FCE0101960E94F8A4409287
:10AA000030025092310260923202709233020E9400
:10AA1000A44CADEFB9E02496BFAFAEAF2497229619
:10AA20001FAE1EAE229701E010E021960FAC2197D9
:10AA300002C0000F111F0A94E2F72296EEADFFAD9F
:10AA4000229731962296FFAFEEAF229721E030E0B9
:10AA500021960FAC219702C0220F331F0A94E2F710
:10AA600063963FAF2EAF639783EB282E84E0382E9A
:10AA700083EF94E02A969FAF8EAF2A97A3EDB4E0C0
:10AA80002896BFAFAEAF2897E9EEF9E02696FFAF64
:10AA9000EEAF26972A962EAD3FAD2A9765963FAF2B
:10AAA0002EAF6597D9018D919C919C012023312374
:10AAB000232B09F4ADC06396EEADFFAD63978E23F3
:10AAC0009F23892B09F4A4C02896AEADBFAD28976B
:10AAD0008D919C9180239123892B09F099C020E0CE
:10AAE00030E040E050E42496AEADBFAD24976D91C8
:10AAF0007D918D919C910E94B3EA6B017C0120E0D5
:10AB000030E040E050E42496EEADFFAD2497648140
:10AB10007581868197810E94B2EA4B015C0120E039
:10AB200030E040E850ECC701B6010E9467E687FDBF
:10AB300070C120E030E04BE553E4C701B6010E944C
:10AB4000D9EC181634F4C12CD12CBBE5EB2EB3E4B0
:10AB5000FB2ECBA6DCA6EDA6FEA62696AEADBFAD1F
:10AB600026974D905D906D907C9020E030E040E81D
:10AB70005FE3C301B2010E9467E687FD51C120E097
:10AB800030E04BE553E4C301B2010E94D9EC181642
:10AB900034F4412C512CFBE56F2EF3E47F2E4F8EC5
:10ABA00058A269A27AA24FA258A669A67AA620E066
:10ABB00030E040E850ECC501B4010E9467E687FD33
:10ABC00036C120E030E04BE553E4C501B4010E94FA
:10ABD000D9EC181634F4812C912C7BE5A72E73E464
:10ABE000B72E8BA29CA2ADA2BEA2AE01495D5F4F63
:10ABF000C701B6010E94A44A811120C12896EEAD7A
:10AC0000FFAD289780819181802B912B9183808348
:10AC10002A962EAD3FAD2A972E5F3F4F2A963FAF23
:10AC20002EAF2A976596AEADBFAD65978D919C917D
:10AC300080239123892B09F4A6C0F9018081918199
:10AC400080239123892B09F49EC0F1018081918199
:10AC500080239123892B09F096C020E030E040E06A
:10AC600050E42696AEADBFAD26976D917D918D9146
:10AC70009C910E94B3EA2B013C0120E030E040E0CF
:10AC800050E42696EEADFFAD2697648175818681EE
:10AC900097810E94B2EA4B015C012496AEADBFAD34
:10ACA0002497CD90DD90ED90FC9020E030E040E8DE
:10ACB00050ECC701B6010E9467E687FDFFC020E0A7
:10ACC00030E04BE553E4C701B6010E94D9EC1816F9
:10ACD00034F4C12CD12C5BE5E52E53E4F52ECBA248
:10ACE000DCA2EDA2FEA2CBA6DCA6EDA6FEA620E08D
:10ACF00030E040E85FE3C301B2010E9467E687FDF0
:10AD0000E4C020E030E04BE553E4C301B2010E940F
:10AD1000D9EC181634F4412C512C3BE5632E33E466
:10AD2000732E4FA258A669A67AA620E030E040E82C
:10AD30005FE3C501B4010E9467E687FDCDC020E056
:10AD400030E04BE553E4C501B4010E94D9EC18167C
:10AD500034F4812C912C9BE5A92E93E4B92E8F8E8F
:10AD600098A2A9A2BAA2AE01495D5F4FC701B60180
:10AD70000E94A44A8111B7C0F10180819181802B8A
:10AD8000912B91838083F2E02F0E311C28962EADFB
:10AD90003FAD28972E5F3F4F28963FAF2EAF2897A5
:10ADA00026968EAD9FAD2697049626969FAF8EAFC2
:10ADB00026979DEB291694E0390609F06BCE249670
:10ADC000AEADBFAD249714962496BFAFAEAF249717
:10ADD0002296EEADFFAD2297359709F024CE8091F3
:10ADE0009618809397182F962EAD3FAD2F97215030
:10ADF00031092F963FAF2EAF2F97232B09F4B3C005
:10AE00002D963FAD2D9737FDAEC08FAD87FF47CB59
:10AE1000AAC0C12CD12CA0E8EA2EA0ECFA2E99CE23
:10AE2000412C512CE0E86E2EEFE37E2EB8CE812C23
:10AE3000912C60E8A62E60ECB62ED3CEAE01415E1A
:10AE40005F4FC501B4010E94A44A882309F4D6CEFD
:10AE500080912004882321F1B701A6018DEC95E1B2
:10AE60000E9461C54FA158A569A57AA587EC95E117
:10AE70000E9461C54BA15CA16DA17EA18DEB95E106
:10AE80000E9461C54F8D58A169A17AA187EB95E118
:10AE90000E9461C589E20E94EE938AE00E94EE93CF
:10AEA0009E01215E3F4FAE014D5D5F4FBE01695D6A
:10AEB0007F4FCE018B960E94ADB1A0CEC12CD12C7C
:10AEC00040E8E42E40ECF42E0ACF412C512C20E82F
:10AED000622E2FE3722E25CF812C912C80E8A82E94
:10AEE0008FE3B82E3CCFAE01415E5F4FC701B60184
:10AEF0000E94A44A882309F43FCF8091200488232C
:10AF000021F1B701A60183E995E10E9461C54FA136
:10AF100058A569A57AA58DE895E10E9461C54BA168
:10AF20005CA16DA17EA183E895E10E9461C54F8D72
:10AF300058A169A17AA18DE795E10E9461C589E2D6
:10AF40000E94EE938AE00E94EE939E01215E3F4FA5
:10AF5000AE014D5D5F4FBE01695D7F4FCE018B96A7
:10AF60000E94ADB109CF0E9451B180E090E0A0EA0B
:10AF7000B0E48093B6109093B710A093B810B0933C
:10AF8000B91019821A821B821C829E012F5F3F4FCB
:10AF900046EB50E162EB70E18EEA90E10E94AE4C2C
:10AFA0008091170590911805A0911905B0911A0587
:10AFB0008093AE109093AF10A093B010B093B110E7
:10AFC0008091130590911405A0911505B091160577
:10AFD0008093B2109093B310A093B410B093B510B7
:10AFE00019821A821B821C829E012F5F3F4F46EB03
:10AFF00050E162EB70E18EEA90E10E94AE4C609607
:10B00000FFAD6097F11113C01092450410924404F3
:10B010000E94B77680E090E0E7D109C02FADF42C14
:10B02000052D162DE72C24300CF033CB20CBCC5A39
:10B03000DF4F0FB6F894DEBF0FBECDBFDF91CF91CB
:10B040001F910F91FF90EF90DF90CF90BF90AF9046
:10B050009F908F907F906F905F904F903F902F9038
:10B0600008951F920F920FB60F9211240BB60F92F4
:10B070002F933F938F939F93EF93FF932091120F02
:10B080003091130F8091140F9091150F28173907E5
:10B0900031F4809131018F7D8093310114C0E091B2
:10B0A000140FF091150FEE56F14F20818091140F7F
:10B0B0009091150F01968F7799279093150F809394
:10B0C000140F20933601FF91EF919F918F913F9143
:10B0D0002F910F900BBE0F900FBE0F901F901895E1
:10B0E0001F920F920FB60F9211240BB60F922F934F
:10B0F0004F935F938F939F93EF93FF9380913001D2
:10B1000082FD1CC0209136018091960F9091970F7F
:10B110004091980F5091990F01968F779927481772
:10B12000590771F0E091960FF091970FEA5EF04F9A
:10B1300020839093970F8093960F02C080913601E1
:10B14000FF91EF919F918F915F914F912F910F9070
:10B150000BBE0F900FBE0F901F901895CF92DF92ED
:10B16000EF92FF920F931F93CF93DF936C017A01BD
:10B170008B01C0E0D0E0CE15DF0581F0D8016D91E4
:10B180008D01D601ED91FC910190F081E02DC60179
:10B190001995892B11F02196EECF7E01C701DF9121
:10B1A000CF911F910F91FF90EF90DF90CF90089576
:10B1B0000E94C3ED3FB7F8948091CF069091D006DE
:10B1C000A091D106B091D20626B5A89B05C02F3F0D
:10B1D00019F00196A11DB11D3FBFBA2FA92F982FBD
:10B1E0008827820F911DA11DB11DBC01CD0142E038
:10B1F000660F771F881F991F4A95D1F708952FB7BB
:10B20000F8946091CB067091CC068091CD06909118
:10B21000CE062FBF08951F920F920FB60F921124E2
:10B220002F933F938F939F93AF93BF938091CB06C0
:10B230009091CC06A091CD06B091CE063091CA0671
:10B2400023E0230F2D3720F40196A11DB11D05C069
:10B2500026E8230F0296A11DB11D2093CA068093F4
:10B26000CB069093CC06A093CD06B093CE068091EA
:10B27000CF069091D006A091D106B091D20601964A
:10B28000A11DB11D8093CF069093D006A093D10647
:10B29000B093D206BF91AF919F918F913F912F9123
:10B2A0000F900FBE0F901F9018951F920F920FB620
:10B2B0000F9211240BB60F922F933F934F935F93EE
:10B2C0006F937F938F939F93AF93BF93EF93FF936E
:10B2D00080912B0590912C05A0912D05B0912E0504
:10B2E000892B8A2B8B2B59F190912A05E091280507
:10B2F000F091290580818927808380912B05909189
:10B300002C05A0912D05B0912E05181619061A06C8
:10B310001B060CF056C080912B0590912C05A09136
:10B320002D05B0912E050197A109B10980932B0538
:10B3300090932C05A0932D05B0932E0542C08091CB
:10B340001902E9E4F8E1E4919FEF90931902E230E9
:10B35000C9F050F4EE2399F0E13081F590916F003F
:10B360009D7F90936F002AC0E43019F1E0F0E53042
:10B3700029F5909173009D7F909373001FC01092E8
:10B380006E001CC0909170009D7F9093700091E0C2
:10B390009093B0009091B100987F94609093B10029
:10B3A0001092B3000BC0909171009D7F909371003B
:10B3B00005C0909172009D7F9093720060E00E94A2
:10B3C00009B6FF91EF91BF91AF919F918F917F91BE
:10B3D0006F915F914F913F912F910F900BBE0F9006
:10B3E0000FBE0F901F90189590934B0480934A04C2
:10B3F00080E00C9403772F923F924F925F926F926E
:10B400007F928F929F92AF92BF92CF92DF92EF92F4
:10B41000FF920F931F93CF93DF93CDB7DEB7C8573B
:10B42000D1090FB6F894DEBF0FBECDBFE0914A0739
:10B43000F0914B07EF2B11F00C94BB622896DFAE16
:10B44000CEAE28976E2C79016A015B01FC01208148
:10B450003181428153816C962CAF3DAF4EAF5FAFCF
:10B460006C972091921030919310409194105091CC
:10B4700095106C966CAD7DAD8EAD9FAD6C970E94B6
:10B48000CCE60E94E4ECE0966CAF7DAF8EAF9FAF50
:10B49000E097D5018D919D910D90BC91A02DA09626
:10B4A0008CAF9DAFAEAFBFAFA097209196103091FB
:10B4B00097104091981050919910BC01CD010E94B5
:10B4C000CCE60E94E4ECE4966CAF7DAF8EAF9FAF0C
:10B4D000E497D6012D913D914D915C91A4962CAFAE
:10B4E0003DAF4EAF5FAFA49720919A1030919B1063
:10B4F00040919C1050919D10A4966CAD7DAD8EAD89
:10B500009FADA4970E94CCE60E94E4ECE8966CAF55
:10B510007DAF8EAF9FAFE897D7012D913D914D91B3
:10B520005C9122962CAF3DAF4EAF5FAF229720913A
:10B530009E1030919F104091A0105091A110229622
:10B540006CAD7DAD8EAD9FAD22970E94CCE60E9482
:10B55000E4EC60966CAF7DAF8EAF9FAF609780914B
:10B56000100783FF1CC060962CAD3DAD4EAD5FADA6
:10B5700060972093E5093093E6094093E7095093DB
:10B58000E80922968CAD9DADAEADBFAD22978093FC
:10B59000D5099093D609A093D709B093D809D801BB
:10B5A000BC91B9A7F801F181F9ABD8011296BC9111
:10B5B000BEABF801F381FAAF8091B3099091B40961
:10B5C000891B8F708F3019F40E942CA1F5CF009148
:10B5D000B309E9960FAFE9978091B309082F10E0FE
:10B5E0001CA30BA38091D9099091DA09A091DB09E2
:10B5F000B091DC09E0968CAC9DACAEACBFACE097F2
:10B60000881A990AAA0ABB0A8091DD099091DE097D
:10B61000A091DF09B091E009E4962CAC3DAC4EACB2
:10B620005FACE497281A390A4A0A5B0A8091E1095B
:10B630009091E209A091E309B091E409E8962CAD5C
:10B640003DAD4EAD5FADE897281B390B4A0B5B0B48
:10B650002DA33EA34FA358A78091E5099091E60939
:10B66000A091E709B091E80960960CAD1DAD2EAD33
:10B670003FAD6097081B190B2A0B3B0B0DA71EA7AC
:10B680002FA738AB012B022B032B09F4BCC08091F0
:10B690000F0781114BC060914C0470914D04809153
:10B6A0004E0490914F040E94F7EB209125023091B7
:10B6B0002602621773070CF039C060962CAD3DADC1
:10B6C0004EAD5FAD60972093E5093093E609409356
:10B6D000E7095093E80922968CAD9DADAEADBFADA4
:10B6E00022978093D5099093D609A093D709B09358
:10B6F000D809E6EEFDE184918F010F5F1F4F8111A4
:10B7000003C0EDEBF9E104C00E94EE93F801F3CF22
:10B7100084918F010F5F1F4F882321F00E94EE93C9
:10B72000F801F6CF1DA61EA61FA618AA94E0699ED2
:10B73000800111240F5D1D4F6DA57EA58FA598A9D1
:10B740000E946DE6D8012D913D914D915C910E9432
:10B75000CCE66B017C0120E030E0A9010E94D9EC2D
:10B7600087FF04C0F7FAF094F7F8F09460919E1008
:10B7700070919F108091A0109091A1100E94F7EB02
:10B780009B01AC01A8ECB0E00E9493EA0E946DE638
:10B79000A70196010E9467E687FF39C060960CAD4D
:10B7A0001DAD2EAD3FAD60970093E5091093E609FE
:10B7B0002093E7093093E80922962CAD3DAD4EADBC
:10B7C0005FAD22972093D5093093D6094093D709CE
:10B7D0005093D809E6EEFDE184918F010F5F1F4F72
:10B7E000811103C0EEE9F9E104C00E94EE93F80173
:10B7F000F3CF84918F010F5F1F4F882321F00E94A8
:10B80000EE93F801F6CF1DA61EA61FA618AAD50115
:10B81000C4018827B7FD83959927AA27BB27782ECF
:10B8200057FE03C0382F3260732E8DA19EA1AFA1A9
:10B83000B8A5B7FF03C0972D9460792E0DA51EA55E
:10B840002FA538A937FF03C0172D1860712E24E0EB
:10B85000629E800111240F5D1D4F6DA57EA58FA5F1
:10B8600098A90E946DE6D8012D913D914D915C9172
:10B870000E94CCE66B017C0120E030E0A9010E942F
:10B88000D9EC87FF04C0C701B601905802C0C701B8
:10B89000B60120E030E040E05FE30E94B3EA0E949E
:10B8A000FCEB6AAB7BAB8CAB9DAB88E60BA11CA120
:10B8B000809FF001819FF00D1124E159FE4E10820E
:10B8C000EA5BFF4F7082B501A401B7FE07C04427B1
:10B8D0005527BA01481959096A097B0988E60BA15D
:10B8E0001CA1809FF001819FF00D1124E159FE4EB3
:10B8F000458B568B678B708F2C962CAE3DAE4EAE23
:10B900005FAE2C9757FE0DC088279927DC0182195E
:10B910009309A409B5092C968CAF9DAFAEAFBFAF0C
:10B920002C9728E60BA11CA1209FF001219FF00D70
:10B930001124E159FE4E2C968CAD9DADAEADBFAD40
:10B940002C97818F928FA38FB48F0DA11EA12FA151
:10B9500038A537FF07C030952095109501951F4FEA
:10B960002F4F3F4FE8E67E2EABA1BCA17A9EF0019F
:10B970007B9EF00D1124E159FE4E058F168F278F07
:10B9800030A38AA99BA9ACA9BDA981A392A3A3A313
:10B99000B4A323964FAF2397752EF62FE72F2C963F
:10B9A0008CAD9DADAEADBFAD2C97481759076A075A
:10B9B0007B0778F429969FAD299723969FAF23970D
:10B9C0002A967FAC2A972B96FFAD2B972C96EFAD3E
:10B9D0002C9723968FAD2397972DAF2FBE2F8017CF
:10B9E0009107A207B30710F4D901C8010AA91BA93E
:10B9F0002CA93DA980179107A207B30710F4D9011C
:10BA0000C80128E60BA11CA1209FF001219FF00D89
:10BA10001124E159FE4E85A396A3A7A3B0A70697CC
:10BA2000A105B10508F4A0C5DF01AE59BF4F809153
:10BA30004204909143048D939C9361A6452B462B21
:10BA4000472B09F05F9888E60BA11CA1809FF001AD
:10BA5000819FF00D1124E159FE4E818D928DA38DB1
:10BA6000B48D892B8A2B8B2B11F08A98479888E606
:10BA70000BA11CA1809FF001819FF00D1124E159C1
:10BA8000FE4E858D968DA78DB0A1892B8A2B8B2B91
:10BA900031F08091080181708093060147982AA9AE
:10BAA0003BA94CA95DA9232B242B252B09F465C5A3
:10BAB00080911507882319F0815080931507611034
:10BAC00004C0129880E28093150760900B07709075
:10BAD0000C0700910D0710910E079301A80169A5AD
:10BAE00079A98EA99AAD0E9467E687FF04C069A66E
:10BAF00079AA0EAB1AAFC501B4010E946DE6209180
:10BB00005F113091601140916111509162110E945A
:10BB1000CCE626966CAF7DAF8EAF9FAF2697698B34
:10BB20007A8B8B8B9C8BC201B1010E946DE62091B8
:10BB300063113091641140916511509166110E941A
:10BB4000CCE62B013C016D8B7E8B8F8B988F6DA18A
:10BB50007EA18FA198A50E946DE62091671130917A
:10BB600068114091691150916A110E94CCE64B0115
:10BB70005C01698F7A8F8B8F9C8F20916B11309134
:10BB80006C1140916D1150916E11C701B6010E9468
:10BB9000CCE66B017C016D8F7E8F8F8F98A388E63A
:10BBA0000BA11CA1809FF001819FF00D1124E15990
:10BBB000FE4E258936894789508D2DA33EA34FA37C
:10BBC00058A7263031054105510508F4DFC42896F1
:10BBD000AEADBFAD2897CD90DD90ED90FC9020E00C
:10BBE00030E0A901C701B6010E9467E68111EDC4EA
:10BBF00026962CAD3DAD4EAD5FAD2697CA01B9017D
:10BC00000E94CCE66B017C01A3019201C301B20149
:10BC10000E94CCE69B01AC01C701B6010E94B3EAC9
:10BC20006B017C01A5019401C501B4010E94CCE621
:10BC30009B01AC01C701B6010E94B3EA0E941EED50
:10BC400028E60BA11CA1209FF001219FF00D1124DB
:10BC5000E159FE4E658776878787908B88E60BA132
:10BC60001CA1809FF001819FF00D1124E159FE4E2F
:10BC70004584568467847088A301920160E070E077
:10BC800080E89FE30E948FEB64966CAF7DAF8EAF30
:10BC90009FAF649729A539A94EA95AAD0E94CCE659
:10BCA0004B015C018091B3099091B109891B8F70A0
:10BCB00027968FAF2797A501940160E074E284E78F
:10BCC00099E40E948FEB0E94E4EC6B017C012796C3
:10BCD0008FAD27978250863008F486C4A501940161
:10BCE000C301B2010E94CCE69B01AC010E94CCE6EC
:10BCF00068966CAF7DAF8EAF9FAF689788E6ABA1BB
:10BD0000BCA18A9F80018B9F100D112401591E4EEA
:10BD100068962CAD3DAD4EAD5FAD6897D8011196DC
:10BD20002D933D934D935C93149795962D913D9152
:10BD30004D915C9198972EAB3FAB48AF59AFCA017C
:10BD4000B9010E946BE66AAF7BAF8CAF9DAF9B01E0
:10BD5000AC01C501B4010E94CCE60E9479EB0E94BF
:10BD6000FCEBA8966CAF7DAF8EAF9FAFA897F801A4
:10BD7000EE5AFF4F60837183828393838E010F5E3F
:10BD80001F4F2A961FAF0EAF2A9700511109249614
:10BD90001FAF0EAF249703EF16E0AC961FAF0EAFA8
:10BDA000AC978E010F5D1F4F1AA309A324960EAD09
:10BDB0001FAD2497AA961FAF0EAFAA97312C212C46
:10BDC00010E819A70FE309AB2A96AEADBFAD2A97CD
:10BDD0002D913D914D915D912A96BFAFAEAF2A97BF
:10BDE000C501B4010E94CCE66B017C01AA96EEADC0
:10BDF000FFADAA976193719381939193AA96FFAF38
:10BE0000EEAFAA9720E030E0A9010E94D9EC87FFAD
:10BE100004C0F7FAF094F7F8F094AC96AEADBFAD6D
:10BE2000AC974D905D906D907D90AC96BFAFAEAFEE
:10BE3000AC97A7019601C301B2010E9467E687FD96
:10BE40000DC409A11AA12A962EAD3FAD2A9702175B
:10BE5000130709F0B9CF20E030E040E85FE3632D3D
:10BE6000722D89A599A90E9467E687FF58C07E01B7
:10BE700031E1E30EF11C24960EAD1FAD2497232D66
:10BE8000322D49A559A9D8016D917D918D919C9133
:10BE90000E94CCE6F80161937193819391938F0195
:10BEA000EE16FF0661F728E60BA11CA1209FC0013A
:10BEB000219F900D11249C0121593E4E7901890149
:10BEC0000E5A1F4FA8966CAD7DAD8EAD9FADA89755
:10BED0000E946BE6232D322D49A559A90E94CCE67C
:10BEE0000E94FCEBD8016D937D938D939C931397E7
:10BEF000232D322D49A559A9632D722D89A599A904
:10BF00000E94CCE668962CAD3DAD4EAD5FAD689716
:10BF10000E94CCE6F70161837283838394832AAD08
:10BF20003BAD4CAD5DAD64966CAD7DAD8EAD9FAD62
:10BF300064970E94CCE669A77AA78BA79CA70DA15E
:10BF40001EA12FA138A5012B022B032B09F09EC3A4
:10BF500088E62BA13CA1829F8001839F100D1124B4
:10BF600001591E4EF801818D928DA38DB48D892BC0
:10BF70008A2B8B2B09F08AC3858D968DA78DB0A156
:10BF8000892B8A2B8B2B09F081C32091EF063091EE
:10BF9000F0064091F1065091F20669A57AA58BA5AD
:10BFA0009CA50E94CCE60E9479EB0E94FCEB2B0141
:10BFB0003C01F801E95BFF4F108288E62BA13CA110
:10BFC000829F8001839F100D112401591E4EF8019C
:10BFD000E25AFF4F4082518262827382C301B201F2
:10BFE0000E946BE629A53AA54BA55CA50E948FEBA4
:10BFF0006AAF7BAF8CAF9DAFD80151966D937D93A7
:10C000008D939C935497F801E95BFF4F80818823BF
:10C0100081F17801B8E4EB0EF11C37962091E3062C
:10C020003091E4064091E5065091E6066081718109
:10C03000828193810E94CCE62AAD3BAD4CAD5DADD3
:10C040000E94CCE620919E1030919F104091A0104C
:10C050005091A1100E94CCE69B01AC0160E074E21B
:10C0600084EF99E40E948FEB0E94FCEBF70171834F
:10C07000608388E60BA11CA1809FF001819FF00DD9
:10C080001124E159FE4E21813281438154812C9645
:10C090002CAF3DAF4EAF5FAF2C97CA01B9010E94E4
:10C0A0001EED362E272E8C0143ED56E062965FAFD3
:10C0B0004EAF62973E0151E1650E711C83ED96E033
:10C0C0009FAB8EAB24964EAC5FAC24973DA62DA2C1
:10C0D00009A719AB1AAAD201CD90DD90ED90FD9081
:10C0E0002D0120E030E0A901C701B6010E94D9EC82
:10C0F00087FF04C0F7FAF094F7F8F094EEA9FFA9CF
:10C1000081909190A190B190FFABEEABA701960109
:10C11000C501B4010E9467E687FDD8C564147504A3
:10C12000D1F627965FAD2797552309F448C6C090EE
:10C13000B509D090B609E090B709F090B8092DEB99
:10C1400037E346E855E3C701B6010E9467E687FD7D
:10C1500036C6C701B6010E941EED6B017C019B0132
:10C16000AC01632D722DC8010E9467E687FD03C0F4
:10C170003C2C2D2C87019601A701632D722DC8013F
:10C180000E948FEB68966CAF7DAF8EAF9FAF6897C4
:10C1900089EB99E028969FAF8EAF289720E030E09A
:10C1A00040E85FE32AAB3BAB4CAB5DAB1EAA2896E5
:10C1B000AEADBFAD28972D913D914D915D912896E3
:10C1C000BFAFAEAF289768966CAD7DAD8EAD9FAD1D
:10C1D00068970E94CCE64B015C012496EEADFFAD62
:10C1E0002497C190D190E190F1902496FFAFEEAFEB
:10C1F0002497FEA9FF2391F02AA93BA94CA95DA988
:10C200000E94CCE64B015C012AA93BA94CA95DA97F
:10C21000C701B6010E94CCE66B017C01A701960123
:10C22000C501B4010E94D9EC20E030E0A901181644
:10C230000CF092C5C701B6010E94D9EC18160CF497
:10C2400086C520E030E0A901C501B4010E9467E67F
:10C2500087FD7DC52601370177FA709477F87094D1
:10C26000A3019201C501B4010E94D9EC181614F47F
:10C27000240135016296AEADBFAD6297CD90DD90E1
:10C28000ED90FD906296BFAFAEAF6297A3019201B1
:10C29000C701B6010E9467E687FF15C0A30192019E
:10C2A000C701B6010E948FEB9B01AC016AA97BA973
:10C2B0008CA99DA90E94CCE66AAB7BAB8CAB9DABF5
:10C2C000BEA9BF5FBEABE9ECF9E028962EAD3FAD4D
:10C2D0002897E217F30709F06ACF3EA9332361F0EC
:10C2E0002AA93BA94CA95DA9632D722DC8010E9402
:10C2F000CCE6362E272E8C0124EA30E74DE75FE3AB
:10C30000632D722DC8010E94CCE66B017C01209147
:10C3100011073091120740911307509114070E94A2
:10C3200067E687FD42C58DA59DA1A9A5B9A9809302
:10C33000110790931207A0931307B093140728E6F0
:10C340004BA15CA1249FC001259F900D1124DC010D
:10C35000A159BE4E7D01232D322DA801632D722DD2
:10C36000C8010E94CCE6F7016187728783879487B2
:10C370006AAD7BAD8CAD9DAD90589B01AC010E9428
:10C38000B3EAD7011D962D913D914D915C91509747
:10C390000E94CCE69B01AC016BE077ED83E29BE36E
:10C3A0000E94B2EA9B01AC018BE097EDA3E2BBE3F4
:10C3B000F70185839683A783B08710812C966CAD97
:10C3C0007DAD8EAD9FAD2C970E9467E618160CF4DC
:10C3D000FBC483E0182B88E62BA13CA1829FF001CF
:10C3E000839FF00D1124E159FE4E108380E1FE0180
:10C3F0003196A9EBB9E001900D928A95E1F72C9660
:10C400008CAD9DADAEADBFAD2C978093B50990932B
:10C41000B609A093B709B093B809E0960CAD1DAD6D
:10C420002EAD3FADE0970093D9091093DA09209320
:10C43000DB093093DC09E4962CAD3DAD4EAD5FAD2C
:10C44000E4972093DD093093DE094093DF09509390
:10C45000E009E8968CAD9DADAEADBFADE897809399
:10C46000E1099093E209A093E309B093E40960968F
:10C470000CAD1DAD2EAD3FAD60970093E509109357
:10C48000E6092093E7093093E8096C962CAD3DADA1
:10C490004EAD5FAD6C972093C9093093CA094093A4
:10C4A000CB095093CC09A0968CAD9DADAEADBFAD80
:10C4B000A0978093CD099093CE09A093CF09B09314
:10C4C000D009A4960CAD1DAD2EAD3FADA497009341
:10C4D000D1091093D2092093D3093093D40922961D
:10C4E0002CAD3DAD4EAD5FAD22972093D509309375
:10C4F000D6094093D7095093D8099091B3098091F8
:10C50000B409981303C084E68093B009E9968FAD0F
:10C51000E9978F5F8F708093B3098091B3099091F1
:10C52000B20981508F70891351C41091B4091BA3B3
:10C530000091B3090DA728E61BA10DA51013D1C4C6
:10C54000812C912CA12CB12C1DA219A619AA1EAECA
:10C55000212C312C00E010E02DA53BA12313CEC4EB
:10C560002114310409F07FC580916F0082608093AF
:10C570006F0081E0ECC680E0EAC66090070770902B
:10C5800008070091090710910A07A7CA818D928DAB
:10C59000A38DB48D0697A105B10508F018CB858D44
:10C5A000968DA78DB0A10697A105B10508F00FCB18
:10C5B00020E030E0A901C701B6010E94D9EC87FF55
:10C5C00004C0F7FAF094F7F8F09488E60BA11CA1E8
:10C5D000809FF001819FF00D1124E159FE4EC58628
:10C5E000D686E786F08A3ACB8091030790910407BC
:10C5F000A0910507B0910607C816D906EA06FB0602
:10C6000008F06CCB8C199D09AE09BF09BC01CD01A6
:10C61000660F771F881F991F27964FAD2797042F06
:10C6200010E020E030E0A90198010E9455EACA011B
:10C63000B9010E946BE60E94E4EC6C0D7D1D8E1D1D
:10C640009F1D0E946BE69B01AC0160E074E284E7F1
:10C6500099E40E948FEB4B015C0140CBA70196014E
:10C66000C301B2010E948FEB7B018C019B01AC01E5
:10C67000632D722D89A599A90E94D9EC18160CF08A
:10C68000E0CB3E2C2F2C09A719ABDBCB0AA91BA9A9
:10C690002CA93DA9012B022B032B49F02091EB067D
:10C6A0003091EC064091ED065091EE0608C02091C5
:10C6B000E7063091E8064091E9065091EA0669A53F
:10C6C0007AA58BA59CA50E94CCE60E9479EB0E94DE
:10C6D000FCEB2B013C012AA93BA94CA95DA9232B0A
:10C6E000242B252BC9F020E030E0A9016091E3065E
:10C6F0007091E4068091E5069091E6060E9467E657
:10C70000882351F081E00DA51EA52FA538A910168C
:10C710001106120613060CF080E098E62BA13CA14E
:10C72000929F8001939F100D112401591E4E1801F4
:10C7300037E4230E311CD1018C93882309F4B3C054
:10C740002091C9093091CA094091CB095091CC0977
:10C750006C966CAD7DAD8EAD9FAD6C970E94B2EACC
:10C760006DA77EA78FA798AB2091CD093091CE09F8
:10C770004091CF095091D009A0966CAD7DAD8EADA2
:10C780009FADA0970E94B2EA4B015C012091D109B4
:10C790003091D2094091D3095091D409A4966CAD3F
:10C7A0007DAD8EAD9FADA4970E94B2EA6B017C0176
:10C7B0002DA53EA54FA558A9CA01B9010E94CCE6F6
:10C7C0006DA77EA78FA798ABA5019401C501B40101
:10C7D0000E94CCE69B01AC016DA57EA58FA598A912
:10C7E0000E94B3EA4B015C01A7019601C701B601A3
:10C7F0000E94CCE69B01AC01C501B4010E94B3EAE2
:10C800000E941EED6B017C012091D5093091D60963
:10C810004091D7095091D80922966CAD7DAD8EAD6F
:10C820009FAD22970E94B2EAA70196010E948FEB6A
:10C830006B017C01F801E25BFF4F608371838283AF
:10C84000938320E030E040E450E40E94D9EC1816D5
:10C850001CF4F101108227C02091E3063091E40618
:10C860004091E5065091E606C701B6010E94CCE66C
:10C870009B01AC016091DF067091E0068091E106BA
:10C880009091E2060E948FEB29A53AA54BA55CA5E5
:10C890000E94CCE60E94FCEB6415750586059705A1
:10C8A00010F42B013C0180913B1190913C11A0911F
:10C8B0003D11B0913E110EA91FA928AD39AD8017C9
:10C8C0009107A207B30708F4DFC02DA13EA14FA135
:10C8D00058A5232B242B252B41F160913F117091FA
:10C8E00040118091411190914211641575058605A2
:10C8F0009705D8F42EA93FA948AD59AD0E9446EA44
:10C900006B017C012DA13EA14FA158A5C301B2012D
:10C910000E9446EAC616D706E806F90630F4C701B3
:10C92000B6010E9455EA29013A0188E60BA11CA133
:10C93000809FF001819FF00D1124E159FE4EC18CC2
:10C94000D28CE38CF48CC114D104E104F10431F1F4
:10C95000609143117091441180914511909146115D
:10C960006415750586059705C8F42EA93FA948AD3D
:10C9700059AD0E9446EA4B015C01A7019601C30133
:10C98000B2010E9446EA86169706A806B90630F458
:10C99000C501B4010E9455EA29013A0188E60BA1BC
:10C9A0001CA1809FF001819FF00D1124E159FE4EE2
:10C9B000C58CD68CE78CF0A0C114D104E104F1043D
:10C9C00031F1609147117091481180914911909116
:10C9D0004A116415750586059705C8F42EA93FA967
:10C9E00048AD59AD0E9446EA4B015C01A701960192
:10C9F000C301B2010E9446EA86169706A806B90648
:10CA000030F4C501B4010E9455EA29013A0188E6D3
:10CA10000BA11CA1809FF001819FF00D1124E15911
:10CA2000FE4EC1A0D2A0E3A0F4A0C114D104E10441
:10CA3000F10409F4C2CA60914B1170914C118091BC
:10CA40004D1190914E11641575058605970508F0F6
:10CA5000B4CA2EA93FA948AD59AD0E9446EA4B0180
:10CA60005C01A7019601C301B2010E9446EA861645
:10CA70009706A806B90608F0A0CAC501B4010E942D
:10CA800055EA29013A0199CA2DA13EA14FA158A505
:10CA9000232B242B252BC9F160913F11709140115C
:10CAA0008091411190914211641575058605970595
:10CAB00060F50E946BE62AAD3BAD4CAD5DAD0E94CA
:10CAC000CCE66B017C016DA17EA18FA198A50E948F
:10CAD0006BE64B015C01C301B2010E946BE6A5014C
:10CAE00094010E94CCE69B01AC01C701B6010E94F3
:10CAF00067E687FF0AC0A5019401C701B6010E943D
:10CB00008FEB0E94FCEB2B013C0188E60BA11CA1E2
:10CB1000809FF001819FF00D1124E159FE4E818C20
:10CB2000928CA38CB48C81149104A104B104B9F14A
:10CB3000609143117091441180914511909146117B
:10CB4000641575058605970550F50E946BE62AADBC
:10CB50003BAD4CAD5DAD0E94CCE66B017C01C501E7
:10CB6000B4010E946BE64B015C01C301B2010E945B
:10CB70006BE6A50194010E94CCE69B01AC01C701C4
:10CB8000B6010E9467E687FF0AC0A5019401C701AC
:10CB9000B6010E948FEB0E94FCEB2B013C0188E662
:10CBA0000BA11CA1809FF001819FF00D1124E15980
:10CBB000FE4E858C968CA78CB0A081149104A104A4
:10CBC000B104B9F1609147117091481180914911F8
:10CBD00090914A11641575058605970550F50E94D8
:10CBE0006BE62AAD3BAD4CAD5DAD0E94CCE66B0172
:10CBF0007C01C501B4010E946BE64B015C01C301DD
:10CC0000B2010E946BE6A50194010E94CCE69B0153
:10CC1000AC01C701B6010E9467E687FF0AC0A50103
:10CC20009401C701B6010E948FEB0E94FCEB2B011F
:10CC30003C0188E60BA11CA1809FF001819FF00DB3
:10CC40001124E159FE4EC1A0D2A0E3A0F4A0C1146A
:10CC5000D104E104F10409F4B0C960914B11709161
:10CC60004C1180914D1190914E11641575058605FA
:10CC7000970508F0A2C90E946BE62AAD3BAD4CAD0A
:10CC80005DAD0E94CCE64B015C01C701B6010E947C
:10CC90006BE66B017C01C301B2010E946BE6A70148
:10CCA00096010E94CCE69B01AC01C501B4010E9433
:10CCB00067E687FF82C9A7019601C501B4010E94FA
:10CCC0008FEB0E94FCEB2B013C0177C9FAA9FF23F3
:10CCD00031F1A5019401632D722DC8010E94CCE6AB
:10CCE0004B015C012DA53DA149A559A9C701B6017C
:10CCF0000E94CCE69B01AC01C501B4010E9467E62D
:10CD000087FF22C0A7019601C501B4010E948FEBE5
:10CD10006DA77DA389A799AB21E02AABFFC9A70125
:10CD20009601C501B4010E948FEB9B01AC016DA57A
:10CD30007DA189A599A90E94CCE66DA77DA389A7AD
:10CD400099AB31E03AABEAC941E04AABE7C9A70188
:10CD50009601C501B40113C0C701B6010E9467E680
:10CD600087FD09C020E030E0A901C501B4010E949F
:10CD7000D9EC18164CF4A5019401C701B6010E9424
:10CD8000B2EA2B013C0176CA2401350177FA70948E
:10CD900077F87094A3019201C701B6010E9467E67B
:10CDA00087FD68CA2601370165CA2DA53DA149A5A1
:10CDB00059A9C701B6010E9467E687FFB4CA3DA41E
:10CDC0002DA009A519A9AFCA81E004CBF090B30941
:10CDD0008FEF8F0D8F708BA3B090B2098091B30944
:10CDE000B81609F454C0C12CD12C0BA10B1509F4B1
:10CDF0004EC0602E712C28E6269D8001279D100DC7
:10CE0000112401591E4ED8018C9183FD2BC00EAF09
:10CE10001AAB0115110541F11996BC91BDA7F80196
:10CE2000F285FDA3D8011B96BC91B9A7F801F48542
:10CE3000F9ABD80115962D903D904D905C901897C8
:10CE4000A20191016DA57DA189A59F2F0E9467E692
:10CE5000811186C1C114D10439F0F601808180FDB1
:10CE60007FC102C0CEAEDAAA8BA181508F708BA396
:10CE70008091B2098B1103C0CEACDAA8B6CF0BA15A
:10CE80000B1529F081E08B0D8F70B82EF1CF10912A
:10CE9000B2091BA3C12CD12C8091B3090BA180171F
:10CEA00009F443CB802E912C28E6289D8001299DF2
:10CEB000100D112401591E4ED8018C9183FD0AC01A
:10CEC0005801C114D10439F0C6010E94487F811174
:10CED00002C0C5C156018BA18F5F8F708BA3650106
:10CEE000DBCF802F81508F70289FF0011124E159F2
:10CEF000FE4E908193FF24CB8DA71ECB48E6439F27
:10CF0000C0011124DC01A159BE4E1D018C9183FD8D
:10CF100019C015966D917D918D919C9118970E94E5
:10CF20001EEDF62EE72ED82EC92E0115110509F497
:10CF30008CC0F801808180FD0AC0D1018C9180FDF8
:10CF400006C083C0FDA0E9A4D9A8CEAC83C0F80177
:10CF5000808181608083C8010E94487F811171C0F7
:10CF6000F80161817281838194810E941EED2B0101
:10CF70003C019B01AC0160E070E080E89FE30E940F
:10CF80008FEB4B015C019B01AC016F2D7E2D8D2D34
:10CF90009C2D0E94CCE669837A838B839C832DA190
:10CFA00039A549A95EADC501B4010E94CCE6698BE3
:10CFB0007A8B8B8B9C8BAE014F5F5F4FBE016F5E98
:10CFC0007F4FC8010E9477B8F801E95BFF4F80816D
:10CFD0008823B9F12091E3063091E4064091E506FB
:10CFE0005091E606379660817181828193810E941B
:10CFF000CCE620919E1030919F104091A01050914E
:10D00000A1100E94CCE64B015C019B01AC01C30165
:10D01000B2010E94CCE60E94FCEBF801E65BFF4FF8
:10D0200071836083A50194016F2D7E2D8D2D9C2D24
:10D030000E94CCE60E94FCEBF801E45BFF4F718399
:10D040006083D8018C918E7F8C938F2C9E2CAD2C7D
:10D05000BC2C81018BA18F5F8F708BA3FDA2E9A6F1
:10D06000D9AACEAE79CAF101808181608083C801DE
:10D070000E94487F81116FC0D10111966D917D9101
:10D080008D919C9114970E941EED6B017C019B0178
:10D09000AC0160E070E080E89FE30E948FEB2B0121
:10D0A0003C012DEC3CEC4CE45DE30E94CCE6698352
:10D0B0007A838B839C839401A501C301B2010E94F2
:10D0C000CCE6698B7A8B8B8B9C8BAE014F5F5F4F6D
:10D0D000BE016F5E7F4FC1010E9477B8F101E95B2D
:10D0E000FF4F80818823B9F12091E3063091E40657
:10D0F0004091E5065091E606379660817181828104
:10D1000093810E94CCE620919E1030919F10409117
:10D11000A0105091A1100E94CCE64B015C019B0134
:10D12000AC01C701B6010E94CCE60E94FCEBF10104
:10D13000E65BFF4F718360832DEC3CEC4CE45DE3D8
:10D14000C501B4010E94CCE60E94FCEBF101E45B56
:10D15000FF4F71836083F10180818E7F808304CAD9
:10D1600028E6269DF001279DF00D1124E159FE4E81
:10D17000808181FD43C0C114D10441F0D6011596D0
:10D18000CD90DD90ED90FC90189708C08BE0C82EF4
:10D1900087EDD82E83E2E82E8BE3F82EB8E6B69D15
:10D1A000F001B79DF00D1124E159FE4E818992895D
:10D1B000A389B489BC01CD0190589B01AC010E94A8
:10D1C000B3EAF80125853685478550890E94CCE66B
:10D1D0009B01AC01C701B6010E94B2EAE62E872E80
:10D1E000982EA92E262F372F482F592F6DA57DA1B8
:10D1F00089A599A90E9467E687FF04C0EDA48DA0C8
:10D2000099A4A9A82E2D382D492D5A2DC201B1015E
:10D210000E9467E6882309F427CEF8E6F69DC00150
:10D22000F79D900D11249C0121593E4E6901D901B1
:10D230008C9181608C93C8010E94487F882329F0DB
:10D24000F60180818E7F80830FCE8E2D982DA92DA3
:10D25000BA2DF60185839683A783B08705CED601C4
:10D260008C9181FD52C0D60115962D913D914D9125
:10D270005C9118972DA73EA74FA758AB1501B5E0B5
:10D280002B0E311CF8014580568067807084A30105
:10D2900092016DA57EA58FA598A90E9467E687FFDC
:10D2A00034C0F60181899289A389B489BC01CD017A
:10D2B00090589B01AC010E94B3EAD6011D962D91B6
:10D2C0003D914D915C9150970E94CCE69B01AC0141
:10D2D0006DA57EA58FA598A90E94B2EA6B017C017D
:10D2E0009B01AC01C301B2010E94D9EC18166CF489
:10D2F000D8018C9181608C93C5010E94487F88235E
:10D30000E1F0F80180818E7F808318E6189DF0019E
:10D31000199DF00D1124E159FE4E2185328543857A
:10D32000548565817681878190850E9467E68111A9
:10D33000D2CD0BA10093B209CECDD101CD92DD9219
:10D34000ED92FC9213970BA10093B209DECFC8585F
:10D35000DF4F0FB6F894DEBF0FBECDBFDF91CF9188
:10D360001F910F91FF90EF90DF90CF90BF90AF9003
:10D370009F908F907F906F905F904F903F902F90F5
:10D3800008958091B3099091B409891B8F708F30F3
:10D3900019F40E942CA1F5CF8091B3098F5F8F7093
:10D3A000E091B30998E69E9FF0011124E159FE4EE9
:10D3B000DF011D929A95E9F798E090834091D90991
:10D3C0005091DA096091DB097091DC09458B568B2D
:10D3D000678B708F4091DD095091DE096091DF0904
:10D3E0007091E009418F528F638F748F4091E109F2
:10D3F0005091E2096091E3097091E409458F568FDD
:10D40000678F70A34091E5095091E6096091E709A3
:10D410007091E80941A352A363A374A32091B309B7
:10D420009091B409291303C094E69093B0098093B6
:10D43000B30980916F00826080936F00089590918E
:10D44000B3098091B409981306C080914A0790915E
:10D450004B07892B19F00E942CA1F1CF0895CF938F
:10D46000DF938B3D9240B1F0E1EDFDE18491EF015E
:10D470002196882321F00E94EE93FE01F7CFE8ED7C
:10D48000F9E18491EF012196882331F00E94EE9317
:10D49000FE01F7CF80E001C081E0DF91CF910895D8
:10D4A0002F923F924F925F926F927F928F929F92B4
:10D4B000AF92BF92CF92DF92EF92FF920F931F93A2
:10D4C000CF93DF93CDB7DEB7C757D1090FB6F89426
:10D4D000DEBF0FBECDBF2DB63EB6A7961FAE1EAEA9
:10D4E000A79784E690E0A9969FAF8EAFA99701E039
:10D4F0009E012B593F4F44E050E0BE01655A7F4FDB
:10D50000CE0189599F4F0E9422D09E012B593F4F37
:10D5100042E050E0BE0167597F4FCE0189599F4FCD
:10D520000E9422D043E050E0BE01655A7F4F8FED4C
:10D5300092E00E941EEE892B09F43FC06F968FADDA
:10D540006F97882339F08FE36C968FAF6C976D9649
:10D550001FAE6D97E6EEFDE184917F012FEFE21A99
:10D56000F20A811103C0EBE9FAE104C00E94EE93D4
:10D57000F701F2CF84917F013FEFE31AF30A88238A
:10D5800021F00E94EE93F701F5CFBE01655A7F4F5F
:10D5900082E99AE10E9497C5E4E8FAE184917F016B
:10D5A0009FEFE91AF90A882321F00E94EE93F70110
:10D5B000F5CF81E08093160754C5EDB7FEB7E69628
:10D5C000FFAFEEAFE6976B961CAE1DAE1EAE1FAE64
:10D5D0006B97A7961FAE1EAEA79701E09E012B5931
:10D5E0003F4F41E050E0BE0160597F4FCE01895965
:10D5F0009F4F0E9422D080E1EBE5F2E0DE019196A0
:10D6000001900D928A95E1F780E1EBE6F2E0DE0110
:10D61000519601900D928A95E1F780E1EBE7F2E0F7
:10D62000DE01119601900D928A95E1F7E1964FADDA
:10D63000E19750E04D5F5F4F440F551F440F551F5A
:10D640002DB73EB7241B350B0FB6F8943EBF0FBE67
:10D650002DBF8DB79EB701967C0100E09E012B592E
:10D660003F4FBC01CE0189599F4F0E9422D09E019D
:10D670002B593F4F44E050E063E077E0CE018959F9
:10D680009F4F0E9422D0E1968FACE197912C93E0BE
:10D69000890E911C880C991C880C991CEDB7FEB75B
:10D6A000E819F9090FB6F894FEBF0FBEEDBF2DB70C
:10D6B0003EB72F5F3F4F69018DB79EB78819990913
:10D6C0000FB6F8949EBF0FBE8DBFEDB7FEB7319673
:10D6D0005F019E012B593F4FA401B601CE0189592C
:10D6E0009F4F0E9422D09E012B593F4FA401B501AC
:10D6F000CE0189599F4F0E9422D010911707112304
:10D7000009F4A7C000E09E012B593F4F44E050E0D0
:10D710006BEE76E0CE0189599F4F0E9422D09E0188
:10D720002B593F4F44E050E06FEE76E0CE0189592F
:10D730009F4F0E9422D09E012B593F4F44E050E062
:10D7400067EE76E0CE0189599F4F0E9422D09E015C
:10D750002B593F4F44E050E06BE077E0CE01895910
:10D760009F4F0E9422D09E012B593F4F44E050E032
:10D7700067E077E0CE0189599F4F0E9422D09E0139
:10D780002B593F4F40E150E063ED76E0CE018959DF
:10D790009F4F0E9422D09E012B593F4F44E050E002
:10D7A000BE01695A7F4FCE0189599F4F0E9422D0F6
:10D7B0009E012B593F4F4CE050E068E375E0CE01ED
:10D7C00089599F4F0E9422D09E012B593F4F44E020
:10D7D00050E063E371E1CE0189599F4F0E9422D04E
:10D7E0009E012B593F4F44E050E0BE01695A7F4FE4
:10D7F000CE0189599F4F0E9422D001E09E012B59F2
:10D800003F4F41E050E0BE0161597F4FCE01895941
:10D810009F4F0E9422D09E012B593F4F41E050E084
:10D82000BE0162597F4FCE0189599F4F0E9422D07D
:10D8300011118AC06B968CAD9DADAEADBFAD6B972F
:10D840008093C2109093C310A093C410B093C510DE
:10D850007BC0E1968FADE19790E0029623EF36E032
:10D86000E4963FAF2EAFE497B501DE011196E2E9F1
:10D870008E2EE0E19E2EAE014F5E5F4FFFE4AF2E95
:10D88000F1E1BF2EE896FFAEEEAEE8977E0131E201
:10D89000E30EF11C20E030E0821793072CF0E896AD
:10D8A000EEADFFADE89701C0F70140805180628086
:10D8B0007380F50141925192619271925F018217DA
:10D8C000930714F0F60101C0FA0140805180628094
:10D8D0007380F40141925192619271924F018217CB
:10D8E000930734F0FB01408051806280738005C053
:10D8F0004D905D906D907C901397E496EEADFFADEA
:10D90000E4974192519261927192E496FFAFEEAF2B
:10D91000E4972F5F3F4F6C5F7F4F1496F4E0CF0E7C
:10D92000D11C4C5F5F4FE896EEADFFADE8973496A3
:10D93000E896FFAFEEAFE897F4E0EF0EF11C24306D
:10D94000310509F0A9CFDECEE0968FADE0978530A6
:10D9500099F4AF968FADAF97853071F400E09E01DA
:10D960002B593F4F44E650E066EC70E1CE018959F7
:10D970009F4F0E9422D024C0111102C00E94DFBD1F
:10D98000E0968FADE097AF96CFACAF978C9D6001DE
:10D990001124E12CF12CEC14FD0491F000E09E0127
:10D9A0002B593F4F44E050E0BE01695A7F4FCE01F2
:10D9B00089599F4F0E9422D02FEFE21AF20AEBCF33
:10D9C00000E09E012B593F4F44E050E0BE016D5AEC
:10D9D0007F4FCE0189599F4F0E9422D01AE01150EB
:10D9E00079F000E09E012B593F4F44E050E0BE012A
:10D9F000695A7F4FCE0189599F4F0E9422D0EFCFA5
:10DA000001E09E012B593F4F41E050E0BE016359B8
:10DA10007F4FCE0189599F4F0E9422D09E012B59E2
:10DA20003F4F41E050E0BE0164597F4FCE0189591C
:10DA30009F4F0E9422D000E09E012B593F4F44E0AF
:10DA400050E0BE01635C7F4FCE0189599F4F0E9419
:10DA500022D09E012B593F4F44E050E0BE016F5C45
:10DA60007F4FCE0189599F4F0E9422D0AE968FAD35
:10DA7000AE97AD96CFACAD978C9D60011124E12C93
:10DA8000F12C00E09E012B593F4FCE14DF0471F0C2
:10DA900044E050E0BE01695A7F4FCE0189599F4F43
:10DAA0000E9422D03FEFE31AF30AEBCF41E050E0AF
:10DAB000BE016F587F4FCE0189599F4F0E9422D0DF
:10DAC0009E012B593F4F41E050E0BE0165597F4F09
:10DAD000CE0189599F4F0E9422D09E012B593F4F62
:10DAE00044E050E0BE01695A7F4FCE0189599F4FF3
:10DAF0000E9422D09E012B593F4F44E050E0BE01CE
:10DB0000695A7F4FCE0189599F4F0E9422D09E01B2
:10DB10002B593F4F44E050E067E371E1CE01895952
:10DB20009F4F0E9422D09E012B593F4F44E050E06E
:10DB3000BE01615B7F4FCE0189599F4F0E9422D069
:10DB40009E012B593F4F44E050E0BE01655B7F4F83
:10DB5000CE0189599F4F0E9422D09E012B593F4FE1
:10DB600044E050E0BE01695B7F4FCE0189599F4F71
:10DB70000E9422D010E000E09E012B593F4F44E06C
:10DB800050E0BE01695A7F4FCE0189599F4F0E94D4
:10DB900022D0111110C06B96CCACDDACEEACFFAC5A
:10DBA0006B9720E030E84BE355E4C701B6010E94D3
:10DBB00067E6811103C054E0F52E33C0809117074A
:10DBC000811108C0C0923C07D0923D07E0923E0709
:10DBD000F0923F0700E09E012B593F4F44E050E098
:10DBE00068E377E0CE0189599F4F0E9422D09E01C1
:10DBF0002B593F4F44E050E060E477E0CE01895973
:10DC00009F4F0E9422D09E012B593F4F44E050E08D
:10DC1000BE01695A7F4FCE0189599F4F0E9422D081
:10DC200012C0FA94FF2079F000E09E012B593F4F7B
:10DC300044E050E0BE01695A7F4FCE0189599F4FA1
:10DC40000E9422D0EECF1F5F153009F094CF00E084
:10DC50009E012B593F4F42E050E0BE016D597F4F6E
:10DC6000CE0189599F4F0E9422D09E012B593F4FD0
:10DC700044E050E0BE01695A7F4FCE0189599F4F61
:10DC80000E9422D06B96CCACDDACEEACFFAC6B97B7
:10DC900020E030E84BE355E4C701B6010E9467E697
:10DCA000882329F180911707811108C0C092340799
:10DCB000D0923507E0923607F092370700E09E01D8
:10DCC0002B593F4F44E050E060E377E0CE018959A3
:10DCD0009F4F0E9422D09E012B593F4F44E050E0BD
:10DCE0006CE277E0CE0189599F4F0E9422D000E07C
:10DCF0009E012B593F4F42E050E0BE016F597F4FCC
:10DD0000CE0189599F4F0E9422D09E012B593F4F2F
:10DD100041E050E0BE016F587F4FCE0189599F4FBF
:10DD20000E9422D019E0115000E09E012B593F4F74
:10DD3000112359F044E050E0BE01695A7F4FCE01F3
:10DD400089599F4F0E9422D0EECF41E050E06AE215
:10DD500071E1CE0189599F4F0E9422D0F12C00E041
:10DD60009E012B593F4F44E050E0BE01695A7F4F5E
:10DD7000CE0189599F4F0E9422D01091170711118F
:10DD800010C0F1100EC06B968CAD9DADAEADBFADA9
:10DD90006B9780932F1190933011A0933111B09312
:10DDA0003211F39485E0F812DACF111102C00E940B
:10DDB000DFC44CE0F42EFA94F11003C03CE0F32EE3
:10DDC0000FC000E09E012B593F4F42E050E0BE01E2
:10DDD000615A7F4FCE0189599F4F0E9422D0EBCFCD
:10DDE000FA9400E09E012B593F4FFF2059F044E088
:10DDF00050E0BE016D5B7F4FCE0189599F4F0E945D
:10DE000022D0EECF46E050E0BE01635C7F4FCE01F2
:10DE100089599F4F0E9422D09E012B593F4F44E0C9
:10DE200050E063EE76E0CE0189599F4F0E9422D0E8
:10DE30009E012B593F4F4CE050E0BE016F5C7F4F7D
:10DE4000CE0189599F4F0E9422D02CE1F22EFA94E4
:10DE5000F11003C094E0F92E1DC000E09E012B5983
:10DE60003F4F44E050E0BE01695A7F4FCE018959CF
:10DE70009F4F0E9422D0EBCF00E09E012B593F4FD5
:10DE800044E050E0BE01695A7F4FCE0189599F4F4F
:10DE90000E9422D0FA94F110EFCF8BE0F82EFA9482
:10DEA000FF2079F000E09E012B593F4F44E050E005
:10DEB000BE01695A7F4FCE0189599F4F0E9422D0DF
:10DEC000EECFA9968EAD9FADA99784569109C7DA7A
:10DED00080931607882309F1E6EEFDE184917F0126
:10DEE0009FEFE91AF90A882321F00E94EE93F701C7
:10DEF000F5CFA9966EAD7FADA997645671098CE7F1
:10DF00009AE10E947EC56BED72E084E79AE10E947F
:10DF10007EC58AE00E94EE9399C0A7962EAD3FADD4
:10DF2000A797AB968EAD9FADAB972817390709F42D
:10DF30004BC081E080931607E1EDFDE184917F0104
:10DF40002FEFE21AF20A811103C0E4E5FAE104C0FE
:10DF50000E94EE93F701F2CF84917F013FEFE31A25
:10DF6000F30A882321F00E94EE93F701F5CFAB96D8
:10DF70006EAD7FADAB9780E090E04AE00E940F97D6
:10DF8000EFE4FAE184917F019FEFE91AF90A88230F
:10DF900021F00E94EE93F701F5CFA7966EAD7FAD0D
:10DFA000A79780E090E04AE00E940F97EFE3FAE144
:10DFB00084917F012FEFE21AF20A882309F446C008
:10DFC0000E94EE93F701F4CF111142C0E6EEFDE19D
:10DFD00084917F013FEFE31AF30A811103C00FED33
:10DFE00012E004C00E94EE93F701F2CFF801819194
:10DFF0008F01882319F00E94EE93F8CFA9966EAD99
:10E000007FADA9976456710982E29AE10E947EC5AC
:10E01000A7964EAD5FADA79760E070E085E19AE10D
:10E020000E9444C5E2E1FAE184917F012FEFE21AF8
:10E03000F20A811107C080911607811109C00E9460
:10E04000E3D006C00E94EE93F701EECF112399F3BF
:10E05000E6968EAD9FADE6970FB6F8949EBF0FBEC5
:10E060008DBF80911707811102C00E94ACBE9091B4
:10E07000160781E089270FB6F8943EBE0FBE2DBE6D
:10E08000C958DF4F0FB6F894DEBF0FBECDBFDF918A
:10E09000CF911F910F91FF90EF90DF90CF90BF90A5
:10E0A000AF909F908F907F906F905F904F903F9038
:10E0B0002F90089581E080931707F2D910921707E7
:10E0C0008111EEC90E941BC381E008958F929F9237
:10E0D000AF92BF92CF92DF92EF92FF920F931F9376
:10E0E000CF93DF93CDB7DEB7CA5AD1090FB6F894F4
:10E0F000DEBF0FBECDBFE9961CAE1DAE1EAE1FAE7D
:10E10000E9978091EC039091ED03A091EE03B0911B
:10E11000EF03ED968CAF9DAFAEAFBFAFED97C55699
:10E12000DF4F19821882CB59D04084E690E0C35665
:10E13000DF4F99838883CD59D040109216079E01F6
:10E1400025563F4F44E050E0BE0167587F4FCE0157
:10E1500083569F4F0E946FD0C356DF4F88819981AD
:10E16000CD59D0400296C356DF4F99838883CD594D
:10E17000D040C556DF4F19821882CB59D04081E07C
:10E18000CD55DF4F8883C35AD0409E0125563F4F5F
:10E1900041E050E0BE016D557F4FCE0183569F4F49
:10E1A0000E946FD09E0125563F4F40E150E06FE442
:10E1B00071E1CE0183569F4F0E946FD09E0125567C
:10E1C0003F4F44E050E063E077E0CE0183569F4F3D
:10E1D0000E946FD09E0125563F4F40E150E062E91A
:10E1E00070E1CE0183569F4F0E946FD09E0125564D
:10E1F0003F4F40E150E063EF76E0CE0183569F4F02
:10E200000E946FD09E0125563F4F44E050E06BEED8
:10E2100076E0CE0183569F4F0E946FD09E01255617
:10E220003F4F44E050E06FEE76E0CE0183569F4FC3
:10E230000E946FD09E0125563F4F44E050E067EEAC
:10E2400076E0CE0183569F4F0E946FD09E012556E7
:10E250003F4F44E050E06BE077E0CE0183569F4FA4
:10E260000E946FD09E0125563F4F44E050E067E08A
:10E2700077E0CE0183569F4F0E946FD09E012556B6
:10E280003F4F40E150E063ED76E0CE0183569F4F73
:10E290000E946FD08AE097EDA3EABCE3E9968CAFC9
:10E2A0009DAFAEAFBFAFE9979E0125563F4F44E00B
:10E2B00050E0BE016B587F4FCE0183569F4F0E94A6
:10E2C0006FD09E0125563F4F4CE050E068E375E06B
:10E2D000CE0183569F4F0E946FD080917D10909108
:10E2E0007E10A0917F10B0918010C358DF4F8883BB
:10E2F0009983AA83BB83CD57D0409E0125563F4FBB
:10E3000044E050E0BE0163587F4FCE0183569F4FDB
:10E310000E946FD085E0CC55DF4F8883C45AD0402F
:10E32000CB55DF4F8883C55AD0409E0125563F4FBD
:10E3300044E050E062EC70E1CE0183569F4F0E94B2
:10E340006FD09E0125563F4F41E050E0BE016C5515
:10E350007F4FCE0183569F4F0E946FD09E0125565E
:10E360003F4F41E050E0BE016B557F4FCE018356D9
:10E370009F4F0E946FD09E0125563F4F44E650E0CC
:10E3800066EC70E1CE0183569F4F0E946FD0CF574D
:10E39000DF4F188219821A821B82C158D0409E0119
:10E3A00025563F4F44E050E0BE016F577F4FCE01EE
:10E3B00083569F4F0E946FD0E9961CAE1DAE1EAED5
:10E3C0001FAEE9971AE0115071F09E0125563F4F9C
:10E3D00044E050E0BE016B587F4FCE0183569F4F03
:10E3E0000E946FD0F0CF83E0CA55DF4F8883C65AB2
:10E3F000D040C955DF4F8883C75AD040CB57DF4F35
:10E40000188219821A821B82C558D040C757DF4F25
:10E41000188219821A821B82C958D040E9961CAE14
:10E420001DAE1EAE1FAEE9979E0125563F4F41E03F
:10E4300050E0BE016A557F4FCE0183569F4F0E9428
:10E440006FD09E0125563F4F41E050E0BE01695517
:10E450007F4FCE0183569F4F0E946FD09E0125565D
:10E460003F4F44E050E0BE0167577F4FCE018356D7
:10E470009F4F0E946FD09E0125563F4F44E050E0D1
:10E48000BE016B577F4FCE0183569F4F0E946FD0C6
:10E490000AE010E00150110971F09E0125563F4F2E
:10E4A00044E050E0BE016B587F4FCE0183569F4F32
:10E4B0000E946FD0EFCFC855DF4F1882C85AD040A6
:10E4C0008FEFC755DF4F8883C95AD0409E0125562C
:10E4D0003F4F41E050E0BE0168557F4FCE0183566B
:10E4E0009F4F0E946FD09E0125563F4F41E050E064
:10E4F000BE0167557F4FCE0183569F4F0E946FD05C
:10E50000E9961CAE1DAE1EAE1FAEE9979E012556C4
:10E510003F4F44E050E0BE016B587F4FCE01835621
:10E520009F4F0E946FD09E0125563F4F44E050E020
:10E53000BE016B587F4FCE0183569F4F0E946FD014
:10E540009E0125563F4F44E050E067E371E1CE0164
:10E5500083569F4F0E946FD080918B0290918C02C6
:10E56000A0918D02B0918E02C357DF4F88839983AB
:10E57000AA83BB83CD58D04080918F0290919002A6
:10E58000A0919102B0919202CF56DF4F8883998378
:10E59000AA83BB83C159D040CB56DF4F1982188262
:10E5A000C559D040C956DF4F19821882C759D0408B
:10E5B0009E0125563F4F44E050E0BE0163577F4F18
:10E5C000CE0183569F4F0E946FD09E0125563F4F2C
:10E5D00044E050E0BE016F567F4FCE0183569F4FFF
:10E5E0000E946FD09E0125563F4F44E050E0BE018F
:10E5F0006B567F4FCE0183569F4F0E946FD010E025
:10E60000C12C80E8D82E8BE3E82E85E4F82E812CEF
:10E61000912C90E8A92E9FE3B92E111138C09E01CC
:10E6200025563F4F44E050E06CE377E0CE0183563F
:10E630009F4F0E946FD09E0125563F4F44E050E00F
:10E6400068E377E0CE0183569F4F0E946FD09E0112
:10E6500025563F4F44E050E060E477E0CE0183561A
:10E660009F4F0E946FD0E9968CAE9DAEAEAEBFAE0E
:10E67000E9979E0125563F4F44E050E0BE016B589C
:10E680007F4FCE0183569F4F0E946FD02AC0E996DC
:10E69000CCAEDDAEEEAEFFAEE9979E0125563F4F04
:10E6A00044E050E0BE016B587F4FCE0183569F4F30
:10E6B0000E946FD0E9961CAE1DAE1EAE1FAEE9974C
:10E6C00004E0015071F09E0125563F4F44E050E0B8
:10E6D000BE016B587F4FCE0183569F4F0E946FD073
:10E6E000F0CF1F5F153009F098CF84E190E0C1565C
:10E6F000DF4F99838883CF59D0409E0125563F4FE5
:10E7000042E050E0BE0161567F4FCE0183569F4FDD
:10E710000E946FD09E0125563F4F44E050E064E3D5
:10E7200077E0CE0183569F4F0E946FD09E01255601
:10E730003F4F44E050E060E377E0CE0183569F4FC7
:10E740000E946FD09E0125563F4F44E050E06CE29E
:10E7500077E0CE0183569F4F0E946FD080E290E019
:10E76000CF55DF4F99838883C15AD0409E012556EB
:10E770003F4F42E050E0BE016F557F4FCE018356C0
:10E780009F4F0E946FD0C655DF4F1882CA5AD040A3
:10E7900080E2E3E9F2E0DE019D9601900D928A9518
:10E7A000E1F79E0125563F4F41E050E0BE0166551E
:10E7B0007F4FCE0183569F4F0E946FD09E012556FA
:10E7C0003F4F40E250E0BE01635D7F4FCE01835674
:10E7D0009F4F0E946FD09E0125563F4F41E050E071
:10E7E0006AE271E1CE0183569F4F0E946FD010E024
:10E7F00011110EC080912F1190913011A091311103
:10E80000B0913211E9968CAF9DAFAEAFBFAFE99733
:10E810009E0125563F4F44E050E0BE016B587F4FAC
:10E82000CE0183569F4F0E946FD01F5F153001F7B6
:10E83000BE01635B7F4F86E1FB0111928A95E9F788
:10E840009E0125563F4F46E150E0CE0183569F4F33
:10E850000E946FD08CE2E3EBF2E0DE0111960190B2
:10E860000D928A95E1F79E0125563F4F4CE250E00C
:10E87000BE016F5F7F4FCE0183569F4F0E946FD0C6
:10E88000BE0161597F4F86E0FB0111928A95E9F73D
:10E890009E0125563F4F46E050E0CE0183569F4FE4
:10E8A0000E946FD09E0125563F4F44E050E063EE3A
:10E8B00076E0CE0183569F4F0E946FD0BE016D5906
:10E8C0007F4F8CE0FB0111928A95E9F79E01255656
:10E8D0003F4F4CE050E0CE0183569F4F0E946FD0D7
:10E8E000E9961CAE1DAE1EAE1FAEE9971CE111509D
:10E8F00071F09E0125563F4F44E050E0BE016B5839
:10E900007F4FCE0183569F4F0E946FD0F0CFE99684
:10E910001CAE1DAE1EAE1FAEE99714E0115071F093
:10E920009E0125563F4F44E050E0BE016B587F4F9B
:10E93000CE0183569F4F0E946FD0F0CFE9961CAE58
:10E940001DAE1EAE1FAEE9971BE0115071F09E0187
:10E9500025563F4F44E050E0BE016B587F4FCE013B
:10E9600083569F4F0E946FD0F0CF80911607811180
:10E9700067C0C356DF4FE880F980CD59D040F4E638
:10E98000EF1AF108C556DF4F88819981CB59D040E5
:10E99000C756DF4F99838883C959D04084E690E0F9
:10E9A000C356DF4F99838883CD59D0409E012556A9
:10E9B0003F4F44E050E06FED72E0CE0183569F4F31
:10E9C0000E946FD09E0125563F4F42E050E0BE01AD
:10E9D00067567F4FCE0183569F4F0E946FD0E6EE61
:10E9E000FDE184918F010F5F1F4F882321F00E946A
:10E9F000EE93F801F6CFB70180E09AE10E947EC560
:10EA0000C756DF4F48815981C959D04060E070E056
:10EA100083EF99E10E9444C5E0EFF9E184918F0111
:10EA20000F5F1F4F882321F00E94EE93F801F6CF6D
:10EA3000C7010E942F6A90911607892B80931607B1
:10EA40009091160781E08927C655DF4F0FB6F894DD
:10EA5000DEBF0FBECDBFDF91CF911F910F91FF9011
:10EA6000EF90DF90CF90BF90AF909F908F900895E0
:10EA7000FF920F931F93CF93DF938C01EB01F42E42
:10EA800080E20E94EE938FEFF81611F084E501C04A
:10EA900082E40E94EE938AE30E94EE93F801608183
:10EAA00071818281938142E00E94949748815981CB
:10EAB0006A817B818FE49DE10E9461C562E070E024
:10EAC00080E090E0DF91CF911F910F91FF900C9427
:10EAD0003AB78F929F92AF92BF92CF92DF92EF920E
:10EAE000FF920F931F93CF93DF93F0E2FF2EE12C61
:10EAF000AE2DB0E0BD016F0D711D759567956E155A
:10EB000011F0F6120BC0E2E3FBE165917491072E60
:10EB1000000C880B990B0E946DE662C09B0121508E
:10EB20003109220F331F220F331FF901EC54F54E28
:10EB300005911491AB01440F551F440F551FFA0165
:10EB4000EC54F54EC591D4918017910714F4F62E2C
:10EB5000D1CFC817D90714F4E62ECACFF901EA5469
:10EB6000F54EE590F490FA01EA54F54EC590D49034
:10EB7000BC01601B710B072E000C880B990B0E94C7
:10EB80006DE64B015C01B6016E197F09072E000C82
:10EB9000880B990B0E946DE69B01AC01C501B40185
:10EBA0000E94CCE64B015C01C01BD10BBE01DD0F06
:10EBB000880B990B0E946DE69B01AC01C501B40165
:10EBC0000E948FEB4B015C01B701FF0C880B990B86
:10EBD0000E946DE69B01AC01C501B4010E94B3EA3D
:10EBE000DF91CF911F910F91FF90EF90DF90CF9029
:10EBF000BF90AF909F908F9008950F931F93CF93E6
:10EC0000DF93CDB7DEB728970FB6F894DEBF0FBEFF
:10EC1000CDBF60914A0470914B04072E000C880B05
:10EC2000990B0E946DE66D837E838F839887809118
:10EC30004C0490914D04A0914E04B0914F048983EF
:10EC40009A83AB83BC834DEFBE016B5F7F4FCE01D8
:10EC500001960EDF6091440470914504072E000C6C
:10EC6000880B990B0E946DE66D837E838F83988756
:10EC70008091460490914704A0914804B0914904C2
:10EC800089839A83AB83BC834FEFBE016B5F7F4F59
:10EC9000CE010196EDDEE7E5FDE184918F010F5F86
:10ECA0001F4F882321F00E94EE93F801F6CFE091E8
:10ECB0004E07F0E0E45BF84F608170E080E090E0A8
:10ECC0000E947A97E2E5FDE184918F010F5F1F4F6B
:10ECD000882321F00E94EE93F801F6CF60914D0752
:10ECE00070E080E090E00E947A9728960FB6F89442
:10ECF000DEBF0FBECDBFDF91CF911F910F91089561
:10ED00000F930FB70F9300916E000B7F00936E006F
:10ED100078940F930BB70F930CB70F921F922F930A
:10ED20003F934F935F936F937F938F939F93AF9393
:10ED3000BF93EF93FF931124EFD2FF91EF91BF9117
:10ED4000AF919F918F917F916F915F914F913F9183
:10ED50002F911F900F900CBF0F910BBF0F9104606C
:10ED6000F89400936E000F910FBF0F911895CF92FA
:10ED7000DF92EF92FF92C0904604D0904704E0905B
:10ED80004804F09049046091440470914504665031
:10ED90007109072E000C880B990B0E946DE69B01F0
:10EDA000AC01C701B6010E9467E687FF1FC020E0E3
:10EDB00030E040E050E4C701B6010E94B3EA0E948F
:10EDC000FCEB70938607609385070E94FF58DC0177
:10EDD000CB01805A9541AF4FBF4F809381079093ED
:10EDE0008207A0938307B093840708C0109281071D
:10EDF000109282071092830710928407FF90EF9081
:10EE0000DF90CF900895CF92DF92EF92FF92C09063
:10EE10004C04D0904D04E0904E04F0904F0460916B
:10EE20004A0470914B0469507109072E000C880B3D
:10EE3000990B0E946DE69B01AC01C701B6010E94CF
:10EE400067E687FF1FC020E030E040EA50E4C701DA
:10EE5000B6010E94B3EA0E94FCEB709380076093B6
:10EE60007F070E94FF58DC01CB0188549747AF4FC2
:10EE7000BF4F80937B0790937C07A0937D07B0934F
:10EE80007E0708C010927B0710927C0710927D07C6
:10EE900010927E07FF90EF90DF90CF9008958F92B1
:10EEA0009F92AF92BF92CF92DF92EF92FF920F9319
:10EEB0001F93CF93DF93F0E4FF2EE12CAE2DB0E053
:10EEC000BD016F0D711D759567956E1511F0F612E8
:10EED0000BC0E4EAFCE165917491072E000C880BED
:10EEE000990B0E946DE662C09B0121503109220FEF
:10EEF000331F220F331FF901EA55F44E0591149187
:10EF0000AB01440F551F440F551FFA01EA55F44E4B
:10EF1000C591D4918017910714F4F62ED1CFC8175C
:10EF2000D90714F4E62ECACFF901E855F44EE5905E
:10EF3000F490FA01E855F44EC590D490BC01601BE2
:10EF4000710B072E000C880B990B0E946DE64B018C
:10EF50005C01B6016E197F09072E000C880B990B16
:10EF60000E946DE69B01AC01C501B4010E94CCE694
:10EF70004B015C01C01BD10BBE01DD0F880B990B4F
:10EF80000E946DE69B01AC01C501B4010E948FEBAC
:10EF90004B015C01B701FF0C880B990B0E946DE6D9
:10EFA0009B01AC01C501B4010E94B3EADF91CF918E
:10EFB0001F910F91FF90EF90DF90CF90BF90AF9097
:10EFC0009F908F90089560E08091910790919207B3
:10EFD00080DD60934C0470934D0480934E049093B5
:10EFE0004F0480918F079091900759DF60934604FA
:10EFF000709347048093480490934904A895109215
:10F00000490708957F928F929F92AF92BF92CF92BD
:10F01000DF92EF92FF920F931F93CF93DF9320E045
:10F0200030E048E452E460914C0470914D048091CA
:10F030004E0490914F040E94D9EC18164CF4EAE368
:10F04000FBE1E491C1E001C0CC0FEA95EAF701C011
:10F05000C0E084E3E82E8BE1F82E0AE31BE196E0A2
:10F06000A92E912CD0E0CC24C394D12CF70174901C
:10F07000F801849077FC23C0892D90E0082C02C011
:10F08000959587950A94E2F780FD19C0BE01082C7A
:10F0900002C0759567950A94E2F76170B62EB19437
:10F0A0006B2D872D0E9409B66B2D70E0872D0E9475
:10F0B00073B6C60101C0880F8A94EAF7982AAA9409
:10F0C000FFEFEF1AFF0A0F5F1F4FA110CFCFDF91A5
:10F0D000CF911F910F91FF90EF90DF90CF90BF9055
:10F0E000AF909F908F907F9008950F931F93809182
:10F0F0002B07813019F40E94FF5808C06091270740
:10F10000709128078091290790912A070091530751
:10F11000109154072091550730915607601B710BD1
:10F12000820B930B28EE33E040E050E00E9455EA5A
:10F1300080914F0790915007A0915107B0915207CD
:10F14000BC01CD01620F731F841F951F1F910F918A
:10F15000089510922B0710925307109254071092A3
:10F160005507109256071092270710922807109201
:10F17000290710922A0710924F07109250071092F9
:10F18000510710925207089580912B078130E1F0CA
:10F19000823051F4AADF60934F0770935007809339
:10F1A00051079093520701C0D4DF81E080932B0771
:10F1B0000E94FF586093530770935407809355073C
:10F1C0009093560781E0089580E0089580912B0781
:10F1D000813079F482E080932B070E94FF5860937E
:10F1E0002707709328078093290790932A0781E0C7
:10F1F000089580E0089580912B078150823010F0AF
:10F2000080E0089510922B070E94FF586093270713
:10F21000709328078093290790932A0781E0089527
:10F220001092480780E090E00E94F4591092450443
:10F23000109244049CDDDFDF80E090E00E94F459EE
:10F2400010924C072C98109245041092440410928E
:10F250004D07809102018072809300010895DF9232
:10F26000EF92FF920F931F93CF93DF93F82ED62E3A
:10F27000E72E8A0180912702882309F439C0E1ED45
:10F28000FDE18491EF012196882321F00E94EE9305
:10F29000FE01F7CFED2DFE2D8491EF0121968823FD
:10F2A00021F00E94EE93FE01F7CFE5E4FBE18491AB
:10F2B000EF012196882321F00E94EE93FE01F7CF03
:10F2C000F7FC0BC06F2DFF0C770B880B990B0E947E
:10F2D0007A978AE00E94EE930BC0E0E4FBE1849110
:10F2E000EF012196882321F00E94EE93FE01F7CFD3
:10F2F00080915707811108C01092270281E0809306
:10F300005707C8010E94E5A0DF91CF911F910F918F
:10F31000FF90EF90DF9084CFEF92FF920F931F93B7
:10F32000CF93DF9380912A028F37A0F08F5790916F
:10F330004C079093A207992311F02C9A01C02C98A6
:10F3400020914D072093A10790910201222369F09B
:10F3500090950BC09091A207891708F02C98909176
:10F36000A107891728F090910201907290930001F3
:10F370008F5F80932A029091A00781E08927809374
:10F38000A0078091290285301CF4C1E0C80F01C09C
:10F39000C0E0823009F4B4C054F4882301F1813014
:10F3A00009F0E3C088E080937B0085E4C0C084302E
:10F3B00009F4C5C00CF4B7C0853009F0D6C09091EF
:10F3C0009F07911102C080939F0780919F078150F2
:10F3D00080939F07882309F4C8C0C5E0C6C0809108
:10F3E00028028F5F80311CF480932802BEC01092E7
:10F3F000280280914907811113C08091950790914F
:10F40000960790939207809391078091930790912C
:10F4100094079093900780938F0781E0809349072A
:10F420008AE0E5E9F7E0DF011D928A95E9F710929D
:10F4300094071092930700919107109192071195EC
:10F440000195110980914A0490914B04D1E018165E
:10F4500019062CF080914C07811101C0D0E08091F9
:10F460003205909133059195819591098017910707
:10F4700034F44DED5CE16EEF7CE180E0F0DE8091F4
:10F480001C0290911D029195819591090817190709
:10F4900044F4DD2331F040E15DE161E37DE180E0B2
:10F4A000DEDE809144049091450411E0181619069F
:10F4B0002CF080914D07811101C010E0E0908F0782
:10F4C000F090900780913005909131058E159F0541
:10F4D00034F04DEE5CE16EEF7CE18FEFC0DE8091A9
:10F4E0001A0290911B02E816F9060CF43EC0112393
:10F4F000E1F140E25DE161E37DE18FEFB0DE35C037
:10F5000080917A0086FD2EC08091780090917900DC
:10F510002091950730919607820F931F909396073D
:10F520008093950722C088E080937B0086E48093D7
:10F530007C0080917A00806480937A0016C080916C
:10F540007A0086FD11C08091780090917900209119
:10F55000930730919407820F931F909394078093A1
:10F56000930703C0C2E001C0C4E0C09329028091A8
:10F57000370581110E94EFBD80914A0790914B079A
:10F580000097A9F0019790934B0780934A07892B26
:10F5900071F483E49DE19093A4078093A307DF9126
:10F5A000CF911F910F91FF90EF900C941A94DF91DF
:10F5B000CF911F910F91FF90EF9008952F923F925E
:10F5C0004F925F926F927F928F929F92AF92BF9273
:10F5D000CF92DF92EF92FF920F931F93CF93DF931F
:10F5E00000D01F92CDB7DEB75C017A8369834A01F0
:10F5F000170107FD07C0802F002E000C990B9C837C
:10F600008B8304C0E1E0F0E0FC83EB83F9014080F0
:10F610005180628073808B819C81880F991F880F35
:10F62000991F9C838B838957984F7C01A30192017A
:10F63000FC0160817181828193810E9467E6882349
:10F6400091F0F701408251826282738211E020E0E2
:10F6500030E0A901C301B2010E94D9EC18160CF0E8
:10F6600010E0F5011083F50180818230D1F0833004
:10F6700009F45EC0813009F07CC0EB81FC81E95760
:10F68000F84F2081318142815381F4016081718181
:10F69000828193810E9467E687FD6BC082E0F5015D
:10F6A00080838B819C818957984F9C838B83B60183
:10F6B00080E090E00E946BE69B01AC01EB81FC8155
:10F6C00060817181828193810E94B2EA9B01AC01C9
:10F6D000F40160817181828193810E94D9EC87FD60
:10F6E00014C00E94FF586B017C019101A8EEB3E0A9
:10F6F0000E94A3EAC60ED71EE81EF91EE981FA8110
:10F70000C082D182E282F38234C00E94FF58E98134
:10F71000FA81C080D180E280F380DC01CB018C19BA
:10F720009D09AE09BF09B7FD24C083E0F5018083C0
:10F730000F3F19F046EA5CE102C049EB5CE16DEC79
:10F740007CE1802F0F900F900F900F90DF91CF9161
:10F750001F910F91FF90EF90DF90CF90BF90AF90EF
:10F760009F908F907F906F905F904F903F902F90E1
:10F7700076CD0F900F900F900F90DF91CF911F914A
:10F780000F91FF90EF90DF90CF90BF90AF909F9040
:10F790008F907F906F905F904F903F902F90089543
:10F7A0004F925F926F927F928F929F92AF92BF9291
:10F7B000CF92DF92EF92FF920F931F93CF93DF933D
:10F7C000CDB7DEB760970FB6F894DEBF0FBECDBFE2
:10F7D00080914907811117C060960FB6F894DEBF7B
:10F7E0000FBECDBFDF91CF911F910F91FF90EF9092
:10F7F000DF90CF90BF90AF909F908F907F906F9051
:10F800005F904F900895DFDB0E94FF584B015C0131
:10F8100060914A0470914B04072E000C880B990BE1
:10F820000E946DE669837A838B839C8344E1C42EB6
:10F83000D12C5CE3E52EF12C00E09E012F5F3F4FC1
:10F840004CE454E067E777E086E797E0B7DEC090E6
:10F850004C04D0904D04E0904E04F0904F04609121
:10F86000340570913505072E000C880B990B0E940A
:10F870006DE69B01AC01C701B6010E94D9EC1816D8
:10F880000CF009C160911E0270911F02072E000C3E
:10F89000880B990B0E946DE69B01AC01C701B60174
:10F8A0000E9467E687FFF7C000914A0410914B045D
:10F8B000B801012E000C880B990B0E946DE6A70180
:10F8C00096010E94B2EA2B013C0120ED3CEC4CE495
:10F8D0005DE36091400770914107809142079091EC
:10F8E00043070E94CCE66D837E838F8398872091A7
:10F8F0006D0730916E0740916F0750917007C701F7
:10F90000B6010E94B2EA9B01AC016D817E818F81BC
:10F9100098850E94CCE66D837E838F83988723E34E
:10F9200033E343E75FE36091690770916A07809171
:10F930006B0790916C070E94CCE69B01AC016D8136
:10F940007E818F8198850E94B3EA6D837E838F8349
:10F9500098876093690770936A0780936B07909309
:10F960006C07C0926D07D0926E07E0926F07F0921D
:10F97000700720E030E040E251E4C301B2010E9490
:10F98000D9EC18160CF431C220E030E040E251EC22
:10F99000C301B2010E9467E687FD2FC2012B09F463
:10F9A0002CC28091680781112CC22091640730918C
:10F9B0006507409166075091670729873A874B870B
:10F9C0005C8720913C0730913D0740913E07509164
:10F9D0003F07C301B2010E94CCE66B017C01A30189
:10F9E000920169857A858B859C850E94B3EA698737
:10F9F0007A878B879C8760936407709365078093F1
:10FA00006607909367072091380730913907409136
:10FA10003A0750913B070E94CCE6A70196010E944D
:10FA2000B3EA2D813E814F8158850E94B2EA6B0175
:10FA30007C0120E030E04FE753E40E94D9EC20E065
:10FA400030E0A90118160CF4E3C1C701B6010E9409
:10FA500067E687FD07C0C701B6010E94F7EB759501
:10FA600067951AC020E030E0A901C301B2010E94ED
:10FA700067E687FF10C0A301920169857A858B85AF
:10FA80009C850E94B2EA6093640770936507809337
:10FA900066079093670760E060934C0780917B074F
:10FAA00090917C07A0917D07B0917E070097A105FA
:10FAB000B10521F1A5019401281B390B4A0B5B0B01
:10FAC00057FD1CC060917F077091800780E090E037
:10FAD0000E946BE69B01AC0160914C0470914D0457
:10FAE00080914E0490914F040E9467E687FF82C187
:10FAF00045E85BE167E97BE180E0B1DB80914407A9
:10FB000090914507A0914607B0914707A501940140
:10FB1000281B390B4A0B5B0B57FD0FC073DAD5015D
:10FB2000C4018C53964FAF4FBF4F809344079093BF
:10FB30004507A0934607B0934707809181079091AE
:10FB40008207A0918307B09184070097A105B105B2
:10FB500011F1881A990AAA0ABB0AB7FC1CC0609165
:10FB600085077091860780E090E00E946BE69B011C
:10FB7000AC016091460470914704809148049091D3
:10FB800049040E9467E687FF20C143E65BE166E720
:10FB90007BE18FEF64DB6091440470914504072E94
:10FBA000000C880B990B0E946DE669837A838B8326
:10FBB0009C8395E0C92ED12C24E1E22EF12C0FEF8D
:10FBC0009E012F5F3F4F46E454E061E777E085E711
:10FBD00097E0F4DCC0904604D0904704E0904804DD
:10FBE000F090490420E030E040EA50E4C701B6015B
:10FBF0000E94D9EC87FDE5C020E030E04CED52E4F6
:10FC0000C701B6010E9467E618160CF4DAC06091CD
:10FC1000440470914504072E000C880B990B0E9438
:10FC20006DE6A70196010E94B2EA4B015C012091AA
:10FC300034073091350740913607509137070E94BD
:10FC4000CCE669877A878B879C8720916007309103
:10FC500061074091620750916307C501B4010E949A
:10FC6000B3EA6D837E838F83988760936007709378
:10FC7000610780936207909363072091300730916A
:10FC8000310740913207509133070E94CCE66D87CF
:10FC90007E878F87988B20ED3CEC4CE45DE3609190
:10FCA0002C0770912D0780912E0790912F070E94AD
:10FCB000CCE62B013C0120915C0730915D0740911F
:10FCC0005E0750915F07C701B6010E94B2EA9B012F
:10FCD000AC01C301B2010E94CCE62B013C0123E33D
:10FCE00033E343E75FE360915807709159078091D0
:10FCF0005A0790915B070E94CCE69B01AC01C301BF
:10FD0000B2010E94B3EA2B013C0160935807709343
:10FD1000590780935A0790935B07C0925C07D09273
:10FD20005D07E0925E07F0925F072D853E854F8567
:10FD3000588969857A858B859C850E94B3EAA301E1
:10FD400092010E94B2EA6B017C0120E030E04FE7B3
:10FD500053E40E94D9EC20E030E0A9011816C4F564
:10FD6000C501B4010E94D9EC181684F4A5019401D0
:10FD70006D817E818F8198850E94B2EA60936007D1
:10FD80007093610780936207909363076FE71AC0CF
:10FD900020E030E0A901C501B4010E9467E687FFB9
:10FDA00010C0A50194016D817E818F8198850E948C
:10FDB000B2EA609360077093610780936207909343
:10FDC000630760E060934D0707CD0E94B776E3CEEE
:10FDD000C701B6010E9467E687FDDACFC701B60109
:10FDE0000E94F7EB75956795EDCF81E080936807EA
:10FDF0006FE752CE80E007D881CE81E0809368071C
:10FE00004ACE1092680719861A861B861C86D9CDA1
:10FE1000C301B2010E94D9EC181654F7A301920154
:10FE200069857A858B859C850E94B2EA6093640718
:10FE30007093650780936607909367076FE72CCEF2
:10FE400090916F00292F227091FF05C090916F0053
:10FE50009D7F90936F0034E0839FC0011124FC01CB
:10FE6000EE57FF4E4081518162817381FC01E55E56
:10FE7000F84F408351836283738381E080931A0734
:10FE8000222329F080916F00826080936F00089593
:10FE9000BC01209118073091190740911807509123
:10FEA00019072417350711F09A01F7CF81E02617BB
:10FEB000370709F080E008958F929F92AF92BF922A
:10FEC000CF92DF92EF92FF921F93CF93DF93C82FD1
:10FED00083ED9BE09093AF098093AE091092EF0BF6
:10FEE00082E090E0A0E0B0E08093D80B9093D90B33
:10FEF000A093DA0BB093DB0B1092AD091092A90915
:10FF00001092AA091092AB091092AC098FEF9FEFE3
:10FF1000DC018093A5099093A609A093A709B0934B
:10FF2000A809CC2379F1C53008F0F8C040E060E0C2
:10FF300070E0CB010E94CBD1882309F4EFC020E10F
:10FF4000C29FC00111248B56984FFC01E254FE4F12
:10FF500020812F7709F0E2C03C9640815181628177
:10FF60007381443651056105710508F4D7C0349793
:10FF7000C080D180E280F380C114D104E104F10497
:10FF800021F4CCC0C12CD12C760140E0C701B601D0
:10FF90000E94CBD1182F882309F4C0C08091B007EC
:10FFA0009091B1078115924009F0B8C0A091B507B2
:10FFB000AA2309F4B3C06091B3077091B407611527
:10FFC000710509F4ABC02091B207222309F4A6C041
:10FFD000A093EA0B2093DC0B80E030E041E050E09E
:10FFE000C82FFA01082E02C0EE0FFF1F0A94E2F795
:10FFF0002E173F0739F08F5FC83091F789E0809363
:020000021000EC
:10000000E50B8CC08093E50B2091BB073091BC07BA
:100010002115310519F040E050E008C02091C907D2
:100020003091CA074091CB075091CC072093DD0B4C
:100030003093DE0B4093DF0B5093E00B46015701EA
:10004000860E971EA11CB11C8092EB0B9092EC0BBC
:10005000A092ED0BB092EE0BE091B607F091B707CE
:10006000F093F10BE093F00BB0E00E9493EA860E60
:10007000971EA81EB91E8092F20B9092F30BA092CD
:10008000F40BB092F50B85E0EE0FFF1F8A95E1F7B8
:10009000E150FE4FEF2FFF27E6958E0E9F1EA11C0D
:1000A000B11C8092E60B9092E70BA092E80BB09205
:1000B000E90B2091B8073091B9072115310521F0DE
:1000C000A90160E070E008C04091C5075091C607E3
:1000D0006091C7077091C807D701C60188199909AF
:1000E000AA09BB09840F951FA61FB71F04C0B695A8
:1000F000A79597958795CA95D2F78093E10B909332
:10010000E20BA093E30BB093E40B853F2FE0920743
:10011000A105B10528F48CE08093EF0B10E01AC024
:10012000853F9F4FA105B10510F480E111C080917A
:10013000D1079091D207A091D307B091D4078093B3
:10014000F20B9093F30BA093F40BB093F50B80E2BA
:100150008093EF0B812FDF91CF911F91FF90EF9054
:10016000DF90CF90BF90AF909F908F900895682FB1
:100170008AE99FE00C94E14ACF92DF92EF92FF92DE
:100180001F93CF93DF931092320A8091650A8823E0
:1001900021F082E69AE00E9409991092D70B109202
:1001A000D40B85E38093D30B0E94FF58EB01A895F5
:1001B00061E08091D30B0E9437B683ED9BE00E94F3
:1001C0006A9A2398229A219A209A289A85E0809305
:1001D000D50B82E58CBD1DBC1AE08FEF0E946F9A93
:1001E0001150D9F720E030E0A90160E083ED9BE0F9
:1001F0000E94749A182F8093D60B813049F00E9488
:10020000FF586C1B7D0B613D774060F381E054C06B
:100210002AEA31E040E050E068E083ED9BE00E9494
:10022000749A82FF03C01093D70B0EC014E00E9493
:10023000829F8093D60B1150D1F78A3A11F082E059
:100240003BC082E08093D70B8091D70B823021F0A6
:10025000C12CD12C760105C0C12CD12CE12C80E41D
:10026000F82E20E030E0A90167E383ED9BE00E94D7
:10027000749AA701960169E283ED9BE00E94749A4B
:100280008093D60B882349F00E94FF586C1B7D0B8E
:10029000613D774030F38AE00FC08091D70B823008
:1002A00011F520E030E0A9016AE383ED9BE00E94B4
:1002B000749A882351F088E08093D40B83ED9BE0FF
:1002C0000E946A9AE6EEFDE119C00E94829F807C3E
:1002D000803C19F483E08093D70B0E94829F0E9498
:1002E000829F0E94829F83ED9BE00E946A9A1092F7
:1002F000D50B81E0E1DD811131C015C08491EF01A2
:100300002196882321F00E94EE93FE01F7CFE8EDBD
:10031000FDE18491EF012196882309F456C00E94E3
:10032000EE93FE01F6CF80E0C7DD811117C0E1ED4D
:10033000FDE18491EF012196882321F00E94EE9344
:10034000FE01F7CFEDEBFDE18491EF0121968823CB
:1003500009F43BC00E94EE93FE01F6CF68ED7BE00E
:1003600082E69AE00E94B698811116C0E1EDFDE1A7
:100370008491EF012196882321F00E94EE93FE01E3
:10038000F7CFECEAFDE18491EF0121968823E9F0B3
:100390000E94EE93FE01F7CF81E08093320AE6EEF1
:1003A000FDE18491EF012196882321F00E94EE93D4
:1003B000FE01F7CFE0EAFDE18491EF012196882369
:1003C00021F00E94EE93FE01F7CF8BE1E2E6FAE026
:1003D000A1E8BAE001900D928A95E1F78091600A58
:1003E0009091610A9093800A80937F0ADF91CF9168
:1003F0001F91FF90EF90DF90CF90089580913F0E76
:10040000823041F48BE89DE19093A4078093A30789
:100410000E941A940E94FF586093430E7093440EFA
:100420008093450E9093460E8091320A882319F0EE
:1004300081E08093310A81E080933F0E0895CF934D
:10044000DF931092310A83E080933F0E80918C0EEF
:100450008823B1F0E3E8FDE18491EF01882341F0C6
:10046000082E000C990B83DE2196FE018491F6CFB5
:100470008DE090E07CDE8AE090E0DF91CF9177CE56
:10048000E7E8FDE18491EF01882391F3082E000C49
:10049000990B6DDE2196FE018491F6CF8F929F928B
:1004A000AF92BF92CF92DF92EF92FF920F931F9382
:1004B000CF93DF9300D01F92CDB7DEB7FC018381CD
:1004C000813079F5818181FF2CC081899289A3894E
:1004D000B489892B8A2B8B2B09F448C07F0140E01B
:1004E00050E0BA01CF010E941F988823D1F0F70194
:1004F00085889688A788B08CC18CD28C82E090E0E9
:10050000A0E0B0E0F60180839183A283B3839E01D3
:100510002F5F3F4FB501A401C6010E9494D2811103
:1005200002C080E03CC000E010E09801B501A401E9
:10053000C6010E9403D28823A1F389809A80AB80F0
:10054000BC80F6018789803141F4F8EF8F16FFEF08
:100550009F06A104B10460F4DACF88EF88168FEF0C
:100560009806A8068FE0B80618F4D1CF81E017C02E
:10057000F701158A168A178A108E118A128A138A31
:10058000148A818180688183C7010E94E2D3882315
:1005900041F240E050E0BA01C7010E941F980F905D
:1005A0000F900F900F90DF91CF911F910F91FF90BF
:1005B000EF90DF90CF90BF90AF909F908F90089575
:1005C0001092340A1092310A8091FD0B882321F099
:1005D0008AEF9BE00C94099908952F923F924F92D5
:1005E0005F926F927F928F929F92AF92BF92CF92C3
:1005F000DF92EF92FF920F931F93CF93DF93CDB7CC
:10060000DEB7C257D1090FB6F894DEBF0FBECDBF1B
:100610008C013B014A014DB75EB7E1965FAF4EAF2B
:10062000E197AD961FAEAD971B0154E0250E311C2E
:100630007E018FE5E80EF11C9DEE492E92E0592EC9
:10064000E0E4F0E0EC0FFD1F3496E396FFAFEEAF71
:10065000E397F3018781823008F462C18485958530
:10066000A685B7858F719927AA27BB27892B8A2B47
:100670008B2B09F055C11092420A42E45AE0BE01A8
:100680006F5F7F4FC1010E947AD318160CF048C1EA
:100690008C85982F9871903129F42091AF0C2150BE
:1006A000223078F42981222309F43AC1253E89F2C7
:1006B0002E3279F22091420A2E3259F28A7049F68E
:1006C000B8C04DB75EB7AF965FAF4EAFAF97BE0144
:1006D0006F5F7F4FC7010E9475D10115110521F091
:1006E000F801808181119BC021E081E090E0F70159
:1006F00001900020E9F73197EE19FF098E0F9F1F37
:1007000002964DB75EB7481B590B0FB6F8945EBF03
:100710000FBE4DBF8DB79EB701965C01211102C07F
:10072000B80102C062E273E0C5010E9417EEB70192
:10073000C5010E94F8ED62E273E0C5010E94F8ED88
:1007400025961FAE259728961FAE289724961FAE94
:100750001EAE249722965FAE4EAE229721E0A701EF
:10076000B101E3968EAD9FADE3970E94959E8111F6
:100770002AC08091AF0C811126C0E6EEFDE1849184
:100780006F019FEFC91AD90A882321F00E94EE93C6
:10079000F601F5CFEFE6FDE184916F012FEFC21A6C
:1007A000D20A882321F00E94EE93F601F5CF67016B
:1007B000F60181916F01882319F00E94EE93F8CF22
:1007C0008AE00E94EE938BE1FE01EC5BFF4FDE01BD
:1007D000959601900D928A95E1F724968EAD9FAD86
:1007E00024979CA38BA35AA249A240E050E0BE01EB
:1007F0006F5D7F4FC501F1DECE0181960E94C2A0E0
:10080000CE01805C9F4F0E94C2A0AF964EAD5FADFF
:10081000AF970FB6F8945EBF0FBE4DBF1ACFF80169
:1008200001900020E9F73197CF01801B910B20E068
:100830005ECF81E0903109F080E08093330A9031FF
:1008400041F08985873409F004CF8A858E3709F411
:1008500000CF8091AF0C813029F08230D9F1811125
:10086000F8CE0AC08091B00C9091B10C0196909393
:10087000B10C8093B00CEDCEBE016F5F7F4F85E36E
:100880009AE00E9475D10115110529F485E3C82E5F
:100890008AE0D82E09C06801F60181916F01882392
:1008A000A9F30E94EE93F8CFF60181916F0188239E
:1008B00019F00E94EE93F8CF80E20E94EE936D8DC6
:1008C0007E8D8F8D98A14AE00E940F978AE00E944A
:1008D000EE93BFCEBE016F5F7F4F85E39AE00E942B
:1008E00075D18114910441F065E37AE0C4010E945E
:1008F000E5ED892B69F414C0AD96FFADAD978F2F50
:1009000090E02091BC0F3091BD0F8217930741F00A
:10091000AD962FADAD972F5FAD962FAFAD9799CE1A
:10092000E1968EAD9FADE1970FB6F8949EBF0FBED6
:100930008DBFCE58DF4F0FB6F894DEBF0FBECDBFD0
:10094000DF91CF911F910F91FF90EF90DF90CF90AB
:10095000BF90AF909F908F907F906F905F904F90DF
:100960003F902F9008950F931F93CF93DF93CDB7B0
:10097000DEB76F970FB6F894DEBF0FBECDBF8B0109
:1009800022E02093AF0C9093BD0F8093BC0F81E8C1
:100990009AE00E94669A8BE1E1E8FAE0DE011596A2
:1009A00001900D928A95E1F780917F0A9091800ADB
:1009B0009C838B838DEE92E09A838983A801BE018C
:1009C0006F5F7F4F80E090E008DECE0101960E94CD
:1009D000C2A06F960FB6F894DEBF0FBECDBFDF91F9
:1009E000CF911F910F9108952F923F924F925F9256
:1009F0006F927F928F929F92AF92BF92CF92DF922F
:100A0000EF92FF920F931F93CF93DF93CDB7DEB793
:100A10006F970FB6F894DEBF0FBECDBF6C012DB639
:100A20003EB61D8218861C821B828DEE92E09A8350
:100A30008983FB0180819E012F5F3F4F39018F32F7
:100A400041F08DE79AE0F60191838083F62E172F0F
:100A500064C08EE59AE0F601918380838B010F5F7D
:100A60001F4F0115110509F456C04DB65EB66FE271
:100A700070E0C8010E9403EE4C010817190708F046
:100A800048C07C01E01AF10AFF24C70101962DB786
:100A90003EB7281B390B0FB6F8943EBF0FBE2DBFD3
:100AA0008DB79EB701965C01A701B8010E942CEE9C
:100AB000F501EE0DFF1D1082F60160817181611557
:100AC000710511F06C5F7F4F21E0A501CE01059605
:100AD0000E94959E811111C0B5018BE59DE10E9498
:100AE00097C58EE20E94EE938AE00E94EE930FB6C5
:100AF000F8945EBE0FBE4DBE0EC0F60171826082DC
:100B000084010F5F1F4F0FB6F8945EBE0FBE4DBE3F
:100B1000A8CFF02E02C0F12C10E0C3010E94C2A0A9
:100B20008F2D912F0FB6F8943EBE0FBE2DBE6F963F
:100B30000FB6F894DEBF0FBECDBFDF91CF911F91EE
:100B40000F91FF90EF90DF90CF90BF90AF909F906C
:100B50008F907F906F905F904F903F902F9008956F
:100B6000CF92DF92EF92FF920F931F93CF93DF9379
:100B700088E50E944F4CD82E89E40E944F4CC82E25
:100B8000882319F00E94E84B1CC0DD20C1F00E94B0
:100B9000184C20E030E040E251E40E94B2EA20E04C
:100BA00030E048EC51E40E94B3EA2AE037ED43EA32
:100BB0005CE30E94CCE60E94F7EB653010F01FEF7B
:100BC00001C0162F89E50E944F4C082F8AE40E942D
:100BD0004F4CC82F882319F00E94E84B1CC00023FB
:100BE000C1F00E94184C20E030E040E251E40E9445
:100BF000B2EA20E030E048EC51E40E94B3EA2AE097
:100C000037ED43EA5CE30E94CCE60E94F7EB6530E7
:100C100010F0DFEF01C0D62F8AE50E944F4CE82E7E
:100C2000811105C081E50E944F4CF82E01C0F12CC6
:100C3000C11001C0C0E02C2F30E0D11001C000E095
:100C4000200F311D2130310521F4E1101AC0F110BF
:100C500018C0E1EDFDE18491EF012196811103C0FF
:100C6000E7E9F0E204C00E94EE93FE01F4CF849124
:100C7000EF012196882309F455C00E94EE93FE01EE
:100C8000F6CF17FD02C0D7FF17C0E1EDFDE184915B
:100C9000EF012196811103C0E8E7F0E204C00E9451
:100CA000EE93FE01F4CF8491EF0121968823D1F1D8
:100CB0000E94EE93FE01F7CF0E94184C9B01AC01FD
:100CC000012F110F110BAD2FDD0FBB0BFF2099F082
:100CD00085E0809FF001819FF00D1124EA0FFB1F3A
:100CE000EE0FFF1FEE0FFF1FEA53FF4E6081718171
:100CF0008281938103C060E070E0CB01E5E0E09F7A
:100D0000E001E19FD00D1124CA0FDB1FCC0FDD1FC6
:100D1000CC0FDD1FCA53DF4E0E94B3EA688379838C
:100D20008A839B83DF91CF911F910F91FF90EF906A
:100D3000DF90CF90089580916F00982F927081FF7F
:100D400005C080916F008D7F80936F008091B40902
:100D50008093B3098093B2098093B10984E68093AC
:100D6000B00928EE33E030934B0720934A079923CC
:100D700029F080916F00826080936F0081E0809302
:100D80001A070E941F6A0E94D3C980917C10882391
:100D900021F084EA98E10E948FC68CE0E4EAF8E151
:100DA000A2E3B4E001900D928A95E1F70C94A2932E
:100DB0002F923F924F925F926F927F928F929F926B
:100DC000AF92BF92CF92DF92EF92FF920F931F9359
:100DD000CF93DF93CDB7DEB7CD54D1090FB6F894DA
:100DE000DEBF0FBECDBF85E40E94984C882321F062
:100DF0000E94E84B7B0102C0E12CF12C83E40E94AD
:100E0000984C882321F00E94E84B6AA302C005E0B9
:100E10000AA385E50E94984C882319F00E94094C8A
:100E200003C085E50E944F4C8CA7F7FC07C0812CBE
:100E3000912C16E1A12E13E4B12E06C0812C912C29
:100E4000BCE8AB2EB2E4BB2E83E50E94984C88230D
:100E500021F00E94184C4B015C01E114F10411F4E3
:100E600010924E0710923F10ED820E94FF582B0106
:100E70003C011D8117FF05C00CE310E022E029832F
:100E800004C003E210E035E03983D301C2018C5382
:100E9000964FAF4FBF4F8093440790934507A09361
:100EA0004607B093470761E06E0D623080F0E5EED3
:100EB000FFE184918F010F5F1F4F1A8309838823FD
:100EC00009F45FC30E94EE93E981FA81F2CFEFE06B
:100ED000F0E284917F012FEFE21AF20A882321F0D9
:100EE0000E94EE93F701F5CF0E9410793D8137FF04
:100EF00004C08FE780934D0708C04D81E42F440F55
:100F0000FF0BE45BF84F8FE78083C501B4010E94BB
:100F1000F7EB072E000C880B990B0E946DE66A8791
:100F20007B878C879D878981482F50E09801A8EEA8
:100F3000B3E00E94A3EA6DA77EA78FA798AB8B01B1
:100F40009C01040D151D261D371D0AAF1BAF2CAFCC
:100F50003DAF81E0809320021D811F3F39F40FE4F3
:100F60001FE11FAF0EAF09E11FE106C00DE31FE156
:100F70001FAF0EAF06E01FE122961FAF0EAF229704
:100F80004CA25DA26EA27FA249AA5AAA6BAA7CAA11
:100F90001DAA1EAA1FAA18AE19AE188E10E4198F2A
:100FA0000CE10A8F16E41B8F1C8E1D8E1E8E1F8E69
:100FB0001C8A1D8A1E8A1F8A188A198A1A8A1B8A05
:100FC00019821A821B821C828FE790E0A0E0B0E0B9
:100FD0008E839F83A887B987FFE7CF2ED12CE12C82
:100FE000F12C18A619A61AA61BA611E01F861E86AC
:100FF0002D961FAE2D97212C312C2E961FAE2E979D
:101000000D81802F000F990B9C01245B384F249693
:101010003FAF2EAF2497880F991F880F991FDC01CF
:10102000A45BBB4FB9A3A8A3CA01052E000CAA0B51
:10103000BB0B28968CAF9DAFAEAFBFAF28974C5F70
:101040005F4FCA01550FAA0BBB0B2C968CAF9DAFFF
:10105000AEAFBFAF2C97AAA10A2E000CBB0BBBA34F
:10106000AAA380912002882309F489C20E94FF5814
:101070004B015C0180914907882309F4D4C00E9488
:10108000E3770D8107FD0CC0A8A1B9A1BC912D96F5
:10109000BFAF2D97E8A1F9A12180328003810BC059
:1010A000009146042D960FAF2D9720904704309065
:1010B0004804009149042E960FAF2E972D962FAD20
:1010C0002D97322D432D2E965FAD2E976C8D7D8DF5
:1010D0008E8D9F8D0E9467E687FF0AC02D960FAD0B
:1010E0002D970C8F2D8E3E8E2E960FAD2E970F8F37
:1010F000288D398D4A8D5B8D2D966FAD2D97722D74
:10110000832D2E969FAD2E970E9467E687FF0AC01B
:101110002D960FAD2D97088F298E3A8E2E960FADF6
:101120002E970B8F8091440790914507A091460719
:10113000B0914707A5019401281B390B4A0B5B0BA3
:1011400057FD10C00E940278D501C4018C53964F00
:10115000AF4FBF4F8093440790934507A093460736
:10116000B09347072D962FAD2D97322D432D2E96F8
:101170005FAD2E976A857B858C859D851123E9F16E
:101180000E9467E687FF4FC0B501A40144195509C5
:1011900066097709DB01CA0188589341A109B109A1
:1011A000B7FD41C0D701C6010E811F812885398551
:1011B000801B910BA20BB30B1D81B595A79597953D
:1011C000879517FF03C080934D0705C02496EEADA9
:1011D000FFAD2497808348A759A76AA77BA70A85F4
:1011E0000C8F1B851D8F0C850E8F1D851F8F8CA26C
:1011F0009DA2AEA2BFA210E016C00E94D9EC1816A4
:1012000094F4D501C4012CA13DA14EA15FA1821B84
:10121000930BA40BB50BAC01BD01485853416109B8
:10122000710977FFCBC120E030E040EA51E46A85E4
:101230007B858C859D850E94B3EA2D962FAD2D97D9
:10124000322D432D2E965FAD2E970E9467E687FFC5
:1012500010C0E1E7FFE184918F010F5F1F4F1A83F8
:101260000983882309F48BC10E94EE93E981FA81F6
:10127000F2CFD501C40129A93AA94BA95CA9821BC7
:10128000930BA40BB50BB7FD96C00E94FD758AE0C9
:101290000E94EE93D501C4018053984FAF4FBF4FCA
:1012A00089AB9AABABABBCAB0DA9011163C02EA946
:1012B0003FA948AD59AD2D966FAD2D97722D832D59
:1012C0002E969FAD2E970E94D9EC18160CF041C0B7
:1012D00028966CAD7DAD8EAD9FAD28970E946DE6D2
:1012E0002D962FAD2D97322D432D2E965FAD2E9737
:1012F0000E94B3EA6EAB7FAB88AF99AF2DA53EA538
:101300004FA558A9280D391D4A1D5B1D2AAF3BAFBB
:101310004CAF5DAF2C966CAD7DAD8EAD9FAD2C9777
:101320000E946DE69B01AC016A857B858C859D855D
:101330000E94B2EA2D962FAD2D97322D432D2E9679
:101340005FAD2E970E9467E6881F8827881F8DABA8
:1013500032C0D501C4012AAD3BAD4CAD5DAD821BA1
:10136000930BA40BB50BB7FD26C04EAD5FAD62E687
:101370007FE11EC020E030E040EA51E46A857B85D1
:101380008C859D850E94B2EA9B01AC012D966FADC4
:101390002D97722D832D2E969FAD2E970E9467E676
:1013A00087FF09C022964EAD5FAD22976DE27FE1C7
:1013B0008D810E942F79D501C401880F991FAA1F22
:1013C000BB1F2CA13DA14EA15FA1821B930BA40BBF
:1013D000B50B84199509A609B70981389F44A24124
:1013E000B10580F0E8EEFEE184918F010F5F1F4FA1
:1013F0001A830983882309F4C2C00E94EE93E9810D
:10140000FA81F2CF2AA13BA14E855F8524173507CB
:101410000CF027CEEBE8FEE184918F010F5F1F4FA8
:101420001F830E83882329F00E94EE93EE81FF81B3
:10143000F3CF1D8117FD03C006E113E002C000EFEA
:1014400013E01F830E836E817F818AE79EE10E94F5
:1014500097C549815A816B817C8186E79EE10E9414
:1014600061C58AE00E94EE936E817F8185E69EE1F0
:101470000E9497C5488959896A897B8981E69EE1DE
:101480000E9461C58AE00E94EE936E817F8180E5B3
:101490009EE10E9497C54C895D896E897F898CE4A5
:1014A0009EE10E9461C58AE00E94EE931CA5112373
:1014B00009F467C00D8107FF31C029813A814B8152
:1014C0005C8120933407309335074093360750935F
:1014D00037072CEA35EC47E25EE3688979898A8927
:1014E0009B890E94CCE6609330077093310780930C
:1014F0003207909333072CEA35EC47E25EE36C89C0
:101500007D898E899F890E948FEB60932C07709351
:101510002D0780932E0790932F0733C089819A81DE
:10152000AB81BC8180933C0790933D07A0933E071D
:10153000B0933F072CEA35EC47E25EE3688979898E
:101540008A899B890E94CCE660933807709339079B
:1015500080933A0790933B072CEA35EC47E25EE331
:101560006C897D898E899F890E948FEB60934007EB
:1015700070934107809342079093430702C00E94F3
:10158000107981E080933F10C35BDF4F0FB6F89472
:10159000DEBF0FBECDBFDF91CF911F910F91FF90A6
:1015A000EF90DF90CF90BF90AF909F908F907F9003
:1015B0006F905F904F903F902F9008950E851F85FC
:1015C000012B09F42BC148A459A46AA47BA4480E9A
:1015D000591E6A1E7B1E28A539A54AA55BA5281B96
:1015E000390B4A0B5B0B6E817F81888599850E9440
:1015F00046EAA30192010E9477EADA01C9018C0D43
:101600009D1DAE1DBF1D84319105A105B105FCF0E6
:101610006C017D018C3E9105A105B1052CF05BEEBE
:10162000C52ED12CE12CF12C20E8C216D104E10406
:10163000F104DCF08EEF90E0A0E0B0E08C199D09A1
:10164000AE09BF098E839F83A887B98712C044E182
:10165000C42ED12CE12CF12C04E110E020E030E08C
:101660000E831F832887398704C0CE82DF82E886F5
:10167000F986EDEDFFE184918F010F5F1F4F882305
:1016800021F00E94EE93F801F6CFC701B6010E9447
:101690007A97E8EDFFE184918F010F5F1F4F882358
:1016A00021F00E94EE93F801F6CF6E817F8188854C
:1016B00099850E947A97488D598D6A8D7B8D81ED31
:1016C0009FE10E9461C54C8D5D8D6E8D7F8D8AEC92
:1016D0009FE10E9461C50E851F85033011050CF442
:1016E0009DC06E817F81888599850E946DE620E08E
:1016F00030E040E850E40E94CCE669837A838B8333
:101700009C83288D398D4A8D5B8D6C8D7D8D8E8D62
:101710009F8D0E94B2EA2BED3FE049E450E40E9425
:10172000CCE620E030E040E05FE30E94CCE69B01A5
:10173000AC0169817A818B819C810E948FEB6983E6
:101740007A838B839C83C301B2010E946DE62FE6EE
:1017500032E143E85AE30E94CCE62B013C01498187
:101760005A816B817C8184EC9FE10E9461C5B30149
:10177000A2018EEB9FE10E9461C52AE939E949E1A6
:101780005FE369817A818B819C810E94CCE66983C9
:101790007A838B839C839B01AC010E94B3EAA301F3
:1017A00092010E948FEB688B798B8A8B9B8B2981AE
:1017B0003A814B815C81C301B2010E94CCE620E0FA
:1017C00030E040E05EE30E94CCE66C8B7D8B8E8B3C
:1017D0009F8BEEEAFFE184918F010F5F1F4F8823FB
:1017E00019F0FCD7F801F7CF49815A816B817C81D0
:1017F00088EA9FE10E9461C5488959896A897B8985
:1018000082EA9FE10E9461C54C895D896E897F896A
:101810008CE99FE10E9461C58AE0E0D78E819F81BB
:10182000A885B9858C0D9D1DAE1DBF1D1D81B5956B
:10183000A7959795879517FF03C080934D0705C01F
:101840002496EEADFFAD249780830E851F850F5F34
:101850001F4F1F870E871A85188F0B85098F1C85D0
:101860001A8F0D850B8F2401350111E0DCCCCF934D
:10187000DF93E6EEFDE18491EF012196882319F0D4
:10188000ADD7FE01F8CF83E50E944F4C882321F0AD
:101890000E94094C80935202ECE3FEE18491EF0137
:1018A0002196882319F09AD7FE01F8CF8091520231
:1018B000811103C0E8E3FEE102C0E4E3FEE18491AC
:1018C000EF012196882319F089D7FE01F8CFECE2C9
:1018D000FEE18491EF012196882319F07FD7FE0164
:1018E000F8CF2091140430911504409116045091C2
:1018F0001704609198187091991880919A18909196
:101900009B180E94B3EAAB01BC018AE29EE10E94EF
:1019100061C5209118043091190440911A04509126
:101920001B0460919C1870919D1880919E18909155
:101930009F180E94B3EAAB01BC0187E29EE10E94BE
:1019400061C520911C0430911D0440911E045091EA
:101950001F046091A0187091A1188091A218909115
:10196000A3180E94B3EAAB01BC0184E29EE10E948D
:1019700061C5ECE1FEE18491EF012196882319F025
:101980002DD7FE01F8CF2091140430911504409119
:10199000160450911704609146027091470280919D
:1019A0004802909149020E94B3EAAB01BC018AE16E
:1019B0009EE10E9461C52091180430911904409164
:1019C0001A0450911B0460914A0270914B0280915D
:1019D0004C0290914D020E94B3EAAB01BC0187E139
:1019E0009EE10E9461C520911C0430911D0440912C
:1019F0001E0450911F0460914E0270914F0280911D
:101A00005002909151020E94B3EAAB01BC0184E103
:101A10009EE10E9461C58AE0DF91CF91DFC6FF920F
:101A20000F931F93CF93DF93F82E092F162FEFE01C
:101A3000FEE18491EF012196882319F0CFD6FE01B3
:101A4000F8CFEF2DF02F8491EF012196882319F024
:101A5000C5D6FE01F8CFEDE0FEE18491EF012196BD
:101A6000882319F0BBD6FE01F8CF612F70E080E02B
:101A700090E00E947A978AE0DF91CF911F910F91B9
:101A8000FF90ACC64F925F926F927F928F929F921F
:101A9000AF92BF92CF92DF92EF92FF92CF93DF93FC
:101AA00020911404309115044091160450911704AC
:101AB0006091320470913304809134049091350424
:101AC0000E94B3EAAB01BC018AE09EE10E9461C5BD
:101AD000209118043091190440911A0450911B046C
:101AE00060913604709137048091380490913904E4
:101AF0000E94B3EAAB01BC0186E09EE10E9461C591
:101B000020911C0430911D0440911E0450911F042B
:101B100060913A0470913B0480913C0490913D04A3
:101B20000E94B3EAAB01BC0182E09EE10E9461C564
:101B300040913E0450913F046091400470914104F3
:101B40008EEF9DE10E9461C580916F00982F927089
:101B500081FF05C080916F008D7F80936F00409062
:101B60008210509083106090841070908510809047
:101B7000861090908710A0908810B0908910C09027
:101B80008A10D0908B10E0908C10F0908D109923DB
:101B900029F080916F00826080936F00E4EFFDE197
:101BA0008491EF012196882319F018D6FE01F8CF11
:101BB000C301B2010E947A97E0EFFDE18491EF0149
:101BC0002196882319F00AD6FE01F8CFC501B40189
:101BD0000E947A97ECEEFDE18491EF012196882333
:101BE00019F0FCD5FE01F8CFC701B6010E947A9723
:101BF0008AE0DF91CF91FF90EF90DF90CF90BF9080
:101C0000AF909F908F907F906F905F904F90E6C5C0
